:020000040800F2
:1050000008460020D550000871D100088FC700085D
:105010000000000000000000000000000000000090
:1050200000000000000000000000000051DE000849
:10503000000000000000000091D10008C5F3000846
:10504000E7500008E7500008E7500008E750000864
:10505000E7500008C3770008E7500008CD77000844
:1050600000000000E7500008CD760008E576000853
:10507000E750000821CB0008D5060108E7500008DA
:10508000E7500008E7500008E75000080000000063
:10509000E7500008E7500008E7500008E750000814
:1050A000E7500008E7500008E7500008B50601087F
:1050B000C506010855CC00080000000000000000F3
:1050C0000348854600F0DEFC004800470D18010843
:1050D000084600200448804704480047FEE7FEE7F2
:1050E000FEE7FEE7FEE7FEE789F40008C15000088E
:1050F00030B50B46014600202022012409E00D4670
:10510000D5409D4205D31D469540491B25469540F7
:1051100040191546521E002DF1DC30BD70B500243B
:105120002546002801DA01244042002901DA012540
:105130004942FFF7DDFFAC4200D04042002C00D0D6
:10514000494270BDF0B51FB40646002082B0054646
:105150004024019100901BE0019922460F46304601
:1051600000F020F8049A059B801A994110D310464C
:105170001946224600F018FB361A8F410197224645
:1051800001200021009F00F00FFB38184D410090D6
:105190002046641E0028DFDC019B00982946324629
:1051A00007B0F0BD10B5202A04DB0846203AD040F5
:1051B000002110BD0B46D340D0402024A21A9140BC
:1051C0000843194610BD03460B439B0703D009E073
:1051D00008C9121F08C0042AFAD203E00B78037032
:1051E000401C491C521EF9D27047D2B201E0027035
:1051F000401C491EFBD270470022F6E710B513464B
:105200000A4604461946FFF7F0FF204610BD421E2D
:105210005378521C002BFBD10B781370491C521C85
:10522000002BF9D1704730B505462A460B46107859
:105230001C78521C5B1C002801D0A042F7D0002C27
:1052400003D0002802D06D1CEFE7284630BDCAB25B
:10525000401E4178401C8A4202D00029F9D100202A
:105260007047421C0178401C0029FBD1801A70470E
:1052700010B5002200E0521C835C8C5CA34201D17B
:10528000002BF8D1D8B2E1B2401A10BD30B50446B7
:105290000020034600E05B1C934203D2E05CCD5C3F
:1052A000401BF8D030BD03460A780270401C491CF0
:1052B000002AF9D11846704730B50546002003464C
:1052C00000E05B1C934205D2EC5CC85C201A01D163
:1052D000002CF6D130BD70B506460BF09BFD04687E
:1052E00005460A220021304600F0D4FA2C6070BD39
:1052F00070B502464A40D50F40004A00ED0740080D
:105300005208002814D0002A12D0C40DD30D410237
:105310000120C0055202490A520AE41A091812185B
:105320007D34914201D3641C00E04900002C01DA75
:10533000002070BD0023914201D3891A0343400825
:1053400049000028F7D100290AD0914202D1012159
:10535000C90705E0914201D2012101E00121C943C1
:10536000E005C018401900F0CDFA70BDF0B5074651
:105370000846584087B0C00F049048000E465900B8
:1053800040084908BC1A884105D2384631461E46B5
:1053900017460B4602465800400810434CD0300DCB
:1053A000039040055900400D490D0590401A0290A8
:1053B000402872DA18030121000B09050843019007
:1053C00004980092002805D001995242002088419B
:1053D00000920190029840210A1A0199009800F069
:1053E000E3F905460C466B4607CB00F0EDF9C01912
:1053F0007141039A0E0D0023D71756401A467A4082
:10540000164344D0049A002A2DD0029A012A039A06
:1054100015DC1205C01A914101263605001C7141A8
:10542000D20F059ED2070093019202962A46234688
:1054300000F0B6FA07B0F0BD38463146FAE7160577
:10544000224A0F46B218C01AB74101210905001CB3
:105450004F4100187F41114618187941E20F10435F
:105460006D19644113E0E2076D0815436408C20733
:105470001443039A01261205C01A91413605001CF7
:105480007141CE07400830434908C01851412A46AF
:10549000234600F078FACDE7FFE7049801224000A8
:1054A000C117121A00238B4104983146C417381AC9
:1054B000A141EEE730B40124E407634030BC55E776
:1054C00030B40124E407614030BC4FE70000E0FF46
:1054D000F0B51FB488B00B99099800244840099989
:1054E000C00F490049080991C0070B990090490075
:1054F00049080B9109990898A64608431CD00B99B6
:105500000A98084318D0099801244000420D480029
:10551000410D099824050003000B204309900B98C6
:105520000003000B20430B9050181C494018002228
:1055300001901446104605E0002001460DB0F0BD74
:10554000032801DA034600E003239C46C11A0AAE91
:105550000AE05F0008ADED5B4F00F75B7D4300277D
:10556000AA187C41491C5B1E6145F2DD410004AB79
:105570005A522104120C0A43240C401C0828DFDB79
:10558000019802900099704601910090059B049A41
:105590000799069800F004FAD0E700000DFCFFFF21
:1055A000F0B50C465C4085B0E40FE40703944C0072
:1055B0000026640859009446490802460296224390
:1055C00021D062460A431ED06200570D4A000E03E6
:1055D0002303550D012402462C492405781B1B0B7F
:1055E000360B401823432643614600901C46501A50
:1055F000B44103D30098401C009002E09218009838
:105600005B41002803DA0020014605B0F0BD002010
:10561000012109050746864611E064461D46141B14
:10562000B54106D36546521BB341744607430C434C
:10563000A646CD0740084908284392185B41054615
:105640000D43EAD11046184313D060461946504026
:105650007140084306D06046101AB34106D20122B9
:10566000002306E000220123DB0702E00122D243EF
:105670005310009874460105381C6141029C039D3B
:105680000019694100F07FF9BFE70000FD03000049
:1056900010B500229623114600F03CF910BD000021
:1056A0000EB505490291002100910A460B46019171
:1056B00000F076F903B000BD330400004100400261
:1056C0000122400AD205090E80187F2901DA002044
:1056D0007047962903DC9622511AC84070479639C4
:1056E000884070474A0009030123090B1B05194331
:1056F000094B10B5520D9A4201DA002010BD064B3D
:1057000034339A4203DC9A1AFFF74CFD10BD03496B
:105710005118884010BD0000FF030000CDFBFFFFC3
:10572000C20FD207400040080BD0C10D0723DB0198
:10573000C91840020905400A1143C2084007114335
:10574000704700200146704710B5002904DB012492
:10575000E40740428C412146002B04DB1C46012318
:10576000DB075242A341994200D1904210BD000094
:10577000CB0FDB07490010B5490802460A4307D0A2
:105780000A0D07240903E401090B121B002A01DC9E
:10579000002010BDC900440F0C43C100E018D20521
:1057A000801800F0AFF810BD10B5202A04DB0146C8
:1057B000203A9140002010BD914020239C1A0346BE
:1057C000E3401943904010BD10B5202A06DBCB17EB
:1057D0000846203A1041C1170B4306E00B4613411F
:1057E000D0402024A21A91400843194610BD000061
:1057F0000FB400B589B00CA900910B990023CB60C0
:10580000204B214A06930792042201921F4A0292DA
:105810001F4A089202466B46002000F0E2F909B0E8
:1058200008BC04B0184770B586B006460020C043D7
:105830000190002015460C460091029104903246DA
:10584000694604A8FFF7D4FF024604982118002DEA
:1058500005D0002801D0084600E0204628600498C2
:1058600000280DD0002A02DD0098884208D0081BCD
:105870000190009432466946029404A8FFF7B8FFED
:1058800006B070BD395E0008595E0008FFFFFF7F5B
:10589000B15A0008F7B5009C0F4600262578641C15
:1058A000002D05D000F000F90068405DC007F5D17B
:1058B0002B2D02D02D2D18D0641E39462046029A79
:1058C00000F0DCFA002F04D03968A14201D1009920
:1058D00039607105022400290BDA4042002803DDFB
:1058E0000BF098FA0460A007FEBD01208002064379
:1058F000E3E70028F8DA0BF08DFA04600048FEBDFB
:10590000FFFFFF7F002904DA401C490001D1400855
:105910004000704770B40024050C05D11024000429
:1059200002D1002921D01124050E01D10002083432
:10593000050F01D10001241D850F01D18000A41C99
:10594000002801DB4000641C002908D020252E1B04
:105950000D46F540A14000D001212943084301062E
:105960001B1B000ADB1D02D5002070BC7047DB0545
:10597000181880180029F8DA401C4900F5D170BCCD
:1059800040084000704710B5002B08DA0024401C86
:10599000614192185B411A4301D14008400010BD9B
:1059A000F0B51FB482B005460C0003D008460BF0DA
:1059B000D3F902E00BF0D0F92030024600902146E6
:1059C0002846FFF7F1FE049B059A04460F4618434C
:1059D0001143084314D0184610431BD000984021AF
:1059E0000A1A18460599FFF7DDFB05460E46009A90
:1059F00005990498FFF7D8FE084305D0012004E07C
:105A00002046394607B0F0BD0020C11705430E43BC
:105A10002C43374300990E986305401A7905E40A30
:105A200000220C43FD0A0A3002D500200146E9E7B6
:105A30000105101969410C9C0D9D00196941FFF782
:105A4000A2FFDFE74A0009030123090B1B051943E5
:105A50000A4B10B5520D9A4202DA0020014610BDE1
:105A6000064B34339A4203DC9A1AFFF79BFB10BDB6
:105A7000034BD218FFF798FE10BD0000FF03000093
:105A8000CDFBFFFF064C0125064E05E0E36807CC81
:105A90002B430C3C98471034B442F7D3FFF714FB68
:105AA000A42D0108C42D010800487047EC2101080D
:105AB00010B50446FFF7F8FF0068005DC007C00F8F
:105AC00010BD0000FFB5087889B01546FF2805D045
:105AD000491C2D2804D00022002407E000240BE0FC
:105AE0000122F9E70A235C430419491C0878FF28BE
:105AF000F8D1002A00D06442002004902A780146A0
:105B00002D2A01D02B2A0FD16D1C2D2A02D0002264
:105B1000049209E00122FBE700260A2233466D1CAD
:105B200000F0FFF9381871412F78FF2FF4D10C9A4B
:105B3000A218069202460A4304D0FF23069A913324
:105B4000DA4205DA002109980A4606C00DB0F0BD18
:105B50000024B74AB54D2646079200F02FFA02906E
:105B600006980391002801DA474200E0074639050C
:105B70000020AF4A001C51410191009012E0F8074B
:105B800007D022462B4630460799FFF7A1FC064670
:105B9000079122462B4610461946FFF799FC04460A
:105BA0000D467F10002FEAD10698019B0028009A2D
:105BB0000399029806DAFFF7F3FC3246079BFFF7DA
:105BC000EFFC05E0FFF784FC3246079BFFF780FC03
:105BD000049A002A02D00122D2075140099A03C236
:105BE000B4E7FFB591B0002009900025ED432E20C9
:105BF0009E685C681F460190B9696D1C12988847C1
:105C00000090396A88470028F6D10098401C0AD0D5
:105C10000D20C0018443002E12DD00982B2809D0EE
:105C20002D280DD103E00020C04315B0F0BD0120A8
:105C300080020443B9696D1C12988847761E009053
:105C400003A9600501D52D2000E02B206A461073C2
:105C5000491C0CA80F9102900AE0B9696D1C1298BA
:105C6000884700900120400204431398761E056087
:105C7000002E02DD00983028EFD00199009888426C
:105C800046D18020044308E00998401E0990012075
:105C9000400204431399681C0860B9696D1C761EA4
:105CA0001298884700903028EED031E00199884260
:105CB00005D1200603D480200443761E1EE0009800
:105CC0000BF082F9002826D001204002044307A9E6
:105CD0000F980331761E88420BD200980F99303806
:105CE00008700F98401C0F90200607D50998401E99
:105CF00003E0200602D40998401C0990A00502D5B3
:105D00001399681C0860B9696D1C12988847009047
:105D1000002ECBDC59E0002E57DD0098652801D01D
:105D2000452852D1A00550D5032000028443B9690B
:105D30006D1C761E129888470090002E0CDD2B28D3
:105D400004D02D2808D1FF2001300443B9696D1C0F
:105D500012988847761E0090E00501D52D2100E0BD
:105D60002B21029801700298401C0290019025E0BE
:105D70000120400204430EA902980131761E884298
:105D80000ED20098029930380006000E087003D138
:105D90000299019881420AD90298401C029006E0BB
:105DA000E00501D5234801E0224840420990B96945
:105DB0006D1C12988847009013980560002E04DD32
:105DC00000980BF001F90028D2D1F96912988847A0
:105DD0000F99FF200870029903AA087000200A900A
:105DE0000B900CA90AA8099BFFF76CFEA00502D432
:105DF0000120C04319E72420044209D0E00713D151
:105E000038680B9A0A99031D3B60006806C00BE0D6
:105E10000B990A98FFF7ACFC0146E00704D13868FB
:105E2000021D3A60006801602846FEE6000014404A
:105E30000000F03FF1D8FFFF4268002A08D0016857
:105E40000B78491C002B03D0521E06C01846704721
:105E50000121C160881E70474268002A0BD0C368C8
:105E60000168002B07D183688B4204D0491E521C65
:105E700006C0002070470020C0437047F7B582B0CD
:105E8000029C00272078641C15460197302802D018
:105E9000002D15D015E020780127641C782804D047
:105EA000582802D0002D09D00BE0002D01D0102D74
:105EB00007D1002710252078641C02E0082500E0A7
:105EC0000A250026009610E000990127694308186A
:105ED000020C294680B2714300908E183804864225
:105EE00001D3012001902078641C294600F056F867
:105EF0000028E9DA0398002805D0002F01D0641E9D
:105F000000E0029C04600198002806D00AF082FF9D
:105F100002210160C81E05B0F0BD0099300408439D
:105F2000F9E7F0B51FB486B0002000900190029010
:105F30000698069980B204900798090C0204001490
:105F4000114307900027089D099806913E463C465C
:105F500003900398A9B20204000C039004982D0C3E
:105F60001543484300212246FFF71EFCC719714123
:105F700010340E46402CECDB3846029AFFF714FC36
:105F8000009A019B801800905941029801911030AD
:105F900002904028CCDB00980BB0F0BD3A2800D22C
:105FA0003038202302469A43412A01D3104637381D
:105FB000884201D30020C043704700000EB5054A57
:105FC00002920022009213460192FFF7E9FC03B00F
:105FD00000BD00003304000070B58C180578401C2B
:105FE0006B075B0F01D10378401C2A1106D10278A0
:105FF000401C03E006780E70401C491C5B1EF9D162
:106000002B0705D40023521E0DD40B70491CFAE750
:106010000378401CCB1A921C03E01D780D70491CBC
:106020005B1C521EF9D5A142D8D3002070BD0000E0
:1060300038B50446064805490068FFF759F860433B
:1060400000E0401E00900028FBD138BD40420F0008
:10605000A4000020F8B50446006881688907890F0C
:10606000012902D10168C90727D18168144A102685
:1060700011400125002913D1816829438160012045
:10608000FFF7D6FF02F012FE074611E002F00EFE07
:10609000C01B0A280CD920680068C043C00707D07D
:1060A000606D30436065A06D2843A0650120F8BD98
:1060B00020680068C043C007E8D10020F8BD000098
:1060C00017000080F7B592B00D463C224A4901A85E
:1060D000FFF779F81298494C8068372D416B0968B1
:1060E0001091A7681DD019DC444A0C239268002146
:1060F0005A4301ABD618042D2BD008DC002D18D044
:10610000012D20D0022D24D0032D38D121E00E2DD9
:1061100057D00F2D64D0362D31D102E0383D072DF8
:106120002DD81498002F4FD0012F51D0022F5CD1C1
:1061300052E0A160E160019A029904F0F7FCE06886
:10614000401CE06051E004F015FD109805F03EFFA2
:106150004BE02A4A97687F1C042D0DD0B268022DAF
:1061600010D002252A4217D0A760E160052F0BD37B
:1061700021490022403917E0327A5207F4D4012035
:1061800015B0F0BD0125EDE70C214F43F918DA59A0
:10619000496804F0CBFC28E0E068401CE06003287C
:1061A00006D3154900229039129805F01DF81CE01D
:1061B0000E200090124A0021129B109804F0FAFF62
:1061C00013E09A587168E4E703C806F08FFF0CE00B
:1061D00003C806F0A1FF08E003C806F07BFF04E057
:1061E000002006F029FF012801D00020C8E702495D
:1061F0000022A0390348D8E7481F0108C00000204A
:10620000102700003010002010B5044680680B00F5
:106210000AF0D1FD0504090C19131B000CA20E494C
:1062200004F084FC0FE004F0A5FC0CE00321002046
:1062300006F012FF0022094902E008490022203935
:10624000204604F0D1FF002010BD012010BD000049
:10625000415445300D0A000088130000D81E010883
:1062600038B504468068164B022915D004DC002995
:1062700008D0012904D10CE003290DD00A2911D03E
:10628000012038BD516819600EA2114904F04EFC7E
:1062900014E004F06FFC11E000222046196804F0BD
:1062A000A3FF0BE00020009003CA6B4609A206F092
:1062B0005BF8022802D1009806F04CFF002038BDA0
:1062C0004001002041542B4353510D0A00000000AF
:1062D000881300002B4353513A2025642C252A0DA6
:1062E0000A0000001CB500230093C26B52680192A3
:1062F000C06B42685168044A936051606A46024923
:1063000004F072FF00201CBD4401002010B50446BB
:1063100006F018FF012802D00020C04310BD20461F
:10632000FFF7E0FF002010BD10B50446806800298B
:1063300007D001290AD002290BD0032909D0012056
:1063400010BD09A20B4904F0F1FB0BE004F012FCB4
:1063500008E00221084606F07FFE0022064920469A
:1063600004F042FF002010BD41542B4346554E3DE2
:10637000300D0A0088130000F81E010800B5E1B0D6
:10638000FF21813168460AF0D1FC684604F0DEFD49
:10639000002061B000BD000010B596B00021684635
:1063A000417202210172244803904802049023485C
:1063B00005906420069008200790E1204002099093
:1063C00002A903200AF0E0F90024E443002820D1C8
:1063D0001B4805F00FFE00281BD11A480A901A48E6
:1063E0000B9039200C9019480D9019480E901948BF
:1063F0000F90124880216430109080301290104825
:106400001191139114900AA9134804F0DFFB00289E
:1064100002D0204616B010BD01210F480191009016
:106420000E4B0FA21049074804F084FE0F4905489F
:1064300004F0B8FE0020EDE7340A0020340E0020FE
:10644000B800002030100020C01B0108B171000806
:10645000F172000819720008980F0020881D0108C9
:106460004149523738304500881E01087D630008D5
:10647000C3000348C15018188280002070470000F4
:106480001810002010B505490868002803D0898835
:10649000002202F004FC002010BD000018100020B3
:1064A00010B505490868002803D08988012202F048
:1064B000F6FB002010BD000018100020F0B599B0C8
:1064C0000C460646202110A8FEF796FEB5683C2231
:1064D000686B5D49076801A8FEF775FE06F0A4FD2C
:1064E00005225AA10090FEF7E7FE00281CD00522E5
:1064F00058A10098FEF7E0FE002815D0052257A10C
:106500000098FEF7D9FE002810D0052255A100986A
:10651000FEF7D2FE002807D0052254A10098FEF70E
:10652000CBFE002804D008E052A202E053A200E013
:1065300054A2202110A806F00AF80022534801A90D
:10654000372C16D012DC042C2AD008DC002C14D0F6
:10655000012C1ED0022C23D0032C72D120E00E2C53
:1065600068D00F2C63D0362C6BD102E0383C072C5E
:1065700067D8C369042B27D059E0C2610262044680
:106580002846019A029904F0D1FA206A401C206240
:106590004DE0284604F0EEFA384605F017FD46E0D7
:1065A000042C04D0022C0FD0032C15D02BE0C3698F
:1065B0000C245C436418247A640742D5026214E018
:1065C000214900225C3926E0C3690C2463435B182F
:1065D0001B7ADB0707D116E0C3690C2463435B1801
:1065E0001B7A9B070FD50262C3695B1CC361052B35
:1065F000E6D20C204343CA585818416810AB2846CD
:1066000004F094FA13E0016A491C0162032906D3DD
:106610000D490022FC39304604F0E6FD07E00E206B
:10662000009033461A4A0021384604F0C3FD00208A
:1066300019B0F0BDC0690C2250430A584018DCE77D
:10664000FFE70120F4E70000841F010834363030F2
:106650003000000034363030320000003436303044
:10666000310000003436303036000000343630302F
:1066700033000000434D4E4554000000554E494E36
:106680004554000043544E4554000000C000002013
:106690001027000010B5846800292ED001292CD0C5
:1066A0000F2901D0012010BD154900220B78012BC4
:1066B0001ED005F0CFFC204600F0FCFD00281CD0C9
:1066C000204600F0ABFC002817D02046FFF71EFE46
:1066D000002812D0204600F0D9FE00280DD0204618
:1066E00000F048FD002808D0204600F077FD04E0C7
:1066F0000A700022034904F077FD002010BD00005D
:10670000C0000020081F010808B50F2925D006DCAD
:10671000002922D0012908D0042904D108E01A292F
:106720000BD0272916D0012008BD08F0CDFB14E0BE
:1067300000220B4904F058FD0FE00020009003CA2E
:106740006B4608A205F010FE012806D1009808F05B
:10675000BDFC02E0094901200870002008BD0000CE
:10676000981E01082B51495552433A2022636C6F01
:10677000736564222C25640D0A000000C00000200F
:1067800010B58068002907D0012905D00F2901D054
:10679000012010BD00F070FD002010BD10B50029D3
:1067A00009D0012907D0042901D0012010BD002201
:1067B000024904F019FD002010BD0000981E0108D8
:1067C00010B504468068002907D001290AD00229A3
:1067D0000BD0032909D0012010BD09A20B4904F0F8
:1067E000A5F90BE004F0C6F908E00321022006F049
:1067F00033FC00220649204604F0F6FC002010BDC0
:1068000041542B4346554E3D310D0A00881300007C
:10681000081F010810B50446002905D001291DD024
:106820000F2908D0012010BDFFF72CFE0221002007
:1068300006F012FC12E0002006F0FEFB012803D156
:106840000221002006F008FC002006F0FDFB0128D4
:1068500004D100220249204604F0C6FC002010BDED
:10686000B81E0108F7B582B002980E268468214D43
:10687000606B03290068019035D006DC00290DD03B
:1068800001291BD0022906D12DE004292BD00E2985
:1068900017D0322927D0012005B0F0BD0027E762CC
:1068A0002169204688470028FAD0E7626F70FFF719
:1068B000E9FD7D220096D200029B0FE005F086FBE9
:1068C00016E06878002802D0012811D10BE00120E1
:1068D0006870FFF7E5FD084A029B009600210198C9
:1068E00004F068FC04E000220449029804F07CFCF7
:1068F0000020D1E7C000002088130000C81E010856
:1069000000B5002385B0372933D00CDC042915D01D
:1069100004DC002941D001290DD13EE0352912D0F7
:10692000362908D125E0382923D0392921D03A2920
:106930001FD03B291DD0012005B000BD0022184901
:1069400004F052FC29E00293039303A804A90493E2
:106950000091019003CA02AB12A205F005FD0328C5
:106960001BD102AB07CB08F083FC029808F022FC95
:1069700013E001A80393009003CA03AB0EA205F035
:10698000F3FC022809D10FA1029A0198FEF794FCAA
:10699000002802D1039808F099FB0020CCE7000002
:1069A000981E01082B524543454956452C25642C19
:1069B00025643A0D0A25650025642C2025700D0AF2
:1069C00000000000434C4F5345440000002903D011
:1069D000012901D0012070470020704770B505469D
:1069E00084680B000AF0E7F905040D1111111C0071
:1069F00006F01EFB03460BA20C49204604F096F855
:106A00000CE0204604F0B6F808E0104606F060FB03
:106A1000074800224168284604F0E6FB002070BDCC
:106A2000012070BD25730D0A0000000088130000CE
:106A3000E8000020FEB586680346706B3E4F006894
:106A4000019001250020BC7807294CD006DC0029E4
:106A50000CD001290DD0022906D111E0082949D016
:106A60000E2950D00F295FD00120FEBDB87078618B
:106A70004EE0304604F07EF8019805F0A7FA59E0A0
:106A80002D4A51691269491C002C02D0012C0ED0EC
:106A900050E0F870012A07D0052A05D079616429F1
:106AA00018D90022254911E0BD70786134E0F870F2
:106AB000012A04D0052A02D07961B8610AE0B869D8
:106AC000401CB86106D01D4900228031184604F0F0
:106AD0008BFB2FE00E207D220090120100210198F7
:106AE00004F068FB26E0002C24D1134B03CA1033BA
:106AF00013A205E0012C1DD10F4B03CA103314A2C1
:106B000005F032FC16E0002C02D0012C04D011E07C
:106B10003861FD7012A202E03861FD7013A21649BF
:106B2000304604F003F805E0F878002802D130463A
:106B300000F0A2FB0020FEBDC0000020981E01084E
:106B40002B435245473A20252A2C2564000000009B
:106B50002B43475245473A20252A2C256400000044
:106B600041542B435245473F0D0A000041542B43EB
:106B7000475245473F0D0A00881300007FB5054680
:106B80008068214C37292BD00CDC02291FD004DC73
:106B9000002912D001290DD116E0032917D036297A
:106BA00008D11DE038291BD0392919D03A2917D02E
:106BB0003B2915D0012004B070BD1346226113A2F9
:106BC000174903F0B3FF1DE003F0D4FF1AE020697A
:106BD00008F07CFA00221349284604F005FB11E076
:106BE0000020039001A8009003CA03AB0EA205F099
:106BF000BBFB022806D10FA1029A0198FEF75CFBAD
:106C00000028E4D00020D6E72001002041542B4387
:106C10004950434C4F53453D25640D0A0000000088
:106C200030750000381F010825642C2025700D0ADE
:106C300000000000434C4F5345204F4B0000000024
:106C4000F7B584B00498002685684B4C686B3629EC
:106C50000068039010D00CDC022937D004DC002936
:106C600015D001297ED134E0032939D00E29F9D17C
:106C700075E0373904297CD801A80396009003CA2F
:106C800003AB3EA205F070FB02286FD134E0104642
:106C9000A26008F0E3F90746A06808F0CFF90646BD
:106CA000A06808F005FA012811D037A06946C1C1D3
:106CB00036A23E492846A36803F038FF0E20009014
:106CC0003B4A0021049B039804F074FA4EE039A07B
:106CD000ECE7284603F04EFF039805F077F945E00E
:106CE000A06808F011FAE068401CE060032836D381
:106CF00000223149E66034E0A0680399884235D12A
:106D00002EA1029A0198FEF7D7FA00280ED02FA1E3
:106D1000029A0198FEF7D0FA002807D02EA1029A15
:106D20000198FEF7C9FA00280CD01FE0E660A068C1
:106D300008F004FAA06808F033FB00280FD0002206
:106D400029490EE0A06808F0DFF9E068401CE06027
:106D5000032804D30320E060A06808F03BF9002278
:106D6000224900E005E0049804F03EFA002007B054
:106D7000F0BD0120FBE700002001002025642C204D
:106D800025700D0A000000005544500041542B436B
:106D9000495053544152543D25642C222573222CD2
:106DA000222573222C25750D0A000000881300008F
:106DB00020BF020054435000881E0108414C524538
:106DC00041445920434F4E4E45435400434F4E4E8D
:106DD000454354204F4B0000434F4E4E45435420F3
:106DE0004641494C00000000D01F0108381F01082F
:106DF00038B58468002907D0012912D0022914D09F
:106E0000032912D0012038BD0B4D10462A6008F02E
:106E100003F9009009A2104920462B6803F086FE72
:106E200007E0204603F0A6FE03E000220B4904F031
:106E3000DBF9002038BD00002001002041545E48ED
:106E400045415254434F4E4649473D312C25642C11
:106E500025750D0A0000000030750000E01F0108D4
:106E60007CB58568002907D001291AD002291CD0D9
:106E700003291AD001207CBD0F4C1046626008F037
:106E8000BBF80646606808F0B7F8FEF7EAF9410873
:106E90000091019609A210492846636803F046FE56
:106EA00007E0284603F066FE03E000220B4904F0E9
:106EB0009BF900207CBD00002001002041545E4869
:106EC00045415254424541544845583D25642C257E
:106ED000752C25730D0A000030750000381F01085D
:106EE0007FB50646856800203A4C362910D00CDC68
:106EF00002296AD004DC002915D0012968D126E0D6
:106F0000032929D0102963D12AE0373904295FD811
:106F1000039001A8009003CA03AB2FA205F024FA46
:106F2000022852D12BE01046626108F0A5F8002833
:106F30004BD005F0BBFBA061002846D04068009014
:106F400028A22D492846636903F0F0FD3DE0A061C9
:106F5000284603F00FFE38E0606908F0B7F829E032
:106F600003F090FE012803D1A06903C804F03AF8A9
:106F7000A06922490CC8284603F004FE25E0606998
:106F80000399884221D11EA1029A0198FEF794F933
:106F9000002807D01CA1029A0198FEF78DF900285D
:106FA0000BD012E0606908F067F800280DD0A169E5
:106FB00005F050FB0022174904E0606908F086F8EC
:106FC00015490022304604F00FF9002004B070BDCE
:106FD0000120FBE72001002025642C2025700D0AEC
:106FE0000000000041542B43495053454E443D2579
:106FF000642C25750D0A000088130000204E000047
:1070000053454E44204F4B0053454E442046414982
:107010004C000000381F0108981E0108F8B505460D
:10702000002405F017F8204608F034F803281AD099
:10703000204608F02FF804281DD0204608F02AF832
:10704000052814D0641C032CEDDB1C4F0321F869C8
:10705000401CFEF763F80C460026084608F01AF8B4
:1070600006280DD01EE00421204608F089F92246AA
:107070001349E86B12E0124922461039E86B0DE023
:10708000204607F0F9FF00280CD005F00FFB002880
:1070900008D00B49FC6122461031E86B04F0A4F8DB
:1070A0000020F8BD0321601CFEF738F8761C0C4662
:1070B000032ED2DB0020C043F8BD000020010020D9
:1070C00000200108F8B584680346606B224E05680D
:1070D0002248032919D006DC002923D001290AD02F
:1070E000022906D10EE004292FD00E2916D00F292F
:1070F00026D00120F8BD204603F03CFD284604F0D0
:1071000065FF22E00022164916E00E207D22009045
:10711000D2000021284604F04DF816E041680A2903
:1071200007D2491C41600FA23146204603F0FEFC05
:107130000BE00B4900221031184604F055F804E02A
:10714000002005F079FF012801D00020F8BD044996
:10715000002240390648F0E788130000C0000020F4
:10716000E81E010841542B4350494E3F0D0A0000D0
:107170003010002010B50446022005F05DFF012804
:1071800002D00020C04310BD084A00231360E06B0A
:1071900041685160496818329360516003491A464A
:1071A000183104F021F8002010BD0000E800002094
:1071B00010B5032009F096FA10BD000005480649F5
:1071C000406804E0884201D10120704740680028EF
:1071D000F8D1704730100020281F010810B5044670
:1071E000022005F031FF012802D00020C04310BD6D
:1071F000084A00231360E06B4168516049682832F7
:107200009360516003491A46283103F0EDFF0020D6
:1072100010BD0000E800002070B50D461446114670
:10722000284605F087F801280DD1285D00280AD1ED
:10723000002C04D028192038C07F0A2809D02946FC
:1072400005A003F0A7FE22462946032009F0D0FB43
:1072500070BD294604A0F4E75B41542053656E6479
:107260005D2025730D0A00005B41542053656E6458
:107270005D2025730000000010B5044600F01AF8E8
:10728000002815D02046FFF741F8002810D02046EE
:1072900000F0FCF800280BD02046FFF76BFF002819
:1072A00006D02046FFF79AFF002801D00020C043F7
:1072B00010BD000010B5002005F0C6FE012803D166
:1072C0000321002005F0C8FE002005F0B5FE0128CE
:1072D00002D00020C04310BD00220349034803F040
:1072E00083FF002010BD0000A81E01083010002000
:1072F000FEB50446002668460670002C12D0E068F1
:1073000000280FD0606A00280CD02746A06A4D4D97
:107310002037002806D078E0E2686946204690478A
:10732000002802D00020C043FEBD68460178E06A14
:10733000626A431CE3621154E16A606A4654E06A7F
:1073400009280BD1092240A0616AFDF79FFF0028A0
:1073500004D10120287004F07DFEE860287801281F
:1073600003D0022801D0032809D104F073FEE96894
:10737000401A384988424DD82878012809D0C0B22F
:107380000A2822D0684600780D2823D00A2824D065
:1073900026E031A1606AFDF746FF0290002834D054
:1073A000019601AB2DA2E16A606A04F0DDFF0228BC
:1073B00030D1019800282DD0626A0299891A0818E4
:1073C000C01CA8600A2028701FE0E16AA8688142FA
:1073D0001BD11FE00120387405E0387C012806D05D
:1073E000387C022805D0E06A01280ED109E002208D
:1073F0003874E06A022801D03E740BE0E6623E7405
:1074000003E0606A00783E2804D0A06AE16A401E6A
:10741000814281D3E16A606A04F08CFF01280CD1BB
:10742000E06A002805D0616A08182038C07F0A2861
:1074300006D00EA0616A03F089FD2E700020FEBD0B
:107440000EA0F8E7A80000202B52454345495645B9
:107450002C000000DC0500003A0000002B524543E0
:10746000454956452C252A2C25643A005B41542079
:10747000526563765D2025730D0A00005B41542040
:10748000526563765D2025730000000010B5044648
:1074900005F016FE012802D00020C04310BD084AA6
:1074A00000231360E06B41685160496808329360C3
:1074B000516003491A46083103F096FE002010BDC2
:1074C000E800002010B500231A4603E0845CE318AE
:1074D0009BB2521C8A42F9D3D84380B210BD00003F
:1074E00010B506490020C870054902460860012110
:1074F00005200903000701F0D2FB10BDD4010020D4
:107500008C00002001484078704700008C0100206A
:1075100000B589B020216846FDF76EFE012168465E
:107520004170022101700D480190C8010290C00015
:107530000490402005906946002009F025F907488D
:107540000749203801610749C1610749816107493D
:107550004161074804F016FC09B000BDA82C0020CA
:107560006D760008617600089D760008AB7600080D
:1075700008270020FEB5384C607800280BD0374E25
:10758000002501280AD0012702282CD0032804D185
:10759000684605704EE004F069FBFEBD6846057064
:1075A00001A90220019509F0DDF87D27FF000AE01E
:1075B0006846007803280DD065603B460122694685
:1075C000019803F070F96946002009F08BF8002853
:1075D000EED0FEBD6068002802D000206070ECE7AD
:1075E00030686060E9E76846057001A902200195EE
:1075F00009F0B8F806E068460078032809D0A560CD
:1076000009F0E2FA6946002009F06CF80028F2D08F
:10761000FEBDA168002903D0A77000216170EFE7CB
:107620003168A160ECE768460078032809D0E5607E
:1076300009F0CAFA6946002009F054F80028F2D08F
:10764000FEBDE168002903D0A77000216170EFE75B
:107650003168E160ECE700008C010020140000209C
:1076600010B50146002009F03DF810BD0FB400B57B
:10767000FFB082B0012183AB49026846829A09F0CB
:1076800055FB6846FDF7EDFD02466946002009F00E
:10769000AFF97FB002B008BC04B0184701B50122B1
:1076A0006946002009F0A4F908BD10B50446FDF7AD
:1076B000D8FD02462146002009F09AF910BD0000CD
:1076C00001494870002070478C01002010B5034824
:1076D00000F0DCFF024800F0D9FF10BDD409002003
:1076E000FC08002010B5034800F0D0FF024800F06D
:1076F000CDFF10BD8C0900204409002030B5446C3A
:107700001C252C400125A540046C6560046863605D
:107710008368102B036803D099600068C26030BD95
:107720009A600068C16030BD7D2100B5C900484342
:1077300000F001F800BD002140E000BF00BF00BF25
:1077400000BF00BF00BF00BF00BF00BF00BF00BF41
:1077500000BF00BF00BF00BF00BF00BF00BF00BF31
:1077600000BF00BF00BF00BF00BF00BF00BF00BF21
:1077700000BF00BF00BF00BF00BF00BF00BF00BF11
:1077800000BF00BF00BF00BF00BF00BF00BF00BF01
:1077900000BF00BF00BF00BF00BF00BF00BF00BFF1
:1077A00000BF00BF00BF00BF00BF00BF00BF00BFE1
:1077B00000BF00BF00BF00BF00BF491C8142BCD357
:1077C000704710B5012001F07BF910BD10B5012004
:1077D000400201F075F90120800201F071F90120E9
:1077E000000301F06DF90120400301F069F910BDBB
:1077F00072B6FEE710B5084900224A6107494B6896
:107800004C1523434B604B68082423434B60C0094D
:10781000C001026010BD00001C0A002000200240D0
:107820007FB500240D460646039401F079F8E80977
:10783000029003A901960094684601F009F80749EF
:10784000002806D00120088001F03EF8002004B096
:1078500070BD0C8001F038F80120F8E7B801002075
:1078600010B5002302E0C45CCC545B1C9342FAD3F5
:1078700010BD000010B5214A00219069C3052048C1
:1078800004D54169022319434161911593699B0510
:1078900005D5436901242343436163021943936976
:1078A0005B0505D54369082423434361E30119437C
:1078B00093691B0505D5436904242343436163028F
:1078C000194393699B0405D54369102423434361FD
:1078D0006302194393699B0304D5446920231C4325
:1078E000446119439369DB0305D54369402423436D
:1078F0004361A0020143916110BD000000200240DD
:107900001C0A002070B5054601F0D0F90646184C57
:107910000AE0681C08D0002D04D001F0C7F9801BD4
:10792000A84201D9032070BDA069C007F1D1A069A8
:10793000800701D50220A061A069C00511D4A0690B
:1079400080050ED4A06940050BD4A069000508D4B9
:10795000A069800405D4A069800302D4A069C00393
:1079600003D5FFF787FF012070BD002070BD000028
:1079700000200240F8B51746002605460C4600F0E8
:10798000CFFF0BE029460220226800F0ABFF084938
:107990000028488004D1241D2D1D361DBE42F1D380
:1079A00000F092FFBE4201D20020F8BD0120F8BDD8
:1079B000B80100200FB4F8B504460D460026002C8F
:1079C00004D1401EF8BC08BC04B01847E06A002887
:1079D00000D1F7E709A80090E76A29462046009BF6
:1079E000089AB8470646002000903046EAE7FFB5FF
:1079F00004460D46002100260023214600BF11E069
:107A0000D8001150D80080184660D80086185B1C3A
:107A100068684F68B84204D103980660002004B03B
:107A2000F0BD49680029EBD1481EF8E7F8B50546D6
:107A3000002600272E0CAFB20848046809E0208811
:107A4000B04205D100223946204603F00FFB02E088
:107A50006469002CF3D100BFF8BD0000CC02002007
:107A600010B5827F5118C9B28177182914D31839FB
:107A70008177417F0122491CCCB24477017F0B0002
:107A800009F099F90D0A080B0819081908081908CE
:107A9000191E0A001F2C10D810BD817E8B070321F0
:107AA000002B03D01C2CF7D9427702E01D2CFBD809
:107AB00010BD017710BD1E2CFCD94277491CF8E798
:107AC0001F2CF7D942770277418B491C418310BDA7
:107AD00010B5054B64220549054802F0E4FE9620E6
:107AE000FFF722FE10BD0000B80B000018000020B8
:107AF0003007002010B586B003AA009201AB0FA298
:107B000004F032FC0024E443022811D104990398C4
:107B100004F0C1FBC3B201980121027803E001988F
:107B2000405C4240491C02988842F8D89A4202D0F0
:107B3000204606B010BD0020FBE700002425702A77
:107B400025700D0A0000000010B588B000F05CFA46
:107B5000164C0122A188206801F0A1F80A2000F04B
:107B600065FEA1880022206801F099F80A2000F043
:107B70005DFEA1880122206801F091F8012069468C
:107B80004870022008700A49019141020291094996
:107B90000391042104910590694608F0F5FD204603
:107BA0008821103004F056FB08B010BD20250020BD
:107BB0002021002083010020F3B52A4895B0012739
:107BC0000770282108A8FDF717FB16991598FFF7ED
:107BD00091FFBC1E002807D112AB23A2169915985D
:107BE00004F0C2FB0F2802D0204617B0F0BD129857
:107BF00015990278169800240E18274D203E302A39
:107C000029D0AB68002B02D00246002098472348B9
:107C10001121016022480770F477B4772148A978D0
:107C200000780590204803940494069101781F4839
:107C30006A46808813C2FF211DA201312348159B8B
:107C400004F085FCA978491CA9706870204808F0E8
:107C500019FD0020C9E711211048090201601048F0
:107C60000470D9E70500002024252A2C252A2C257C
:107C70002A2C252A2C252A2C252A2C25702C252A2D
:107C80002C252A2C252A2C252A2C252A2C252A2C61
:107C9000252A2C252A2A00008001002088000020A7
:107CA000B8020020DB01002000000020783700200F
:107CB00025732C25582C253032782C25782C2564DA
:107CC0002C25642C25642C25640D0A00E025002059
:107CD00078390020F3B500254468ED43066883B089
:107CE000092C0AD322462E21304604F0A3FC0700BB
:107CF00003D0B81B0190042802D0284605B0F0BD7F
:107D00000221304604F03BFCFDF7CAFC0546009119
:107D10000221B01C04F033FCFDF7C2FC0290019874
:107D20000E46241A641E2146781C04F028FCFDF738
:107D3000B7FC0E4F04E000223B46FDF731FC641E09
:107D4000002CF8D102460B4631460298FDF70EFB97
:107D50000022074BFDF724FC2A46009BFDF706FB9B
:107D6000049AD16090600020C8E700000000244021
:107D700000004E40F3B500254468ED43066883B02B
:107D80000A2C0AD322462E21304604F053FC070069
:107D900003D0B81B0190052802D0284605B0F0BDDD
:107DA0000321304604F0EBFBFDF77AFC0546009119
:107DB0000221F01C04F0E3FBFDF772FC0290019835
:107DC0000E46241A641E2146781C04F0D8FBFDF7E9
:107DD00067FC0E4F04E000223B46FDF7E1FB641E0A
:107DE000002CF8D102460B4631460298FDF7BEFA48
:107DF0000022074BFDF7D4FB2A46009BFDF7B6FA9D
:107E0000049A516110610020C8E70000000024407E
:107E100000004E40F3B59BB00F465E4C1B98FFF739
:107E200069FE0026F6430025002801D02576A0E053
:107E300010AB079313AA0EA915A804AB07C319AB7F
:107E400003930CAA17A90AA86B4607C308AB52A252
:107E500039461B9804F088FA0D2872D10B980A99BC
:107E600001286ED10878412806D02576207E012889
:107E700005D000201DB0F0BD01202076F6E7089F58
:107E80002E213846099A04F0D5FB002871D0C01B7A
:107E900006286ED10221384604F071FBA07702213A
:107EA000B81C04F06CFBE0770221381D04F067FB7E
:107EB000202108551198109F06285AD102213846D2
:107EC00004F05DFB60770221B81C04F058FB2077BA
:107ED0000221381D04F053FB7D2109014018608305
:107EE000214617A8FFF7F6FE002842D1214619A81F
:107EF000FFF740FF00283CD10F9F0E990A2F38D280
:107F0000002F0FD03A4603A8FDF75DF903A8C55529
:107F100009F00EFC2B4A2C4BFDF7DAFAFDF7E2FBD9
:107F2000208000E025802846149F139D002F0DD04F
:107F30003A462E21284604F07DFB002802D0411B42
:107F400001E016E03946284604F019FB60800D98E0
:107F50000C9901280DD8002807D00878532804D19F
:107F60000122E068D2075040E06016981599012878
:107F700001D930467EE7002807D00878572804D179
:107F800001226069D2075040606108212046FFF756
:107F900067FD6EE7B825002024252A2C25702C25A6
:107FA000702C25702C25702C25702C25702C25709C
:107FB0002C25702C25702C252A2C252A2C252A2AA4
:107FC000000000006F1283C0CAA1FD3F08B5002069
:107FD0006946087003E06846007800F023F86946B7
:107FE000022008F07FFB0028F5D008BD10B5002066
:107FF000044902460870012105200903000700F02A
:108000004EFE10BD8001002010B50120044902463B
:10801000087001030520000700F041FE10BD0000BC
:108020008001002070B5224D00262C462B78611C63
:108030008034002B08D022465268022B0CD0032B30
:1080400009D10A2813D030E0242804D102222A7052
:1080500070540120606070BD50546168491C6160BB
:108060007E2922D20D28F6D10320287070BD5054ED
:108070006068401C606046540EA1681CFDF7D3F890
:10808000002808D0681C6168FFF796FD681C6168CD
:10809000FDF7B2F809E009A1681CFDF7C4F8002853
:1080A00003D0681C6168FFF7B5FE2E7070BD00003C
:1080B000302500204747412C00000000524D432C42
:1080C0000000000010B5084800F036FA0A21064802
:1080D00000F0CEF9044800F0B9F8800503D5024855
:1080E00000F0B6F880B210BD84050020F8B5FFF7A7
:1080F000E9FFFDF7CDFA274E3146FDF7F9F8264C9A
:1081000026490025206188423EDB2078244F002844
:1081100015D02570FFF7D6FFFDF7BAFA3146FDF707
:10812000E7F82061FDF7FCFA00223B46FDF7C2F9B3
:1081300000221C4BFDF7CCF9FDF71AFBA06020696B
:10814000FDF7EEFA00223B46FDF7B4F9164A174B4D
:10815000FDF7BEF906460F46A068FDF7E1FA124AA0
:10816000134B5242FDF7B4F932463B46FDF7FEF899
:10817000FDF7FEFA0F49A060884201DDA16004E02E
:10818000FF21C905C84200D3A560A068FDF796FA93
:10819000C0B2F8BD00401B44A401002000006040B4
:1081A00000000C4000E064403333333333B33040DD
:1081B000CCCCEC3F0000C842F8B506460D46403630
:1081C000317C01290DD00121317401688A68520780
:1081D00009D5416D202211434165002030740120F2
:1081E000F8BD0220F8BD174B6A68D80547109A42BF
:1081F000154C8A6A2B6812D05B035B0B1A438A62A8
:108200002968490305D5A1680143A1600A20FDF74B
:108210000FFF2868800312D5A06838430EE05B0387
:108220005B0B9A438A622968490302D5A16881439E
:10823000A1602868800302D5A068B843A060002030
:108240003074F8BD0110000000270140406D7047F8
:108250000068006C7047000070B5040006D0606DC7
:10826000264600254036002802D006E0012070BDD9
:10827000A5653574204600F0D3F8606DC00603D4C0
:1082800021688868400705D5606D10210843606546
:108290003574EBE7606DFF220132904302221043F8
:1082A000606588688207920F5B48012A02D10A68DC
:1082B000D2072BD1032362689B079A4205D05B4209
:1082C0009A4202D05B009A4209D10A699200920850
:1082D0000A6121680A6963681A430A610CE00A6945
:1082E000920092080A6181680F2292049143816092
:1082F00081686268114381602168CA6818239A43C3
:10830000CA602168CA68A3681A43CA6081680122EA
:108310005206914381608168A28E520611438160AA
:1083200020688168C90004D48168012212071143C2
:1083300081602068C168394A1140C1602069E168E4
:10834000022825D000200143204620300278037BFC
:1083500052035B001A431143226B1143A26992033B
:108360001143E269D20311432268D3681943D160F3
:10837000616A0A46FF3AC23A05D0A26A11432268EE
:10838000D3681943D16042780121012A02D00BE061
:108390000420D8E70078002823D0606D2022104305
:1083A0006065A06D0843A065E06B012820681FD0C0
:1083B0000169C90703D001694908490001612068C2
:1083C0004169C908C900416120684169A26B114334
:1083D0004161A565606D80088000401C60650020DB
:1083E00070BD2068C26801231B041A43C260DBE72A
:1083F0000269FF239B009A43026120680269236C93
:10840000A66C1A43636C33431A4302612068026905
:108410000A430261D3E70000002701401902FEFF72
:1084200010B586B0044614216846FCF7E5FE0E49F7
:108430002068884216D10D48416B421511434163B3
:10844000C16A01221143C162C06A694610400590A9
:1084500002200090032001900020029005200007D8
:1084600000F03AFB06B010BD0024014000100240AD
:10847000F8B504464069254640350E4608280BD01D
:108480002068C068C00709D0606D2021084360657E
:10849000002028740120F8BD082700E00C2700F018
:1084A00005FC009015E0701C13D0002E05D000F0E4
:1084B000FDFB0099401AB0420BD920680068384291
:1084C00007D1606D042108436065002028740320F3
:1084D000F8BD206800683842E5D0606D012149028E
:1084E000084360652068C16809058A0F0C21002ACD
:1084F0001BD12022125D002A17D10268120714D561
:10850000826853070122002B08DB43688B434360DA
:10851000606D130298431043606506E0606D202390
:1085200018436065A06D1043A065A069002801D1C3
:10853000206801600020F8BD70B504462168002065
:108540008968490721D425464035297C01291CD05A
:1085500001212974E169012904D02046FDF77AFD43
:10856000002811D1616D0A4A1140FF2201321143E6
:1085700061650021A165297422681C2111602168B0
:108580008A6804231A438A6070BD022070BD00000F
:10859000FEF1FFFF30B5014620314A790023022A5F
:1085A00004D00422C2630B71012030BD026814683C
:1085B0000E25AC43146002681468640864001460FB
:1085C000446C1C22144001221546006CA5404560F5
:1085D0004A7118460B7130BD70B500240146203138
:1085E0004A79022A03D00421C163012418E00268F9
:1085F00013680E25AB431360026813685B085B00C9
:108600001360436C1C221340012215469D40036CED
:108610005D604A7100220A71816B002900D0884791
:10862000204670BD70B5040029D020680168490853
:10863000490001601348256814212818FCF758FDEB
:10864000800060641048206400202860626C1C2157
:108650000A4001239340226C53600B4A8032936A94
:10866000656C0D400F21A9408B439362E06220634B
:108670006063A063E06320346071207170BD0120ED
:1086800070BD0000F8FFFDBF00000240F0B4016CB7
:108690000D6801680C68466C1C2304221E401746B6
:1086A000B7402F420ED067070CD50C68A40602D441
:1086B0000C6894430C60416C19408A40016C4A601C
:1086C000016B1AE00227B74002462F402032002FEC
:1086D00017D0A70715D50C68A40605D40C680A2581
:1086E000AC430C6001215171446C02211C40036CAD
:1086F000A140596000211171C16A002918D0F0BC55
:1087000008470827B7402F4212D0240710D50C681D
:108710000E25AC430C60446C01211C400B46A34069
:10872000046C6360C163517100211171416BE4E716
:10873000F0BC704770B504003CD01F482568142178
:108740002818FCF7D5FC800060641C4820640221D6
:10875000204620300246417129681948E3680140EB
:10876000A06866691843236933431843A369184313
:10877000E3691843236A1843084328600121A0686D
:108780008903884210D00D488030836A656C1C21B3
:108790000D400F26AE40B3438362656C63680D40A5
:1087A000816AAB400B4383620020E0630121517179
:1087B000107170BD012070BDF8FFFDBF00000240C8
:1087C0000F80FFFFF8B504468C4620300179002564
:1087D000012909D00126067141790027012905D018
:1087E000077102252846F8BD0220F8BD022141711B
:1087F000E763206801684908490001606146204636
:10880000FEF77CFF206B00282068016801D00E2253
:1088100005E0042291430160206801680A221143A7
:1088200001602068016831430160DBE770B50446F0
:1088300000F03CFA0546601C02D004480078241879
:1088400000F034FA401BA042FAD370BD980000201B
:10885000F8B51A4E0546307C0F46012807D0012096
:1088600030741748FFF74EF8010002D021E00220D3
:10887000F8BD0020C04338606C6814E02046FEF765
:10888000B9FF0F48FFF73EF801460E48426808233B
:108890009A434260426843159A434260002901D0DE
:1088A0003C6006E08034A8686A68C0018018A04275
:1088B000E4D8002030740846F8BD00001C0A0020EF
:1088C00050C30000002002400548416802221143C5
:1088D000416041680122114341600020704700005F
:1088E00000200240F8B50C4C1646207C0F460128AB
:1088F00008D0012020740948FFF704F8002500285B
:1089000002D006E00220F8BD65613E600348FEF734
:10891000F9FF2574F8BD00001C0A002050C30000B8
:1089200011484168C9070BD0EFF3108172B60F4AA6
:10893000C2600F4AC26081F310884168C9070ED136
:10894000416889070DD5EFF3108172B6094A0261BB
:10895000094A026181F310884068800701D501202F
:10896000704700207047000000200240EFCDAB8927
:1089700005040302BFAE9D8C16151413F0B500223A
:1089800062E0012393401C460C405CD09608304DB9
:10899000B6007519AF68AC4695072E0F0F25B54088
:1089A000AE463D4005273F07B84201D1002719E0F8
:1089B000284FB84201D1012714E0274FB84201D116
:1089C00002270FE0254FB84201D103270AE0244FC8
:1089D000B84201D1042705E0224FB84201D1052752
:1089E00000E00627B740AF4212D11F4D2E68A643C4
:1089F0002E606E68A6436E60EE68A643EE60AE68B9
:108A0000A643AE606546AD687446A5436446A5605E
:108A1000056856000324B44025430560D508AD0021
:108A20002D182E6AAC465507EF0E0F25BD40AE43FC
:108A300065462E62C568A543C56045689D4345608F
:108A40008368A3438360521C0B46D34099D1F0BD89
:108A5000000001400004005000080050000C0050CD
:108A600000100050001C00500004014001231B03B3
:108A7000DA1010B51101984202D104F08BFB10BD41
:108A80000D4C904203D16189491C618108E0884204
:108A900006D1A0890949401CA0810320087010BD9F
:108AA0000128FCD106F094FC6078012801D100F087
:108AB000EFFA0020208110BD00000020B902002044
:108AC00010B504494A69024202D04861FFF7CEFF5F
:108AD00010BD000000040140F8B500230324012567
:108AE000C2E032462E469E40B446324079D00E79DE
:108AF000B607B60F012E01D0022E17D18668274681
:108B0000B6465E00B74000967646BE43B646CF688E
:108B1000009EB74076463743876046686746BE4347
:108B20000F79FF06FF0F9F40374347600E79F643EA
:108B3000B6070ED0C6682746B4465E00B646B740B4
:108B40006646BE43B4468F687646B74066463743AE
:108B5000C7600E79B607B60F022E14D1DE08B60034
:108B600036180096366A5F07B446FE0E0F27B646E3
:108B7000B7406646BE43B4460F697646B740664680
:108B80003743009E376206682746B4465E00B64605
:108B9000B7406646BE430F79B446BF07BF0F76465F
:108BA000B7406646374307604E68B603B60F5AD0E3
:108BB000304F7E6B2E437E639F082F4EBF00BE1941
:108BC0000096B6680F27B4469E07360FB646B740E4
:108BD0006646BE4305273F07B446B84202D1002788
:108BE0001AE040E0254FB84201D1012714E0244F9C
:108BF000B84201D102270FE0224FB84201D103272A
:108C00000AE0214FB84201D1042705E01F4FB842C6
:108C100001D1052700E006277646B7406646374370
:108C2000009EB7601A4EB6684F689643FF0200D5A3
:108C30001643174FBE60FE684F689643BF0200D5CB
:108C40001643134FFE607E684F689643BF0300D5FE
:108C500016430F4F7E603E684F689643FF0300D572
:108C600016430B4A16605B1C0A681646DA4000D0B1
:108C700037E7F8BD0010024000000140000400503A
:108C800000080050000C005000100050001C005064
:108C9000000401400069084000D001207047002A0C
:108CA00001D081617047816270470000014880688F
:108CB000704700009800002070B504000FD02168B4
:108CC0001548086021681548086003CC4160206899
:108CD000083C21688860FFF7E9FF05460CE00120A9
:108CE00070BDFFF7E3FF401B2A2805D92068C06844
:108CF000400701D0032070BD2068C0684007F0D154
:108D000020680269E1688A4201D0016101E00449FA
:108D10000160002070BD0000CCCC00005555000063
:108D2000AAAA000000680249016000207047000004
:108D3000AAAA0000024881680278891881607047F9
:108D40009800002010B50848002401684022114313
:108D50000160032000F00AF8002801D0012401E09E
:108D600000F06AF9204610BD0020024070B50446AC
:108D70000D4D7D202978C000FCF7BAF901460B485B
:108D80000068FCF7B5F901F0A9F8002809D1042C16
:108D900007D200222146401E00F076F900206C60C8
:108DA00070BD012070BD000098000020A4000020CC
:108DB0007047704710B506F00BFB0B48017800298F
:108DC00001D0491E017009A007F08CFF0A484169D3
:108DD000491C4161C188491CC180018A491C01822A
:108DE0000189491C018110BDB90200203173BBBD4E
:108DF000D0D10D0A0000000000000020704770472D
:108E0000704710B5044600680168C943C90708D116
:108E10008168C943C90704D1012141602046FFF799
:108E2000C9FF20680168C943890708D48168C9431C
:108E3000890704D4022141602046FFF7B9FF20686A
:108E40000168C943490708D48168C943490704D464
:108E500004214160204600F0EDF820680168C94314
:108E6000090708D48168C943090704D4082141606F
:108E70002046FFF7C3FF20680168C943C90608D42C
:108E80008168C943C90604D4102141602046FFF718
:108E900090FF20680168C943890608D48168C943E6
:108EA000890604D4202141602046FFF7A9FF2068ED
:108EB0000168C943490608D48168C943490604D4F6
:108EC000402141602046FFF79AFF10BDF8B504002D
:108ED00005D025462035A87B002802D006E00120D9
:108EE000F8BD00206873204600F048F80220A873FF
:108EF0002068C26884466368012B04D00120A16AFF
:108F0000C005814201D11E20824319486169814216
:108F100001D0184802401848A6680240184630435D
:108F2000676A266A3E433043A66A30431043002BEB
:108F300018D0012B03D00122D205964203D1236918
:108F4000E2681A4310430A4A914205D0A2691143CC
:108F5000E2690243084610436146C8600120A873D5
:108F60000020F8BD2369E2691A431043E3E70000DB
:108F7000FFFF00003F1FFFFFFEF119FF10B5006863
:108F8000084988420CD10848816BC20411438163AF
:108F9000002211460D2000F077F80D2000F068F84F
:108FA00010BD0000007C004000100240F8B50446EF
:108FB0000220254620351746A8731D480268C304C1
:108FC0001A4302602068C2689B121A43C26020687C
:108FD0000269012632430261226810205060206835
:108FE00081611021204603F019FE03281FD021685B
:108FF00008204860206847610821204603F00EFEE3
:10900000032814D0204603F093FDA87B03280ED03C
:1090100020688168314381602068016931430161C2
:1090200020680169042211430161AE730020F8BD7C
:1090300000040140704700000448416B01221143C5
:109040004163816B02041143816370470010024049
:10905000002809DBC106C90E0120884003490860C9
:10906000BFF34F8FBFF36F8F7047000080E100E0C8
:10907000002805DBC106C90E0120884001490860AF
:109080007047000000E100E010B507F0A1FE10BD40
:10909000BFF34F8F04490348C860BFF34F8F00BF31
:1090A000FDE700000400FA0500ED00E00248016859
:1090B000821511430160704700700040F0B5154AF9
:1090C0001368154D54152D6A2340ED07ED0F002B45
:1090D00004D0002D02D01668A64316601668B608A4
:1090E000B600064316600D4807690426374307613A
:1090F00001290DD040BF20BF20BF0169B1430161EC
:10910000002B04D0002D02D0106820431060F0BD69
:1091100030BFF2E7007000400000014000ED00E0C9
:10912000F8B5044600780027594D800674D5584E8E
:10913000403EB06BC00004D4B06BA9050843B063D7
:10914000012754480168C90511D4016882151143EB
:109150000160FFF7ABFD009005E0FFF7A7FD009968
:10916000401A642837D84B480068C005F5D53268E6
:109170000321090560680A400140914208D081033B
:10918000890F032904D13168890301D50120F8BD75
:109190002A69032109040A4022D0084090421FD0C6
:1091A0002078800631D528692A6988430121C904BD
:1091B0000A432A612A698A432A612861C0050FD5BA
:1091C000FFF774FD009008E0FFF770FD0099411A69
:1091D0003148814201D90320F8BD28698005F3D5C3
:1091E0002078800611D561688803800F032805D197
:1091F00032680005824301400A4332602869032235
:1092000061681204114008432861002F04D0B16B3B
:10921000012000078143B1632078C00705D0E868CA
:10922000A168800880000843E8602078800705D5A1
:10923000E8680C218843E1680843E860207840072B
:1092400006D5E86803218902884321690843E8605C
:109250002078000706D5E86803210903884361697F
:109260000843E8602088C00506D5E86803210904A2
:109270008843A1690843E8602078000606D5E868BD
:10928000032189048843E1690843E8600020F8BDB0
:10929000401002400070004088130000F8B50E46F0
:1092A000050038D05E480068C007C00FB04214D235
:1092B0005B4C20684008400030432060FFF7F6FC1C
:1092C000074605E0FFF7F2FCC11B564881427AD8F9
:1092D0002068C007C00FB042F4D12878524C8007F4
:1092E00005D5E068F0218843A9680843E060287844
:1092F000C00752D06868022806D0032807D021682A
:1093000001280AD0890504E02168890301E0216869
:109310008901002903DB0120F8BD4907F9E7E1686D
:10932000890889000143E160FFF7C0FC07466868CF
:1093300002280AD0032814D001281ED029E0FFF704
:10934000B5FCC11B374881423DD8E0680007800F5B
:109350000228F4D121E0FFF7A9FCC11B314881426A
:1093600031D8E0680007800F0328F4D115E0FFF73B
:109370009DFCC11B2B48814225D8E0680007800F67
:109380000128F4D109E0FFF791FCC11B2548814277
:1093900019D8E0680007800FF5D121480168C90796
:1093A000C90FB14217D9016849084900314301602A
:1093B000FFF77CFC074608E005E0FFF777FCC11BE0
:1093C0001848814201D90320F8BD15480068C0073C
:1093D000C00FB042F1D12878400706D5E0680721D8
:1093E00009028843E9680843E0602878000707D548
:1093F000E0680721C90288432969C9000843E06081
:1094000000F03AF8E168094A0906090F515CC840C2
:109410000749086007480068FFF7A8FCF8BD00008E
:109420000020024088130000001002409C1B01082D
:10943000A40000209C000020044805490068C96879
:10944000044A4905490F515CC8407047A4000020F8
:1094500000100240B51B0108044805490068C968AE
:10946000044A8904490F515CC8407047A400002099
:1094700000100240B51B010870B51A4AD3681A499A
:109480000C2018408D0004280CD04E00082810D065
:109490000C2810D050680004410F0120C003491C63
:1094A000884070BD1068C00601D5084670BD2846CA
:1094B00070BD304670BD98020C4C000F205C1B0242
:1094C0009C0FD368641CDB0301D5314603E01268AE
:1094D000D20600D4294607F056FC22460023FBF7AB
:1094E00031FE70BD0010024000093D00AC1B0108B8
:1094F000FEB505007ED0F74CE7680C20E668074013
:109500000120000406402878C00747D0082F05D066
:109510000C2F0AD101200004864206D12068800366
:109520003CD568680028E5D038E00120696800046F
:10953000814203D121680143216011E0052301220A
:109540001B0492049942216802D111432160F1E782
:109550008143216021680140009120689043206090
:10956000686800280DD0FFF7A1FB009005E0FFF729
:109570009DFB0099401A64287ED820688003F6D5A8
:109580000CE0FFF793FB009005E0FFF78FFB0099DD
:10959000401A6428F0D820688003F6D42878800721
:1095A0005DD5E868810604D5226820210A4322603F
:1095B00088430923042F0DD00C2F01D1002E09D090
:1095C00000283CD02168994301432160FFF76EFBDE
:1095D000064628E02168490701D500288AD061683D
:1095E0001F22120291432A6912021143616021680D
:1095F000994300E091E101432160FFF73DFFE168FD
:1096000009060A0FB449895CC840B4490860B448E7
:109610000068FFF7ABFB002874D120E0FFF746FBA2
:10962000801B0228A8D820684007F7D560681F2152
:109630000902884329690902084360600FE0206835
:10964000400840002060FFF731FB064604E0FFF7CA
:109650002DFB801B02288FD820684007F7D428787C
:10966000C00661D5002F0DD0A86900284BD0206816
:10967000FF210131084300E0C6E02060FFF716FB40
:1096800006462DE02068800502D5A8690028A5D0EF
:109690006068072149038843296A0843606060685D
:1096A000297F0002000A090608436060286A410B0E
:1096B0000120C003491C8840E16809060A0F864959
:1096C000895CC8408549086085480068FFF74EFB03
:1096D000002817D128E0FFF7E9FA801B0228A1D85B
:1096E00020688005F7D56068072149038843296A07
:1096F000084360606068297F0002000A0906084389
:10970000606011E0E1E02168FF20013081432160C9
:10971000FFF7CCFA064604E0FFF7C8FA801B0228E0
:1097200072D820688005F7D428786E4E000724D5BB
:1097300068690028306910D0012108433061FFF7C3
:10974000B5FA009005E0FFF7B1FA0099401A022837
:109750005AD830698007F6D50FE0400840003061E4
:10976000FFF7A4FA009005E0FFF7A0FA0099401A6D
:10977000022849D830698007F6D42878400765D593
:1097800000200290A06BC00006D4A06B0121090745
:109790000843A0630120029053480168C90511D411
:1097A0000168821511430160FFF780FA009005E01F
:1097B000FFF77CFA0099401A642825D84A480068C7
:1097C000C005F5D5FF20AA680130824203D1316976
:1097D0000143316111E001218902002A07D00523EC
:1097E0001B029A4203D132690A433261EFE73269C0
:1097F00082433261306988433061A86800280FD005
:10980000FFF754FA009007E05EE0FFF74FFA009987
:10981000411A3648814257D830698005F5D50DE0A8
:10982000FFF744FA009006E0FFF740FA0099411A6A
:109830002E48814248D830698005F5D40298002826
:1098400004D0A06B012109078843A063686A00283F
:1098500065D00C2F4CD0012636060228206805D092
:10986000B0432060FFF722FA05462FE0B0432060A6
:10987000FFF71CFA074604E0FFF718FAC01B02289E
:1098800022D820688001F7D4E96AA86AE268084310
:10989000296BFD231B049A4311430843E0602068B1
:1098A00030432060FFF702FA054604E0FFF7FEF9B7
:1098B000401B022808D820688001F7D52FE0FFF769
:1098C000F5F9401B022801D90320FEBD2068800164
:1098D000F5D424E0001002409C1B0108A4000020E5
:1098E0009C000020401002400070004088130000DF
:1098F0000128EAD0E06801210904AA6A01409142E6
:109900000BD10F218904EA6A0140914205D103215C
:1099100089050840296B884201D00120FEBD002046
:10992000FEBD000070B5040005D0254620356878DE
:10993000002802D006E0012070BD002028702046DB
:1099400000F046F8022068702068C168C943C90663
:1099500037D5CA214162216853204862204603F06E
:1099600079FF002827D120688168184A114081605A
:10997000216888686268A369104322691A4310430A
:1099800088602168E0680861206801692289120402
:1099900011430161204603F080FF00280BD12168AC
:1099A000CA6C92089200CA646269E1691143226834
:1099B000D36C1943D1642268FF215162002801D081
:1099C00070BD00200121697070BD0000BFFF8FFFD6
:1099D00000680549884205D10448016901229204C2
:1099E0001143016170470000002800404010024010
:1099F00070B5044621680A48C860FFF757F97D260C
:109A00000546F60006E0FFF751F9401BB04201D9C8
:109A1000032070BD2068C0688006F4D5002070BDAA
:109A20005FFF010070B5040012D0022120464030D3
:109A30000546417420680168402291430160204638
:109A400000F064F80021616569742974084670BDEE
:109A5000012070BDF8B504000ED0FF27606A0537FD
:109A6000002500280AD02561656126464036A5629A
:109A7000707C002807D00AE00120F8BD6068B84279
:109A8000F3D0E561F1E73574204600F053F8022188
:109A900071742068026840239A4302602123A268FF
:109AA00060689B021A4038401043E3688A02134002
:109AB000184323690B40217D1843C907C90F084388
:109AC000A169931019400843E169382319400843FC
:109AD000216A802319400843A16A93001940084372
:109AE00021680860A0690421000C0840616A102305
:109AF00019400843216848602068C1699143C161E9
:109B00006565012070740020F8BD000010B5006884
:109B10000649884209D10648416B8214914341634A
:109B20000520E0210007FEF729FF10BD00300140AD
:109B30000010024010B586B0044614216846FBF7B9
:109B40005BFB10492068884219D10F48416B821491
:109B500011434163C16A01221143C162C06A0021FD
:109B600010400590E0200090022001900320039017
:109B700002910491052069460007FEF7ADFF06B08B
:109B800010BD00000030014000100240FFB5054646
:109B900004464035287C002781B01646012809D0AC
:109BA00001202874FFF782F80090687C012804D017
:109BB000022797E0022005B0F0BD0298002874D07B
:109BC000002E72D003206874002060650299216322
:109BD000A686E686A063A087E087606420640122F1
:109BE000A068D2034021904208D1206802688A43CD
:109BF0000260206802680B021A4302602068026853
:109C0000520602D402680A4302600121E068C902D8
:109C10008842606828D1002801D0012E1ED1206B17
:109C200021680088C86006E020688168890709D536
:109C3000216B0988C160206B801C2063E08E401E70
:109C4000E0860BE0FFF732F80099411A0498814250
:109C500002D3401C02D005E0002803D0E08E00288B
:109C6000E2D128E003273BE0002801D0012E1FD1DC
:109C7000206B21680078087306E0206881688907F6
:109C800009D5216B09780173206B401C2063E08E9D
:109C9000401EE0860CE0FFF709F80099411A04988D
:109CA000814203D3401C03D0DCE717E00028D9D061
:109CB000E08E0028E1D12046009A049904F00EF8C5
:109CC000002801D020206065A068002803D120680A
:109CD000C16880680090606D002801D0012701E014
:109CE0000120687400202874384664E7FFB50446F4
:109CF00083B00120254640350090287C00271E4671
:109D000001280FD001202874FEF7D0FF0190687C55
:109D1000616801280DD0CA1FFD3A08D1A168002949
:109D200005D102E0022007B0F0BD042801D00227CF
:109D3000D0E0049800287AD005980028FBD0002EA7
:109D4000F9D0687C042801D0052068740020606583
:109D50000599A163E687A68704992163E686A6860E
:109D60002064606420680168490603D401684022C9
:109D7000114301600121E068C9028842606847D14F
:109D8000002801D0012E3CD1206B21680088C860DA
:109D9000206B801C2063E08E401EE08631E020684E
:109DA0008168890710D5E18E00290DD0009901291D
:109DB0000AD1216B0988C160206B801C2063E08E72
:109DC000401EE0860020009020688168C9070DD001
:109DD000E18F00290AD0C068A16B0880A06B801CAD
:109DE000A063E08F401EE08701200090FEF75EFF39
:109DF0000199411A0C98814203D3401C01D00327DA
:109E000066E0E08E0028CAD1E08F0028C7D148E084
:109E1000002801D0012E3ED1206B21680078087304
:109E2000206B401C2063E08E401EE08633E04DE056
:109E300020688168890710D5E18E00290DD000992E
:109E400001290AD1216B09780173206B401C206322
:109E5000E08E401EE0860020009020688168C907DF
:109E60000DD0E18F00290AD0C068A16B0870A06BEB
:109E7000401CA063E08F401EE08701200090FEF7A9
:109E800015FF0199411A0C98814202D3401C02D05F
:109E9000B5E70028B3D0E08E0028C9D1E08F0028B4
:109EA000C6D12046019A0C9903F018FF002803D070
:109EB0000127202060650DE0A068002803D12068FC
:109EC000C16880680090606D002801D0012701E022
:109ED0000120687400202874384624E7094910B529
:109EE000401E884201D9012010BD074C606103214A
:109EF000081F06F06DFF0020A061072020610020F0
:109F000010BD0000FFFFFF0000E000E00248016913
:109F1000022291430161704700E000E0F0B5024683
:109F20002032137E012B21D0012515760223537692
:109F300006687468B3687027BC430F68274377606E
:109F40000068AC07A04208D0094CA04205D0094CDB
:109F5000A04202D0084CA04204D180244968A34307
:109F600019438160557600201076F0BD0220F0BDC7
:109F70000004004000080140001401400246203265
:109F8000137E012B06D001231376006801650020A3
:109F9000107670470220704710B502210446203425
:109FA000617601680A6A094B1A4203D10A685208AD
:109FB00052000A6000F00CF80020A077A076E0764E
:109FC000207760776076207610BD000011110000C8
:109FD000704700000168CA6852085200CA600168F0
:109FE0000A6A064B1A4203D10A68520852000A60F4
:109FF000012120304176002070470000111100003F
:10A0000010B586B0044614216846FBF7F5F80D49F3
:10A010002068884213D10C48C26A04210A43C262F4
:10A02000C06A084005904020009002210020019164
:10A0300002900491039069460448FEF74DFD06B076
:10A0400010BD000000040040001002400008005055
:10A05000F8B5064604462036307E00270D46012816
:10A060000ED001203076002A0CD0042A1BD0082AFA
:10A070002FD00C2A3ED00127002030763846F8BD7C
:10A080000220F8BD206805F03BFA206881690822AB
:10A09000114381612068826904218A4382612068BA
:10A0A0008169EA6812E0206805F042FA2068826956
:10A0B0000121C9020A43826120688169012292025A
:10A0C0009143816120688169EA68120211438161CC
:10A0D000D2E7206805F045FA2068C16908221143DB
:10A0E000C1612068C26904218A43C2612068C169D4
:10A0F000EA6812E0206805F04FFA2068C169012281
:10A10000D2021143C1612068C269012189028A43D8
:10A11000C2612068C169EA6812021143C161ABE7FC
:10A1200070B5050005D02C462034607E002802D092
:10A1300006E0012070BD00202076284600F010F8CF
:10A1400002206076291D286805F0A6F90120A07775
:10A15000A076E076207760776076002070BD000002
:10A1600000680449884204D10348816B02221143EC
:10A170008163704700040040001002407047704740
:10A1800070B504001BD02420E067206801684908EE
:10A19000490001602068002505602068456020684E
:10A1A0008560204600F09EF9204680304560E567D6
:10A1B00005602566656660342576002070BD012047
:10A1C00070BD10B506F0C6FB10BD0000F8B5026802
:10A1D0000446D06911689368A44D06462E40254672
:10A1E0008035002E71D0A24FDE07F60F0F403743A7
:10A1F0007ED0C70706D0CF0504D5012717626A684D
:10A200003A436A60820708D5DA0706D02768022237
:10A210003A626A6804273A436A60420708D5DA0757
:10A2200006D0236804221A626A6802231A436A600D
:10A23000020709D520220A40324305D023680822AC
:10A240001A626B6813436B60020509D54A0107D592
:10A2500001222368D2021A626A6820231A436A60C4
:10A260006A68002A39D0800606D5880604D5A16E12
:10A27000002901D020468847686821688968490616
:10A2800002D4282108422DD0204605F020FB216869
:10A290008868400622D5EFF31080012282F31088EF
:10A2A0008A6840239A438A6080F31088606F002890
:10A2B00014D070498163606FFEF78EF900280CD0CE
:10A2C000606F816B08E000E012E0860610D58E0614
:10A2D0000ED5A16EAFE020468847F8BD2046FFF7B7
:10A2E00070FFF8BD2046FFF76CFF00206860F8BDE6
:10A2F000266E012E7DD1C6067BD5CE0679D51023DC
:10A30000136222689068264640064036002849DAE3
:10A31000616F086840680004000CE8D0378B874202
:10A32000E5D9708308680068800634D4EFF31080A4
:10A33000012181F3108811681F01B943116080F376
:10A340001088EFF31080012181F3108821688A685A
:10A35000520852008A6080F31088EFF310800121C8
:10A3600081F3108821688A684027BA438A6080F3A5
:10A3700010882020286000202066EFF31080012143
:10A3800081F3108821680A689A430A6080F3108874
:10A39000606FFEF7FFF802206066308B718B401A09
:10A3A00081B234E0308B718B401A81B2708B0028FF
:10A3B0009DD000299BD0EFF31080012686F31088F2
:10A3C0001668FF272137BE43166080F31088EFF32D
:10A3D0001080012282F31088226896687608760041
:10A3E000966080F310882020286000202066A066F8
:10A3F00000E010E0EFF31080012282F31088226861
:10A4000015689D43156080F3108802206066204621
:10A41000FFF7B4FEF8BDC50208D55B0206D50120E2
:10A42000000510622046FFF7AAFEF8BD030606D518
:10A430000B0604D5E16E002900D04CE7F8BD4006BC
:10A44000FCD54806FAD52046EFF31081012383F3AB
:10A45000108813684024A343136081F310882021DF
:10A46000C1670021C16600F011FBF8BD0F080000B4
:10A47000200100045DF7000810B5040003D0E06F70
:10A48000002802D007E0012010BD002178200155EE
:10A49000204600F087F82420E0672068016849081A
:10A4A00049000160204605F02BFB0128ECD0606AD2
:10A4B000002802D0204605F08AF820684168092269
:10A4C000D20291434160206881682A2291438160D1
:10A4D00020680168012211430160204605F0DCF884
:10A4E00010BD000070B504460068274B2749284A74
:10A4F00098420FD1886BD30198438863302110466E
:10A50000FEF73CFA606FFEF78DF8206FFEF78AF8D1
:10A510001D200FE01F4D05231B07A8420DD1486BDE
:10A520000122920390434863032149021846FEF733
:10A5300025FA1B20FEF78CFD70BD174DA8420DD1EA
:10A54000886B01225204904388630C211846FEF761
:10A5500015FA606FFEF766F81C20EBE70F4B984288
:10A56000EAD1886B01231B059843886319121046B2
:10A57000FEF704FA04210A48FEF700FA606FFEF7BE
:10A5800051F80E20D6E700000048004000100240BD
:10A5900000080050003801400044004000500040D6
:10A5A000000C0050F0B587B0044614216846FAF755
:10A5B00023FE7C4B22687C490427022603200025C9
:10A5C0009A4248D18A6B73041A438A63CA6A3A432F
:10A5D000CA62C96A03903940059130210091019601
:10A5E0000496029569467148FEF776FA714E7048F6
:10A5F0003060B560F5608027756137610520B56111
:10A60000706020203562F0613046FEF793F8002834
:10A6100001D0FDF7EDF86667B462674E64483146D5
:10A62000503030600520706010200831A1C1756184
:10A63000B561F56130463562FEF77CF8002801D03F
:10A64000FDF7D6F82667002211461D20B462FEF7FA
:10A650001BFD1D2020E0594B9A4221D14A6B01235A
:10A660009B031A434A63CA6A01231A43CA62C96A2E
:10A670000390194005910321490200910520049798
:10A680000196029569460007FEF726FA0022114658
:10A690001B20FEF7F9FC1B20FEF7EAFC07B0F0BD1B
:10A6A000474B9A4234D18A6B01235B041A438A6375
:10A6B000CA6A01231A43CA62C96A03901940059104
:10A6C0000C21009105200497019602956946000728
:10A6D000FEF702FA3B4E3648B5602830F56081C679
:10A6E000F56080203561B0602020B561706135482B
:10A6F000083EFEF71FF8002801D0FDF779F86667DD
:10A70000002211461C20B462FEF7BEFC1C20C3E7E9
:10A710002D4B9A42C2D18A6B01231B051A438A63CF
:10A72000CA6A3A43CA62CA6A3A400592CB6A0822A8
:10A730001343CB62C96A0320114005915102009175
:10A74000039001960496029569461848FEF7C4F9ED
:10A750000320039006200490009701960295694615
:10A760001A48FEF7B9F91248194E14383060B5602E
:10A770000D20F560706075618020B561306120202A
:10A780003562F0613046FDF7D5FF002801D0FDF7B6
:10A790002FF86667002211460E20B462FEF774FCA3
:10A7A0000E2079E7004800400010024000080050E9
:10A7B00030000240FC08002044090020003801401D
:10A7C000004400408C09002000500040000C005064
:10A7D000D409002070B580231B58202B01D0022003
:10A7E00070BD00290BD0002A09D0012483682403FE
:10A7F000A34206D10369002B03D1CB0701D001206E
:10A8000070BD002303660B4B04689C420ED0636846
:10A810001B020BD5EFF31083012585F31088256803
:10A820000126B6063543256083F3108805F072FAD9
:10A8300070BD00000048004070B580231B58202BDD
:10A8400001D0022070BD00290BD0002A09D00124BC
:10A8500083682403A34206D10369002B03D1CB07ED
:10A8600001D0012070BD002303660B4B04689C429D
:10A870000ED063681B020BD5EFF31083012585F31F
:10A88000108825680126B6063543256083F31088B5
:10A8900005F096FA70BD00000048004010B506F0C3
:10A8A0007BF810BD7047FFB50446C06F83B01746F4
:10A8B0000D46202802D0022007B0F0BD002D0BD09D
:10A8C000002F09D00120A1680003814206D1206930
:10A8D000002803D1E80701D00120EDE70021842002
:10A8E00001512120E067FEF7E1F92646403601904C
:10A8F000378277820120A1680003814202D120695A
:10A90000002802D02F46002511E000270FE000228A
:10A910008021204605F014FB002815D1002F17D008
:10A920002168387888627F1C708A401E7082708A25
:10A93000019B002806980090E9D100224021204682
:10A9400005F0FEFA00280AD02020E0670320B3E7D4
:10A9500028882168C005C00D8862AD1CE4E720206E
:10A96000E0670020A8E7000070B50446C06F20280B
:10A9700001D0022070BD00290BD0002A09D001238C
:10A98000A0681B03984206D12069002803D1C8079C
:10A9900001D0012070BD20464030E1640282428235
:10A9A00000202546803568602121E167216F00295C
:10A9B00018D0154BCB62236F14491963236F1449C8
:10A9C0005963216F134688632668E16C324628324A
:10A9D000206FFDF7F7FE002804D0102068602020CB
:10A9E000E067D6E7216840200862EFF3108001217C
:10A9F00081F3108821688A6880231A438A6080F373
:10AA00001088002070BD000079F80008C5F8000823
:10AA100071F7000830B5C36F202B01D0022030BD84
:10AA200000290BD0002A09D0012384681B039C4213
:10AA300006D10569002D03D1CD0701D0012030BD1D
:10AA4000C164014640310A824A8200218422C166E3
:10AA500011502121C1679C4202D1016900290FD008
:10AA60000849C166EFF31081012282F31088006863
:10AA7000026880231A43026081F31088002030BDF1
:10AA80000149EEE7E7FE000889FE000810B506F070
:10AA90001BF810BD7047F0B585B0044600250020B6
:10AAA0000390002602900027002C02D06068002846
:10AAB00001D105B0F0BDA068402800D9F9E7002514
:10AAC0002EE0204600F0E4F82E46002003901FE020
:10AAD000606A825D02AB2046039900F07AF907466E
:10AAE000022F0DD1606A0090E06A01906068029ABE
:10AAF000D20080186A464168204600F0A7F80AE0B4
:10AB0000002F00D107E000BF761C0398401C039083
:10AB1000E06AB042DCD800BF022F00D103E06D1C18
:10AB2000E06AA842CDD800BF00BFC2E70FB438B575
:10AB300004460D4607A80090E169A069009B069AAB
:10AB400006F0F4F8206200200090094800780128FF
:10AB500003D1216AA06900F079FA29462046236AC8
:10AB6000A26900F00FF838BC08BC04B01847000018
:10AB70007805002010B50446A06B01F027FA0020EC
:10AB800010BD0000F8B504460D4616461F463A466D
:10AB9000314620466369984700280AD12046FFF7CE
:10ABA000E9FF0094074B2A460021A06B01F0A6FAAA
:10ABB00006E00094044B01220021A06B01F09EFAF4
:10ABC0000020F8BD0DAD0008FDAC000870B50446CE
:10ABD0000D468021204601F03DFB2868E06368684F
:10ABE0006060A868A060E868E06028692061686922
:10ABF0006061A869A061E869E06100202062286ABC
:10AC00006062686AA0620020E06200213020015585
:10AC1000A86A60632046383001F0ECF9002802D0C1
:10AC20000020C04370BD204600F002F8FAE70000A3
:10AC30000146002901D1401E7047034800680860A2
:10AC4000014801600020F7E77405002070B5044654
:10AC50000D461646022D06D0032D05D0042D04D036
:10AC6000052D07D102E000BF00BF00BF2046FFF75F
:10AC700081FF00E000BF00BF32462946E06B00F0D4
:10AC8000F5F970BD01480078704700007805002094
:10AC900010B50446012240216018FAF7A6FA10BD4B
:10ACA00010B50024124804681FE020462169884737
:10ACB000002819D10F480078012810D1E16A606A94
:10ACC00001F038FB012803D1606A00F03FF906E08B
:10ACD000E16A606A00F086F907A000F037F92046C3
:10ACE000FFF7D9FE0020E0622468002CDDD110BD02
:10ACF00074050020780500200D0A000010B50446F8
:10AD0000002205212046FFF7A1FF10BD10B5044623
:10AD1000002204212046FFF799FF10BD70B50446BC
:10AD20000D46204600F02CF8012801D1801E70BD90
:10AD30002268501CE168FAF7DBF921602369216879
:10AD40005943A368C81829462269FAF73CFA00203B
:10AD5000EDE710B58160C260036101244460002406
:10AD6000046010BD10B504462268501CE168FAF773
:10AD7000BFF96068814201D1012010BD0020FCE7CD
:10AD800010B504462268901CE168FAF7B1F96068D2
:10AD9000814201D1012010BD0020FCE770B50446BE
:10ADA0000D462046FFF7DEFF012801D1801E70BD51
:10ADB000236960685843A368C11828462269FAF7D6
:10ADC00002FA6268501CE168FAF792F961600020AB
:10ADD000EDE7F0B504460D46002600211DE02046B3
:10ADE0004030405C012817D1CF006068C059405DF9
:10ADF000904204D000202746403778540CE0761C5F
:10AE0000CF006068C0596F1CC05D002804D1002BC2
:10AE100000D019600220F0BD491CA0688842DED82D
:10AE2000002E01D10020F6E70120F4E770B50446BA
:10AE30000D46002C01D1401E70BD00BF2068A84205
:10AE4000FCD32068401B206062685019E168FAF763
:10AE50004FF961600020EFE770B504460D46002C05
:10AE600001D1401E70BD20684019206000BFE1681C
:10AE700020688842FBD8A2685019E168FAF738F9CF
:10AE8000A1600020EEE7FFB581B004460D461646EE
:10AE90000027002E06D00498002803D0E16820681F
:10AEA000884203D30020C04305B0F0BD2168E068AC
:10AEB000401AA84202D20020C043F5E7A06840191A
:10AEC000E16888420BD9A168E068471A2168E06808
:10AED000401AE919884202D20020C043E4E7A26880
:10AEE000D019E168FAF704F9316079190498016022
:10AEF0000020D9E7014648687047014688687047D6
:10AF00000246002A01D1401E704700205060906028
:10AF10001060D16000BFF7E70146002901D1012090
:10AF200070470868002801D10120F9E70020F7E701
:10AF30000146002901D1012070470A68C868904283
:10AF400001D10120F8E70020F6E700000FB400B5BA
:10AF50000E48FFB0407882B0002805D07FB002B024
:10AF600008BC002004B01847012183AB49026846A1
:10AF7000829A05F0DBFE06490246884200D90A465D
:10AF80006946002005F034FDE8E700008C01002050
:10AF9000FF0100000FB400B51048FFB0407882B048
:10AFA000002805D07FB002B008BC002004B01847CC
:10AFB00000226946104605F01BFD012183AB4902C2
:10AFC0006846829A05F0B2FE05490246884200D9D9
:10AFD0000A466946002005F00BFDE3E78C010020DE
:10AFE000FF010000F0B5064616480C46417891B0C6
:10AFF000002923D10078012820D10127102C01D964
:10B00000102500E02546402101A8FAF7F5F8402375
:10B0100001AA29463046009701F0CCF80AA101A800
:10B02000FAF7F5F801A8FAF71CF9024601A9002081
:10B0300005F0DEFC641B7619002CDFD1002011B076
:10B04000F0BD00008C0100200D0A000010B5064A7A
:10B050005278002A01D0002010BD0A460146002087
:10B0600005F0C6FC10BD00008C010020F7B582B0D1
:10B0700004460D46002700266088012820D120695B
:10B0800000280AD1606800680195009019A200218B
:10B090002046E368FCF78EFC12E0A90020694058C6
:10B0A00000782D280CD0A9002069405861680968F3
:10B0B0000091019017A200212046E368FCF77AFC7A
:10B0C0006668F36829462046049A984707460CE0CC
:10B0D0007068002808D07068C36829462046049A22
:10B0E00098470746766800E001E0012FF0D000BFE6
:10B0F00005B0F0BD46534D3A252D387320535441C9
:10B1000054453A252D323873204556454E543A253C
:10B11000750D0A0046534D3A252D3873205354417E
:10B1200054453A252D323873204556454E543A251C
:10B13000730D0A00FFB581B004460E461746002580
:10B14000002C01D105B0F0BD30212046FAF754F8AB
:10B150000A98A060049820616660E7600021A162FF
:10B1600061620E48008820800B9860800C4800685F
:10B1700060610B48046009480088401C074908804A
:10B18000656806E06560002211462046FFF76EFF05
:10B19000AD68002DF6D100BFD4E70000D00200203A
:10B1A000CC0200200246002A01D1401E7047D16225
:10B1B0000020FBE7FFB583B005460E461C460C9FFA
:10B1C0000020029020880004B9B20843029002983F
:10B1D000044B009031462846059A00F08FFF07B0D7
:10B1E000F0BD00002D7A0008F7B596B005460E4672
:10B1F0006F680024002015903C462AE06C60002215
:10B2000001212846FFF732FFA64205D1002128463A
:10B21000189AFFF72BFF1EE0502101A8F9F7ECFF69
:10B2200015AB01AA21463046FCF7E1FB00280FD1FF
:10B230000AE015980068686000212846189AFFF710
:10B2400015FF15984068159015980028F1D102E077
:10B250006468002CD2D100BFB46806E06C600021A5
:10B260002846189AFFF702FFA468002CF6D119B0FF
:10B27000F0BD016E05E002467C324B1CD35C53549A
:10B28000491CC26D8A42F6D8704710B5C26D511E76
:10B2900005E002467C32545C4B1CD454491E026EBD
:10B2A0008A42F6DD10BD70B505460C46A879002827
:10B2B00002D001282ED100E000BF432C1BD004DCBB
:10B2C000412C0CD0422C22D10FE0442C19D07E2CE2
:10B2D0001DD100220821284600F040FB18E0002282
:10B2E0000321284600F03AFB12E000220421284600
:10B2F00000F034FB0CE000220621284600F02EFB73
:10B3000006E000220521284600F028FB00E000BFEF
:10B3100000BF2CE0432C1BD004DC412C0CD0422C71
:10B3200022D10FE0442C19D07E2C1DD100220821FF
:10B33000284600F081F818E000220321284600F09A
:10B340007BF812E000220421284600F075F80CE09A
:10B3500000220621284600F06FF806E000220521B1
:10B36000284600F069F800E000BF00BF00BF00BF42
:10B3700070BD70B504460D46432D46D008DC1B2D2C
:10B380000DD0332D25D0412D3DD0422D4DD13BE068
:10B39000442D3BD05B2D11D07E2D46D124E0207969
:10B3A000002802D0042804D100E000BF0120207151
:10B3B00002E00020207100BF00BF39E020790128A1
:10B3C00002D10220207102E00020207100BF00BFE6
:10B3D0002EE02079022802D10320207102E0002013
:10B3E000207100BF00BF23E02079032806D1294641
:10B3F0002046FFF758FF0420207102E00020207152
:10B4000000BF00BF14E000BF00BF00BF20790228CA
:10B4100006D129462046FFF746FF0420207102E0AE
:10B420000020207100BF00BF02E00020207100BF9B
:10B4300000BF207970BD0000F7B504460D46092D08
:10B4400002D00020A066E0662B0005F0B4FC0AFDE7
:10B450000646CBFCFBFAF9F8F7FD6079002802D02C
:10B46000012837D100E000BFE06D63282FD20B2008
:10B47000C00120188169029888472046FFF705FF20
:10B48000029821467C31226E8854206E401C206632
:10B49000E06D401CE065266E002709E022467C3204
:10B4A000905D0B22D201A21891698847761C7F1CFF
:10B4B000E06DB042F2D805E00B20C0012018816990
:10B4C0000820884738467F1E0028F5D100BF00209D
:10B4D000607100E000BF00BF3EE2E06D002806D1D1
:10B4E0000B20C00120184169FEA0884734E2607932
:10B4F000002802D0012856D11FE0002120467C30D0
:10B50000E26D81546422616F51430246C83288184B
:10B5100021467C31F9F7C7FE606F401C6067606FA1
:10B520000A2801DB00206067A06F401CA067A06FA5
:10B530000A2801D30A20A06736E000BF00BF6422BA
:10B54000206F50432246FF32453281186422E6487C
:10B550002018F9F738FE266F11E00A21701CF9F760
:10B56000C7FD0F4664227A432346FF334533D11883
:10B5700064227243D0186422F9F725FE3E46616FBB
:10B58000084609300A21F9F7C9FDB142E5D1642125
:10B5900071432246FF32453288186422D24961182D
:10B5A000F9F711FE00E000BF00BF0B20C00120181A
:10B5B0004169CEA08847204600F002FD20467C303D
:10B5C00000F054FC002000F0FBFC00202066E06549
:10B5D000606F0A3020670B20C00120184169C4A0A9
:10B5E0008847B9E16079002802D0012855D100E0F0
:10B5F00000BFA06F002800D150E0A06F0A2803D13F
:10B60000616F206F88420CD1A06F0A2842D0616F11
:10B610000A31A26F881A0A21F9F76AFD206F814268
:10B6200038D0216F084609300A21F9F761FD2167FA
:10B630006422206F50432246FF3206E01CE1DBE02B
:10B6400096E084E076E02BE085E1453281182046E3
:10B650007C30F9F728FE20467C30F9F702FEE065E1
:10B66000E06D20660B20C00120184169A1A0884729
:10B670006423226F5A432346FF334533D0180B22ED
:10B68000D201A218516988470B20C00120184169D6
:10B6900099A088470120607100E000BF00BF5BE116
:10B6A0006079002802D0012841D100E000BFA06FDE
:10B6B000002800D13CE0616F084609300A21F9F703
:10B6C0002DFD206F81422FD0216F481C0A21F9F7F0
:10B6D0000FFD21676422206F50432246FF3245321E
:10B6E000811820467C30F9F7DEFD20467C30F9F7E2
:10B6F000B8FDE065E06D20660B20C00120184169AF
:10B700007CA088476423226F5A432346FF33453386
:10B71000D0180B22D201A218516988470B20C00112
:10B720002018416974A088470120607100E000BFC3
:10B7300000BF11E1206E002808DD206E401E20664B
:10B740000B20C001201881690820884704E1E16DC1
:10B75000206E88420BD222467C32236ED05C0B22B4
:10B76000D201A21891698847206E401C2066F3E040
:10B770006079002802D001283BD100E000BFE06DD5
:10B78000002833D0206E002830DD0B20C0012018A7
:10B79000816908208847266E012709E022467C320D
:10B7A000905D0B22D201A21891698847761C7F1CFC
:10B7B000E06DB042F2D80B20C00120188169202032
:10B7C000884705E00B20C0012018816908208847C0
:10B7D00038467F1E0028F5D1206E401E2066204688
:10B7E000FFF747FDE06D401EE06500BF002060717F
:10B7F00000E000BF00BFAFE06079002802D0012860
:10B8000037D100E000BFE06D00282FD0206E002867
:10B810002CDD216EE06D884228D0206E461C012769
:10B8200009E022467C32905D0B22D201A218916978
:10B830008847761C7F1CE06DB042F2D80B20C00117
:10B84000201881692020884705E00B20C0012018BE
:10B8500081690820884738467F1E0028F5D1204698
:10B86000FFF707FDE06D401EE06500BF002060713E
:10B8700000E000BF00BF6FE06079002802D001281F
:10B8800066D100E000BFE06D00285ED0E06E0028C9
:10B890000AD10120E06621467C312046E030E26D8D
:10B8A000F9F791FCE06D606642E0A06E00F026FBC7
:10B8B00006462146E031626EF9F7FEFC002834D1DD
:10B8C0000B20C001201841690CA08847A06E00F031
:10B8D00015FB06460B20C0012018416930468847F9
:10B8E000A06E0FE00D0A3E002C0500000D0A0000BE
:10B8F0003E0000000D3E00001B5B4A000D1B5B4A32
:10B900003E00000000F0FAFA0646314620467C3040
:10B91000F9F7C9FC20467C30F9F7A3FCE065E06D3F
:10B920002066A06E401CA06607E0A06E401CA066CA
:10B9300000F0DEFAA16E8842B7D800BF00F0D8FA56
:10B94000A16E884201D80020A0660020607100E04E
:10B9500000BF00BF00E000BF00BFFEBDF7B504465A
:10B960000E46330005F027FA09F2064EF2F2B0BD9A
:10B97000D8F1F200E06D632843D2A079012806D106
:10B980000B20C001201881692A20884705E00B2080
:10B99000C00120188169029888472046FFF775FC8E
:10B9A000029821467C31226E8854206E401C20660D
:10B9B000E06D401CE065256E002713E0A0790128AA
:10B9C00006D10B20C001201881692A20884707E092
:10B9D00022467C32505D0B22D201A2189169884721
:10B9E0006D1C7F1CE06DA842E8D805E00B20C0016B
:10B9F000201881690820884738467F1E0028F5D125
:10BA00000DE10CE1E06D002809D1A079002806D1F4
:10BA10000B20C0012018416982A08847FFE0A0796F
:10BA2000002802D001284CD117E0002120467C30AC
:10BA3000E26D81540B20C001201841697DA0884728
:10BA40000120A07100202066E06522467C32102192
:10BA500020460C3000F07BFD34E0002120467C3095
:10BA6000E26D81540020E06522467C324021204670
:10BA70001C3000F06CFD21461C3120460C3000F0DB
:10BA80008BF900280CD10B20C001201841696DA052
:10BA900088470220A07100202066E06560710FE0F9
:10BAA0000B20C001201841696AA088470B20C00103
:10BAB000201841695BA088470020A0712066E065DE
:10BAC00000E000BF00BFAAE0206E002808DD206E65
:10BAD000401E20660B20C00120188169082088477D
:10BAE0009DE0E16D206E884215D2A079012806D133
:10BAF0000B20C001201881692A20884708E02246CF
:10BB00007C32236ED05C0B22D201A2189169884747
:10BB1000206E401C206682E0E06D00283FD0206E41
:10BB200000283CDD0B20C0012018816908208847CF
:10BB3000256E012715E0A079012808D10B20C0014E
:10BB4000201881692A20884709E029E066E022461A
:10BB50007C32505D0B22D201A218916988476D1C7E
:10BB60007F1CE06DA842E6D80B20C0012018816937
:10BB70002020884705E00B20C0012018816908209B
:10BB8000884738467F1E0028F5D1206E401E20666B
:10BB90002046FFF76EFBE06D401EE06500BF3EE013
:10BBA000E06D002839D0206E002836DD216EE06D72
:10BBB000884232D0206E451C012713E0A07901286D
:10BBC00006D10B20C001201881692A20884707E090
:10BBD00022467C32505D0B22D201A218916988471F
:10BBE0006D1C7F1CE06DA842E8D80B20C001201816
:10BBF00081692020884705E00B20C0012018816959
:10BC00000820884738467F1E0028F5D12046FFF7D8
:10BC100030FBE06D401EE06500BF00E000BF00BFEC
:10BC2000FEBD00000D0A757365726E616D653A2088
:10BC3000000000000D0A70617373776F72643A2020
:10BC4000000000000D0A57656C636F6D65210D0AD9
:10BC50003E0000000D0A55736572207665726966B4
:10BC600079206661696C65642E00000038B500209B
:10BC700000900024414804687CE072E000F0EAF99A
:10BC80000546684601782046FFF773FB002800D080
:10BC900067E0A068281A3A49884205D9A5600220C1
:10BCA000A0710020E0652066A079002802D001285C
:10BCB0002BD100E000BF684600780D2806D1684609
:10BCC000027802212046FFF749FE1DE06846007811
:10BCD0000A2819D068460078082805D100220721D3
:10BCE0002046FFF73BFE0FE068460078092805D1A3
:10BCF000002209212046FFF731FE05E06846027860
:10BD000001212046FFF72AFE29E0684600780D2829
:10BD100006D16846027802212046FFF78DFB1DE020
:10BD2000684600780A2819D068460078082805D1A6
:10BD3000002207212046FFF77FFB0FE068460078CE
:10BD4000092805D1002209212046FFF775FB05E0EF
:10BD50006846027801212046FFF76EFB00BF00BF56
:10BD600000BF0B20C0012018C16968468847002821
:10BD700084D02468002C80D138BD0000E802002067
:10BD800040771B0003490968016002218171014964
:10BD900008607047E802002002460020704700005B
:10BDA00000BFEFF30580002800D070470748006807
:10BDB000002804D1012080F3108800BF00BF034891
:10BDC0000068401C0149086000BFEEE7D402002073
:10BDD00070B504460D4600F0A3F800280FD000F01F
:10BDE0009FF80B21C90140180069002807D000F016
:10BDF00097F80B22D2018018016902A08847002021
:10BE000070BD00001B5B481B5B4A000070B502461A
:10BE10000C4600210023002A01D0002C02D1002072
:10BE2000C04370BD0021002316E0C8000D4D285806
:10BE3000002810D1D8001058CD000A4E7051D800FB
:10BE400080184068CD00AD19686007480068401C44
:10BE5000054D28605B1C491C502901D2A342E4D344
:10BE60000020DEE7F4020020F0020020F0B595B0DB
:10BE70000446002600E0641C20782028FBD02046E1
:10BE8000F9F7EFF9002801D115B0F0BD2046F9F718
:10BE9000E8F90019461E02E000203070761E307866
:10BEA0002028F9D0142301AA2021204600F078FB95
:10BEB0000746002513E0E9000C4A50582146F9F7DF
:10BEC000D7F900280AD1E8000849401801A94268BA
:10BED00038469047002800D105E004E06D1C00F0D2
:10BEE00007F8A842E7D800BF0020CDE7F402002001
:10BEF0000148006870470000F00200200146054834
:10BF00000068814201D304A07047C800034A10585A
:10BF1000FAE70000F002002000000000F402002018
:10BF20000148006870470000EC020020F8B50646A2
:10BF30000F46002536E0002418E0FFF7F1FF002847
:10BF400013D0FFF7EDFF0B21C9014018006900284D
:10BF50000BD0FFF7E5FF0B23DB01C018026928199E
:10BF6000C000134B195813A09047641C052C04DA29
:10BF7000FFF7BEFF29198842DFD8FFF7D1FF00285D
:10BF80000FD0FFF7CDFF0B21C90140180069002831
:10BF900007D0FFF7C5FF0B22D2018018016907A067
:10BFA00088476D1DFFF7A4FFA842C4D80020F8BD44
:10BFB000F4020020252D3136730000000D0A000028
:10BFC0000149086070470000EC020020014620296A
:10BFD00002D30020C0437047012218204843044B7D
:10BFE0001A50002218204843C01882600020F2E74F
:10BFF000083B002070B505460024002D01D1401EED
:10C0000070BD00240CE0182060430C49085800283B
:10C0100005D1012118206043084A115002E0641C38
:10C02000202CF0D300BF202C05D105A0FEF78EFFF9
:10C030000020C043E4E72C600020E1E7083B00203B
:10C0400074696D65722049442069732066756C6C53
:10C050000D0A00000148006870470000D802002067
:10C0600010B5002400BF41E0182060432149085862
:10C0700002283AD118206043401880681E49096898
:10C08000091A182060431B4A8018C06881422CD9C5
:10C0900018206043114640184069002820D018201D
:10C0A000604340180079002804D101211820604322
:10C0B00011500AE00221182060430E4A11500E4828
:10C0C0000168182060438018816018226243094B80
:10C0D000D218106918226243D2185169884704E0C7
:10C0E000012118206043034A1150641C202CBBD34B
:10C0F00010BD0000083B0020D8020020F0B5044627
:10C10000059D202C02D30020C043F0BD022618203C
:10C1100060430E4F3E50182060433E468019017127
:10C120000B48066818206043C019866018206043D9
:10C130003E468019C2601820604380194361182070
:10C140006043801905610020DFE70000083B002004
:10C15000D802002007480068401C064908600648CD
:10C16000026840680021521C484103490A60486047
:10C1700070470000D8020020E002002000BFEFF36B
:10C180000580002800D0704709480068002804D0C6
:10C1900007480068401E06490860054800680028F6
:10C1A00004D100BF80F3108800BF00BF00BFEAE7E2
:10C1B000D4020020FFB581B005460C4600260023BE
:10C1C00000200090002D03D0002A01D0002C02D1C5
:10C1D000002005B0F0BD0A98012801D1032000E03D
:10C1E00002206043401C0499884201D90020F0E7F6
:10C1F000002618E0A85D00900099081100F019F8D9
:10C2000019465B1C505400990807000F00F011F804
:10C2100019465B1C50540A98012803D12021184666
:10C220005B1C1154761CA642E4D30020D05418465F
:10C23000CFE70146092903DC08463030C0B2704719
:10C240000A2905DB0F2903DC08463730C0B2F6E7C0
:10C250003020F4E770B504460D4629462046F8F72D
:10C26000CBFF70BD0146302904DB392902DC0846CA
:10C2700030380EE0412904DB462902DC0846373815
:10C2800007E0612904DB662902DC0846573800E034
:10C290000020C0B2704710B502460B46002406E0ED
:10C2A0001078FFF7DFFF21014418521C5B1E002BA2
:10C2B000F6D1204610BD00B50246002305E01078F7
:10C2C000FFF7D0FF19014318521C10780028F6D14F
:10C2D000184600BD70B588B005460C460020079092
:10C2E0000690059004902846F8F7BBFF064604A880
:10C2F00005A906AA07AB0092019102900AA2314655
:10C30000284600F031F8042803D00020C04308B0CC
:10C3100070BD07982070069860700598A07004980A
:10C32000E0700020F3E7000025642E25642E2564CC
:10C330002E25640002460B46002100BF10E0505C31
:10C34000202803DB505C7E2800DC08E0505C0D28D0
:10C3500002D0505C0A2800D101E000207047491C3F
:10C360009942ECD30120F9E70FB4F0B585B004464B
:10C370000020049000222020039000200290002C36
:10C3800002D00C98002805D1002005B0F0BC08BCF4
:10C3900004B018470DA80490CFE0002908D10C98EC
:10C3A0000078252803D10C984078652800D0C9E092
:10C3B0000C98007825286ED10C98401C0C900C9895
:10C3C000007803900C98401C0C900398652877D057
:10C3D00004DC2A2807D0642873D113E0702872D0B7
:10C3E0007828F9D13EE008E020780C9B1B78984231
:10C3F00002D0641C491E00E001E00029F4D100BF16
:10C40000521C88E00026019600960023002520207B
:10C41000049E20CE049618E02078009E002E05D1C0
:10C420002D2803D10126019600960CE0302809DB67
:10C43000392807DC012600960A265E430746303F6E
:10C44000F31900E003E0641C491E0029E4D100BF99
:10C45000019E012E01D1DE43731C002D00D02B6004
:10C46000521C58E000230025049E20CE04961FE0B5
:10C470002078302806DB392804DC1E010746303FCF
:10C48000F31913E0612807DB662805DC1F01064667
:10C49000573EBB190AE043E0412806DB462804DC8E
:10C4A0001F010646373EBB1900E003E0641C491E2D
:10C4B0000029DDD100BF002D00D02B60521C2AE0E6
:10C4C0001BE024E0FFE7049E01CE04960025002334
:10C4D000254609E026780C9F3F78BE4201D05B1CC0
:10C4E00000E003E0641C491E0029F3D100BF0028CE
:10C4F00001D005604360521C0DE0049B01CB049306
:10C50000002800D00460521C0123029303E00120A4
:10C510000290002200BF00BF029801280DD111E057
:10C5200020780C9B1B78984205D1641C0C98401C09
:10C530000C90491E01E0002204E00C9800780028CD
:10C5400000D02AE700BF0020049010461DE70FB47A
:10C55000F8B506460C46002509A80090214630464D
:10C56000009B089A04F0E2FB054600200090A542DB
:10C5700000D3651E2846F8BC08BC04B0184710B5A7
:10C5800002460B46002407E01078FFF76BFE0A21F5
:10C5900061434418521C5B1E002BF5D1204610BD90
:10C5A000FFB504461D4621460023002D03D0002C74
:10C5B00001D0002A02D1002004B0F0BD18465B1C57
:10C5C000800011500BE00E780198864206D10020C1
:10C5D0000870481C1E465B1CB6009051491C087828
:10C5E000002801D0AB42EED31846E5E770B5064609
:10C5F0000025002478213046F8F729FE0446002C57
:10C6000004D158213046F8F722FE0446002C0BD006
:10C61000641C05E02078FFF725FE29014518641CFD
:10C6200020780028F6D103E03046F8F754FE05469E
:10C63000284670BD10B503460C46002100BF05E03A
:10C64000585CA04201D1581810BD491C9142F7D343
:10C650000020F9E770B504460D46002C01D0002DEE
:10C6600002D10020C04370BD012120461030FEF7EA
:10C67000DDFB20462030A968FEF7D8FB0020F2E75A
:10C6800070B504460D46002C01D0002D02D10020CB
:10C69000C04370BD012120461030FEF7DDFB20466F
:10C6A0002030A968FEF7D8FB0020F2E710B5044659
:10C6B000002C00D110BD20461030FEF72DFC0128C3
:10C6C00001D10020F6E720462030FEF725FC0128A6
:10C6D00001D10020EEE720461030FEF70BFC0C21C4
:10C6E000484321684018E5E77CB504460E4600251E
:10C6F000002001900090002C00D17CBD204610301D
:10C70000FEF716FC002801D00020F6E76B4601AAD0
:10C71000314620462030FEF7B6FB002801D000202D
:10C72000EBE720461030FEF7E8FB0C214843216878
:10C730004518A0680199401828606E600098A860AC
:10C740002846DAE7FFB581B004460E461D460027AD
:10C750000C2068430399884202D3781E05B0F0BDCF
:10C760000C202F4647432660676060688019A060F0
:10C770000398C11BE160294620461030FEF7C0FB3C
:10C7800020462030E168FEF7BBFB0020E6E7FEE72D
:10C7900070B501240E4D6403002221462846FCF7A3
:10C7A0007EFA002261002846FCF779FA0A2004F09C
:10C7B000DBFF012221462846FCF771FA0A2004F02B
:10C7C000D3FF002221462846FCF769FA70BD00001D
:10C7D0000004005070B501240E4D64030022214670
:10C7E0002846FCF75CFA012291032846FCF757FA29
:10C7F0000A2004F0B9FF012221462846FCF74FFA2F
:10C800000A2004F0B1FF002221462846FCF747FA2F
:10C8100070BD000000040050F1B500240126164F41
:10C8200025467603002231463846FCF738FA0A20BE
:10C8300004F09AFF012231463846FCF730FA6006D0
:10C84000040E012189033846FCF724FA002801D0A0
:10C85000641CE4B2052004F087FF6D1CEDB2082DC6
:10C86000E0D30098002803D0FFF792FF2046F8BDE0
:10C87000FFF7B0FFFAE7000000040050F8B501260A
:10C88000164F05467603002231463846FCF707FA74
:10C890000024E80901D0012200E0002201218903DF
:10C8A0003846FCF7FCF96806050E0A2004F05CFF28
:10C8B000012231463846FCF7F2F90A2004F054FF11
:10C8C000002231463846FCF7EAF90A2004F04CFF12
:10C8D000641CE4B2082CDCD3F8BD00000004005056
:10C8E00070B501220C4D940321462846FCF7D7F978
:10C8F0000122560331462846FCF7D1F90022214691
:10C900002846FCF7CCF90A2004F02EFF002231461D
:10C910002846FCF7C4F970BD0004005070B501242E
:10C920000E4D6403002221462846FCF7B8F9660044
:10C93000002231462846FCF7B2F90A2004F014FF21
:10C94000012221462846FCF7AAF901223146284651
:10C95000FCF7A5F90A2004F007FF70BD00040050A1
:10C96000F8B50122144D9603002431462846FCF701
:10C9700096F9062004F0F8FE0122570339462846AE
:10C98000FCF78DF9062004F0EFFE07E0641CE4B22A
:10C99000FA2C03D9FFF7C2FF0120F8BD3146284623
:10C9A000FCF778F90028F1D1002239462846FCF737
:10C9B00076F90020F8BD00000004005010B50A48C8
:10C9C000018C012903D100210184FCF761FB064899
:10C9D000064A40380188914202D1C088002801D11E
:10C9E000FCF756FB10BD0000B8370020AA55000028
:10C9F00010B5F9F7D1FC002801D00020C04310BDCC
:10CA000010B5FAF7DBFB10BD10B500220F2102486C
:10CA1000FEF72CFB002010BD3010002010B5184888
:10CA200000F032F81648401E4178817037212020EE
:10CA300000F071F80321212000F06DF84021222040
:10CA400000F069F80821232000F065F8AA213020C1
:10CA500000F061F80B4802210187322000F05BF8FA
:10CA60000121332000F057F85F21202000F053F817
:10CA7000034800F009F80A2004F076FE10BD00001B
:10CA8000C30200207837002010B501460F2000F0C7
:10CA900021F8002800D0012010BD10B50446FFF792
:10CAA0001FFF3220FFF7EAFEFFF75AFFE0B2FFF761
:10CAB000E5FEFFF755FFFFF713FF3320FFF7DEFE1C
:10CAC000FFF74EFF0020FFF7A7FE0446FFF726FF03
:10CAD000204610BD10B50C46FFF7DFFF2070012087
:10CAE00010BD70B50D460446FFF7FAFE3220FFF781
:10CAF000C5FEFFF735FFE0B2FFF7C0FEFFF730FFDE
:10CB00002846FFF7BBFEFFF72BFFFFF707FF0A20C2
:10CB100004F02AFE70BD10B5FFF7E3FF012010BD41
:10CB200010B50248FCF76DF910BD0000F0050020BB
:10CB3000FEB504460027EFF310800290012080F339
:10CB40001088344B2168CA1804D13348C7680320C1
:10CB50008004074088680190C868009048698E6921
:10CB6000002A08D12C4940398A6ACD042A438A62B6
:10CB70008A6AAA438A62014631433CD02549226829
:10CB8000CA4205D12449CB68032292049343CB6067
:10CB900025462035002810D021680A6901231A4350
:10CBA0000A61216848610821204600F037F803280F
:10CBB00000D1A873216808204860002E10D020689A
:10CBC000016901221143016120688661102120461C
:10CBD00000F024F8032800D1A873216810204860D1
:10CBE0000C482168C14206D10B48C1680322920457
:10CBF00091433943C16020680169490849000161D6
:10CC000021680198886021680098C860029880F3C4
:10CC10001088FEBD0084FFBF4010024070B506467C
:10CC20000B480D46002409490068F8F761FA7D2198
:10CC3000C90048433168401E00D103240B682A46CE
:10CC40009A4301D00028F6D1204670BD204E000046
:10CC5000A400002010B50248FDF7B8FA10BD00008E
:10CC6000200600201CB5002118480091164A0191A9
:10CC70000260C16312054260816007228263012263
:10CC800002610246C16020321170FF235170C2332D
:10CC900043628162117301638161042241634261D5
:10CCA000C161FBF7D9FA002801D072B6FEE7084847
:10CCB00000908013019069460448FBF77DFA002834
:10CCC00001D072B6FEE71CBD00240140840500209F
:10CCD00002000004F0B587B014216846F8F78CFA1A
:10CCE0005548C26A04210A43C262C26A0A400592D8
:10CCF000C16A01252943C162C16A29400591C16AFF
:10CD000002263143C162C16A31400591C26A0821DD
:10CD10000A43C262C06A0122084005900C214748BC
:10CD2000FBF7BDFF81210520002209010007FBF769
:10CD3000B6FF002242494348FBF7B1FF01224249B6
:10CD40004048FBF7ACFF91210520012209020007B2
:10CD5000FBF7A5FF1320400211273F040024009099
:10CD60006946019702943548FBF7B6FE0C20009007
:10CD700002946946019503943048FBF7ADFE052007
:10CD800069460007019700950294FBF7A5FE2F481E
:10CD90000090052002946946019503940007FBF773
:10CDA0009BFE2B4800900294694601950394254808
:10CDB000FBF792FE69462348009602950194FBF723
:10CDC0008BFE280300906946019702941D48FBF7EB
:10CDD00083FE0320400300900320039001950294FA
:10CDE00069461848FBF778FEE8020090019469460E
:10CDF00002941248FBF770FE6802009001946946A5
:10CE000002941048FBF768FE002202210520FCF77F
:10CE10003BF90520FCF72CF9002211460720FCF70E
:10CE200033F90720FCF724F905200122102100071F
:10CE3000FBF735FF07B0F0BD0010024000080050BE
:10CE4000810400000004005060E000001099000020
:10CE5000E184000010B50E480C490160FF21053146
:10CE6000416000218160C16001614161C1610122B5
:10CE7000016252024162826181620721C162FCF754
:10CE8000E9FD002801D072B6FEE710BD0030014078
:10CE90006408002010B586B0002405941E48049450
:10CEA0000094019402941B49039401601F21846043
:10CEB00041600461F9214461C160FDF731F9002846
:10CEC00001D072B6FEE7049404A913480594FDF757
:10CED00025F8002801D072B6FEE7602000907D2082
:10CEE000019002940022694603940B48FDF7B0F8C4
:10CEF000002801D072B6FEE704210748FDF73EF88E
:10CF0000002801D072B6FEE70348FDF779F806B0B5
:10CF100010BD000000040040BC08002010B50C4803
:10CF20000A490160E1214902416000218160C1603C
:10CF300001618161C1610C22016242614162FDF7C0
:10CF40009BFA002801D072B6FEE710BD0038014000
:10CF5000A806002010B50C480A490160E1214902E9
:10CF6000416000218160C16001618161C1610C2269
:10CF7000016242614162FDF77FFA002801D072B67A
:10CF8000FEE710BD004400403007002010B50C48FB
:10CF90000A490160E1214902416000218160C160CC
:10CFA00001618161C1610C22016242614162FDF750
:10CFB00063FA002801D072B6FEE710BD00500040B1
:10CFC000B807002010B512480078002807D0114893
:10CFD000FBF7A8FE01210846FCF770F810BD00F031
:10CFE0002DF9FAF7C7FAFFF7E9FCFAF7EFFFFFF7B9
:10CFF0000BFDFFF735F8FDF753FE03F0C3FA0548C4
:10D00000FBF790FE00F0C6F801F01CFF10BD000019
:10D0100002000020E005002000487047801000203A
:10D0200000487047601000200048704770100020D2
:10D0300000487047B8100020024900230A5C0B54D6
:10D04000104670475D010020024900230A5C0B5422
:10D05000104670476001002010B5044A536A002B47
:10D0600001D0926A9847002010BD000054010020B2
:10D07000034A012111540021D21C11540846704763
:10D080005D010020034A012111540021D21E1154D8
:10D09000084670476001002010B5002809D0064AF4
:10D0A00001219170024680210448FFF750FA0020C8
:10D0B00010BD0020C04310BD54010020B810002056
:10D0C0000249002288788A707047000054010020CD
:10D0D0000020704710B5192904D28A1E0146024863
:10D0E000F8F771F8002010BD8010002010B502295B
:10D0F00002D20020C04310BD8C1E102C07D2014666
:10D1000022460448F8F75FF802490020085500203D
:10D1100010BD00006010002010B5022902D20020CE
:10D12000C04310BD8C1E102C07D201462246044875
:10D13000F8F749F8024900200855002010BD00000A
:10D14000701000200249002208780A707047000021
:10D150005401002070B5054C0546A269002A01D093
:10D16000616990470020256170BD000054010020D6
:10D17000FEE7000010B501200449024608600103E3
:10D1800005200007FBF78BFD10BD00008C00002080
:10D1900070470000F8B50126214D36033146284678
:10D1A000FBF778FD1F4C002835D0FEF753FF61696F
:10D1B000401A7D21C900884230D31B4F1B4831469D
:10D1C00007601B4807601B4807601B48076028462C
:10D1D000FBF760FD0028F1D1A061FEF73BFF2F4671
:10D1E00005252D076061FEF735FF6169401A642847
:10D1F000F9D3002231462846FBF751FD01210022D8
:10D2000089023846FBF74BFDFF21002201312846F9
:10D21000FBF745FDE7E7FEF71DFF6061F8BD000085
:10D2200000040050D40100201111110088000020DA
:10D23000840000208C00002090000020F8B501211F
:10D2400049027648FBF726FD0024754E754D0028EF
:10D2500073D0754F7548BC81BC710460744804601C
:10D26000744804603460744839780078014358D1B8
:10D27000FAF736F90320FAF723FA0120387050E064
:10D280006E480480FEF7E6FE67490969411A6C485A
:10D29000814224D96B48FBF745FD63486249808988
:10D2A000801D8881FEF7D6FE5F4908610121890251
:10D2B0003846FBF7EFFC002803D0FAF717FF287079
:10D2C0000DE0012291023846FBF7E9FCFAF70EFF68
:10D2D00028700121002289023846FBF7E0FC2878FB
:10D2E00063280ED350498879002807D08889E12126
:10D2F000C900884205D31120000404E00120887190
:10D300008C81112000023060642004F026FAFAF7C4
:10D3100031F9FFF779FB002211461046336800F01F
:10D32000D9FD3E4F012149023846FBF7B3FC0028E6
:10D3300003D0FAF7E7F80328A2D03B4F7C70387887
:10D34000002807D00020FAF7BBF93C706420B870C1
:10D35000FFF710FF012149023048FBF79BFC002832
:10D3600001D135480470FEF775FE7D21C900F7F73D
:10D37000BFFE38790A2913D2002821D128780F2836
:10D3800001D9112001E01120000230600120387124
:10D3900028483368026826480168244800680DE080
:10D3A00000280DD03C71214934600C602049204692
:10D3B0000C60204903460C600246014600F08AFDDD
:10D3C000FEF748FE3969411A1D48814210D9FEF71F
:10D3D00041FE0124114EA402386121463046FBF77C
:10D3E00059FC002807D0FAF781FE287011E0297057
:10D3F000F8BDB870F8BD012221463046FBF74FFC5E
:10D40000FAF774FE2870002221463046FBF747FCED
:10D410002878B9788842ECD9E9E700000004005088
:10D420009000002000000020D40100208400002093
:10D43000880000208C0000208E01002008000020C1
:10D4400070170000E0050020FEB504F019FB314D17
:10D450000320688130496980EA88322A01D2642138
:10D4600003E07D21C9008A4200D9E980298F0A2979
:10D4700001D902212987E98E432901D94321E9866F
:10D48000A98A264A914201D10A21A982A98C244A5B
:10D49000914201D90021A9841E4C224A4034218E98
:10D4A0004B260F46B43F0123F600974202D30129D1
:10D4B0002ED026862386E18FB439914200D3E687A9
:10D4C000E121C900E187698F782901D9782169872D
:10D4D000154AE98F1172154908701548A98801602D
:10D4E00014A003F0FFFB6888C2B2010A15A003F084
:10D4F000F9FBE18DA08D00900191638D228DE18C6F
:10D5000019A003F0EFFB218E1FA003F0EBFBFEBD83
:10D510002386CFE77837002001030000FFFF0000DB
:10D52000102700005D0D0000D401002080000020C5
:10D530007C000020C9E8B1B849443A202578202E63
:10D540000D0A0000B9CCBCFEB0E6B1BE3A20204CBA
:10D55000303731CEDE555742B9A4BFA85625642EC8
:10D5600025642E200D0A0000B7FECEF1C6F7B5D80F
:10D57000D6B73A2025642E25642E25642E25643ADC
:10D5800025642E0D0A000000B5B1C7B0D4CBB6AFEC
:10D59000CAB1475053B9A4D7F7BCE4B8F43A202530
:10D5A00064202E0D0A00000000B504498020886226
:10D5B000FF20F53004F0ECFA00BD0000000400503C
:10D5C000112302461B0200B519020D489A4202D1EE
:10D5D00000F0C0F800BD8A4202D100F057F809E01F
:10D5E000112A04D0824205D100F002F900BD00F0FA
:10D5F00009F800BD002AFCD100F07AF800BD000057
:10D600001111110000B500F02FF800F02DF800F016
:10D610002BF800F029F800F027F800F025F800F0CA
:10D6200023F800F021F800F01FF800F01DF800F0DA
:10D630001BF800F019F800F017F800F015F800F0EA
:10D6400013F800F011F800F0B7F800F0B5F800F0AA
:10D65000B3F800F0B1F800F0AFF800F0ADF800F06A
:10D66000ABF800F0A9F800BD07488021816100BF38
:10D6700000BF00BF00BF00BF00BF816200BF00BF8E
:10D6800000BF00BF00BF70470004005000B500F0AD
:10D6900093F800F091F800F08FF800F08DF800F0AA
:10D6A0008BF800F089F800F087F800F085F8FFF7B4
:10D6B000DBFFFFF7D9FFFFF7D7FFFFF7D5FFFFF736
:10D6C000D3FFFFF7D1FFFFF7CFFFFFF7CDFFFFF746
:10D6D000CBFFFFF7C9FFFFF7C7FFFFF7C5FFFFF756
:10D6E000C3FFFFF7C1FFFFF7BFFFFFF7BDFF00BD9F
:10D6F00000B5FFF7B9FFFFF7B7FFFFF7B5FFFFF77B
:10D70000B3FFFFF7B1FFFFF7AFFFFFF7ADFFFFF785
:10D71000ABFFFFF7A9FFFFF7A7FFFFF7A5FFFFF795
:10D72000A3FFFFF7A1FFFFF79FFFFFF79DFFFFF7A5
:10D730009BFFFFF799FFFFF797FFFFF795FFFFF7B5
:10D7400093FFFFF791FFFFF78FFFFFF78DFFFFF7C5
:10D750008BFF00BD00B5FFF787FFFFF785FFFFF7E1
:10D7600083FFFFF781FFFFF77FFFFFF77DFFFFF7E5
:10D770007BFFFFF779FF00F01FF800F01DF800F0C5
:10D780001BF800F019F800F017F800F015F800F099
:10D7900013F800F011F8FFF767FFFFF765FFFFF7D9
:10D7A00063FFFFF761FFFFF75FFFFFF75DFFFFF725
:10D7B0005BFFFFF759FF00BD0C488021816100BF6E
:10D7C00000BF00BF00BF00BF00BF00BF00BF00BF61
:10D7D00000BF00BF00BF00BF00BF00BF816200BF2D
:10D7E00000BF00BF00BF00BF704700000004005032
:10D7F00000B5FFF7E1FFFFF7DFFFFFF7DDFFFFF702
:10D80000DBFFFFF7D9FFFFF7D7FFFFF7D5FFFFF7E4
:10D81000D3FFFFF7D1FFFFF7CFFFFFF7CDFFFFF7F4
:10D82000CBFFFFF7C9FFFFF7C7FFFFF7C5FFFFF704
:10D83000C3FFFFF7C1FFFFF7BFFFFFF7BDFFFFF714
:10D84000BBFFFFF7B9FFFFF7B7FFFFF7B5FFFFF724
:10D85000B3FF00BDF8B5044600680025C16849065D
:10D8600019D4C16880221143C160FBF71FFA274613
:10D870000646203709E0FBF719FA811B7D20C0001E
:10D88000814202D90420787001252068C0684006D2
:10D8900001D4002DEFD02846F8BD70B504460068CD
:10D8A0000025C16880229143C1602068806880069D
:10D8B00008D42046FCF79CF8002803D0042020342C
:10D8C00060700125284670BD70B5054600F0F7F977
:10D8D0000024E443002819D1284600F027F800224C
:10D8E000C721284600F07AF90028284602D000F027
:10D8F0000FF80BE000F00CF8284600F0D1F90028F2
:10D9000004D1284600F078F9002800D0204670BDE8
:10D9100028214843044910B5401801894068012274
:10D92000FBF7BDF910BD0000E02600202821484388
:10D93000044910B54018018940680022FBF7AFF98F
:10D9400010BD0000E0260020FFB581B00C46019814
:10D9500028214843174900254018406A1F461646AB
:10D96000A0420DD9002E0BD0A119814208D8B900D0
:10D97000114A00915158491E214201D1032F03D36E
:10D980000020C04305B0F0BD002C0ED1B0420CD831
:10D990000198FFF799FF0AE061193A46019800F0F3
:10D9A000D5F80549009808584519B542F4D3002028
:10D9B000E8E70000E02600202420010838B50446EE
:10D9C0000322694600F09EF80025ED43002812D19D
:10D9D00068460078FF2810D168464078FF280CD1AF
:10D9E00068468078FF2808D103226946204600F067
:10D9F00089F8002801D0284638BD6846827828205A
:10DA000044430A48012189052018152A05D0162A01
:10DA100003D0172A04D0182A05D04162002038BD4F
:10DA20000121C905F9E701210906F6E7E0260020F2
:10DA3000FFB50E46C8B2FF2181B0013100250C1A96
:10DA40000A9F9C4200D91C46019800F0D5F8002896
:10DA500042D1019800F033F900283DD10198FFF739
:10DA600065FF00220221019800F0B8F800281FD1BC
:10DA70003002010E0022019800F0B0F8002817D102
:10DA80003004010E0022019800F0A8F800280FD100
:10DA9000F1B20022019800F0A1F8002808D10CE0B2
:10DAA00003980022415D019800F098F8002803D007
:10DAB0000198FFF72DFF0FE06D1CA542F0D30198F0
:10DAC000FFF726FF019800F0EBF8002804D1019839
:10DAD00000F092F8002803D00020C04305B0F0BD4C
:10DAE000002F00D03C600020F8E7000010B528248B
:10DAF0006043034CC900001940184260038110BD07
:10DB0000E0260020F8B515460E4607460024FFF72C
:10DB10000DFF00229F21384600F060F8002807D151
:10DB20000DE03219FF21384600F058F8002805D0E2
:10DB30003846FFF7EDFE0020C043F8BD641CAC4240
:10DB4000EFD33846FFF7E4FE0020F8BDF8B50646EF
:10DB500015469000204A1058401E81430C4630461E
:10DB600000F0ADF80027FF43002833D13046FFF71F
:10DB7000DDFE19480022001F415D304600F02EF8FE
:10DB8000002816D12002010E0022304600F026F8AF
:10DB900000280ED12004010E0022304600F01EF8AD
:10DBA000002806D1E1B20022304600F017F8002824
:10DBB00003D03046FFF7ACFE0CE03046FFF7A8FE7E
:10DBC000304600F06DF8002804D1304600F014F81B
:10DBD000002800D03846F8BD2420010807B51146BA
:10DBE00028225043034A0123105C01AA00F0A6F842
:10DBF0000EBD0000E0260020F8B50546002069466D
:10DC000008706E462846FFF791FE0022052128463F
:10DC1000FFF7E4FF040005D13246FF212846FFF755
:10DC2000DDFF04462846FFF773FE200003D1694656
:10DC30000978C907E5D1F8BDFFB583B00020019090
:10DC40000D46039828214843144900274018406A8C
:10DC5000FF431C461646A84214D9002E12D0002CB1
:10DC600010D0411E2940401AA04201D2044610E0C3
:10DC700001A800902346324629460398FFF7D8FEB4
:10DC8000002802D0384607B0F0BD01982D1836188C
:10DC9000241A002CECD10020F5E70000E02600203B
:10DCA00070B50546FFF742FE002204212846FFF723
:10DCB00095FF04462846FFF72BFE204670BD70B541
:10DCC0000546FFF733FE002206212846FFF786FFB0
:10DCD00004462846FFF71CFE204670BDF8B50446F2
:10DCE00015480E46154613490068F7F701FA7D21DD
:10DCF000C900484300906068C11FFD390ED133460A
:10DD0000002280212046009500F038F800280FD02E
:10DD1000606D2021084360650320F8BD009800284D
:10DD200006D0401E009020688068C0430006F5D5EC
:10DD30000020F8BD00366E01A400002038B514465E
:10DD400000291A460CD064256A430092064A8000D6
:10DD500010580A469BB22146FBF7C8FF002038BD89
:10DD6000214600F067F838BD9C010020024A80007F
:10DD700011500020704700009C010020FFB581B0C9
:10DD80001E4604460A9DFAF791FF401B351AFAF722
:10DD90008DFF0746264800684001000D684339E0C2
:10DDA000701C38D0FAF782FFC01BA84205D2002DA4
:10DDB00003D0009800282BD02BE020684168E02297
:10DDC000914341606068C11FFD390CD10121A068F9
:10DDD000C903884202D04911884204D120680168F1
:10DDE0004022914301600120A16A4003814207D192
:10DDF00021680A6882430A6021680A6802430A604F
:10DE000001204034607400202074032005B0F0BD70
:10DE10000025401E0090206881680298884305D044
:10DE2000002103988142BBD10020EFE70121F8E7F0
:10DE3000A400002010B56423534394B2034A800029
:10DE400010582246FBF7A2FE002010BD9C010020C6
:10DE500070470000F8B5044600206A4610801A4D4D
:10DE600055222A70AA226A700322AA70661DEE70DB
:10DE70002A716971154A49008918AC712246E81D5A
:10DE8000F7F7A1F9002007E029186A468978128877
:10DE900089186A461180401CB042F5DB611DA81C40
:10DEA000F9F710FB01466846018029190078C8710E
:10DEB0006846407808727D232246DB000932024919
:10DEC0000348FCF7F0FCF8BDA43A002078370020A6
:10DED000A8060020F8B516460F4604461D46012246
:10DEE00040210A48FAF7DBFEFFF75EFB2046FFF70A
:10DEF00067FB3846FFF764FB3046FFF761FB2846B7
:10DF0000FFF75EFBFFF750FBF8BD00000004005078
:10DF100010B5002240210248FAF7C1FE10BD0000F2
:10DF20000004005010B5022813D0FDF7F9FF0028B7
:10DF30000DD0FDF7F5FF0B24E4010019006900285E
:10DF400005D0FDF7EDFF0019016904A08847002006
:10DF500010BD4868FFF7A0F8F9E700004552524F9E
:10DF6000520D0A000020704710B50220FFF780F81C
:10DF7000FDF7D6FF00280DD0FDF7D2FF0B24E401FA
:10DF800000190069002805D0FDF7CAFF00190169D2
:10DF900001A08847002010BD4F4B0D0A0000000073
:10DFA00070B50B24E4010D4602280FD0FDF7B8FF31
:10DFB00000280BD0FDF7B4FF00190069002805D038
:10DFC000FDF7AEFF001901692AA088476868F7F7D6
:10DFD00082F9002815D0012826D0022836D0FDF776
:10DFE0009FFF00280BD0FDF79BFF00190069002858
:10DFF00005D0FDF795FF001901691FA08847002093
:10E0000070BD0020F9F75CFBFDF78AFF0028F6D011
:10E01000FDF786FF001900690028F0D0FDF780FFAA
:10E020000019016916A0E9E7FDF77AFF00280BD077
:10E03000FDF776FF00190069002805D0FDF770FF95
:10E04000001901690EA08847012010E0FDF768FF64
:10E0500000280BD0FDF764FF00190069002805D0E7
:10E06000FDF75EFF0019016905A088470220F9F756
:10E0700027FBC4E7417267204552524F520D0A00F8
:10E080004F4B0D0A0000000070B54868F7F723F900
:10E090007D210446C900F7F72BF8050364212046CB
:10E0A000F7F726F80A21F7F723F808022D180A21B6
:10E0B0002046F7F71DF80C460A21F7F719F8080172
:10E0C000281800190D4980B288800D49086003F0B6
:10E0D0003FFDFDF725FF00280DD0FDF721FF0B24A4
:10E0E000E40100190069002805D0FDF719FF0019A7
:10E0F000016904A08847002070BD00007837002027
:10E100007C0000204F4B0D0A0000000010B50228D3
:10E1100014DAFDF705FF00280DD0FDF701FF0B24F1
:10E12000E40100190069002805D0FDF7F9FE001987
:10E13000016903A088470020C04310BD002010BD26
:10E1400064656275675F6F666620666C61670D0A5D
:10E150000000000010B5022814DAFDF7E1FE0028E7
:10E160000DD0FDF7DDFE0B24E40100190069002845
:10E1700005D0FDF7D5FE0019016903A088470020EE
:10E18000C04310BD002010BD64656275675F6F6E8F
:10E1900020666C61670D0A0070B50B25ED010C4619
:10E1A00002280FD0FDF7BCFE00280BD0FDF7B8FE0B
:10E1B00040190069002805D0FDF7B2FE4019016939
:10E1C00011A088476068F7F786F8044600021149F5
:10E1D000000C48828C8203F0BBFC2146022002F036
:10E1E0004DFBFDF79DFE00280BD0FDF799FE401971
:10E1F0000069002805D0FDF793FE4019016906A0CB
:10E200008847002070BD0000417267204552524F80
:10E21000520D0A00B83700204F4B0D0A00000000D5
:10E2200070B5FDF77DFE0B24E40100280CD0FDF74E
:10E2300077FE00190069002806D0FDF771FE00196D
:10E24000026920A122A09047FDF76AFE00280FD0A6
:10E25000FDF766FE00190069002809D0FEF7E0FE10
:10E260000546FDF75DFE0019026929461EA090478C
:10E27000FDF756FE00280FD0FDF752FE0019006989
:10E28000002809D0FEF7C8FE0546FDF749FE001933
:10E29000026929461AA09047FDF742FE00280FD0D8
:10E2A000FDF73EFE00190069002809D0FEF7BCFE0C
:10E2B0000546FDF735FE00190269294616A090476C
:10E2C000002070BD563230323130353130303000C0
:10E2D00056657273696F6E3A20202020202020201E
:10E2E0002025730D0A000000494D45493A202020A1
:10E2F00020202020202020202025730D0A0000004F
:10E30000434349443A202020202020202020202060
:10E310002025730D0A000000494D53493A20202062
:10E3200020202020202020202025730D0A0000001E
:10E3300010B527210248FDF769FD002010BD00003F
:10E340003020010810B50B24E401022812D0FDF79B
:10E35000E7FD00280BD0FDF7E3FD00190069002858
:10E3600005D0FDF7DDFD001901690BA088470020ED
:10E37000C04310BDFDF7D4FD00280BD0FDF7D0FD44
:10E3800000190069002805D0FDF7CAFD00190169D0
:10E3900006A08847002010BD75736167653A206C40
:10E3A0006F6720737472696E670D0A004F4B0D0A18
:10E3B0000000000010B5FDF7B3FD00280DD0FDF7FB
:10E3C000AFFD0B24E40100190069002805D0FDF71A
:10E3D000A7FD0019016902A08847002010BD0000B8
:10E3E0004F4B0D0A0000000010B5032814D0FDF7B4
:10E3F00097FD00280DD0FDF793FD0B24E4010019D3
:10E400000069002805D0FDF78BFD0019016903A004
:10E4100088470020C04310BD002010BD75736167A0
:10E42000653A206C6F675F7072696E742061736308
:10E430005B302D315D20636E740D0A000020704743
:10E440007047000010B50220FEF71CFEFDF768FDC6
:10E4500000280DD0FDF764FD0B24E40100190069CC
:10E46000002805D0FDF75CFD0019016901A088476F
:10E47000002010BD4F4B0D0A0000000010B5002019
:10E48000FEF7F6FDFDF74CFD00280DD0FDF748FD29
:10E490000B24E40100190069002805D0FDF740FDB8
:10E4A0000019016901A08847002010BD4F4B0D0ADB
:10E4B0000000000010B50020FEF7E4FDFDF730FD80
:10E4C00000280DD0FDF72CFD0B24E4010019006994
:10E4D000002805D0FDF724FD0019016901A0884737
:10E4E000002010BD4F4B0D0A0000000010B50B249A
:10E4F000E401022812D0FDF713FD00280BD0FDF730
:10E500000FFD00190069002805D0FDF709FD00196D
:10E5100001690BA088470020C04310BDFDF700FD36
:10E5200000280BD0FDF7FCFC00190069002805D07D
:10E53000FDF7F6FC0019016908A08847002010BD0E
:10E5400075736167653A207274635F7365745F61A8
:10E550006C61726D207365630D0A00004F4B0D0AEC
:10E56000000000000020704710B5072814D0FDF708
:10E57000D7FC00280DD0FDF7D3FC0B24E4010019D3
:10E580000069002805D0FDF7CBFC0019016903A044
:10E5900088470020C04310BD002010BD757361671F
:10E5A000653A207274635F73657420797979792094
:10E5B0006D6D206464206868206D6D2073730D0A92
:10E5C0000000000010B5FAF763FD002010BD000048
:10E5D00070B50B24E4010E4603280FD0FDF7A0FC14
:10E5E00000280BD0FDF79CFC00190069002805D01D
:10E5F000FDF796FC0019016920A088477068F6F7BE
:10E600006AFE0546B068F6F766FE0146681E1328E6
:10E6100021D832291FDC002D1DDD1B4E7D203586C3
:10E62000C000F6F77BFD31464039C88003F090FA10
:10E63000FDF776FC00280BD0FDF772FC001900698D
:10E64000002805D0FDF76CFC001901690FA0884770
:10E65000012030840FE0FDF763FC00280BD0FDF7AC
:10E660005FFC00190069002805D0FDF759FC00196E
:10E67000016902A08847002070BD00004172672038
:10E680004552524F520D0A00B83700204F4B0D0A29
:10E690000000000070B50B24E4010D4602280FD0E5
:10E6A000FDF73EFC00280BD0FDF73AFC001900698D
:10E6B000002805D0FDF734FC001901690DA088473A
:10E6C0006868F6F708FE0E49488303F041FAFDF743
:10E6D00027FC00280BD0FDF723FC00190069002857
:10E6E00005D0FDF71DFC0019016906A08847002030
:10E6F00070BD0000417267204552524F520D0A0012
:10E70000B83700204F4B0D0A0000000010B50B2455
:10E71000E401062812DAFDF703FC00280BD0FDF710
:10E72000FFFB00190069002805D0FDF7F9FB00196F
:10E7300001690EA088470020C04310BD03F008FA0D
:10E74000FDF7EEFB00280BD0FDF7EAFB001900698E
:10E75000002805D0FDF7E4FB0019016905A08847F2
:10E76000064801210184002010BD00004552524F8F
:10E77000520D0A004F4B0D0A00000000B837002070
:10E7800010B50B24E401052812DAFDF7C9FB0028B7
:10E790000BD0FDF7C5FB00190069002805D0FDF777
:10E7A000BFFB001901690EA088470020C04310BDBF
:10E7B00003F0CEF9FDF7B4FB00280BD0FDF7B0FB5A
:10E7C00000190069002805D0FDF7AAFB00190169AE
:10E7D00005A08847064801210184002010BD0000E3
:10E7E0004552524F520D0A004F4B0D0A00000000D7
:10E7F000B8370020F8B50B26F6010D46022812DACC
:10E80000FDF78EFB00280BD0FDF78AFB801900690D
:10E81000002805D0FDF784FB8019016914A0884702
:10E820000020C043F8BD69466868FDF753FD68687D
:10E83000FDF7DCFE104CE18A884203D06868FDF7E2
:10E84000D5FEE08203F084F9FDF76AFB00280BD0C7
:10E85000FDF766FB80190069002805D0FDF760FB15
:10E860008019016905A08847012020840020F8BD97
:10E870004552524F520D0A00B83700204F4B0D0A37
:10E8800000000000F8B50B26F6010D46032812DA49
:10E89000FDF746FB00280BD0FDF742FB801900690D
:10E8A000002805D0FDF73CFB8019016923A08847AB
:10E8B0000020C043F8BD69466868FDF70BFD214C98
:10E8C00068460078618E88420ED169464978A28EEA
:10E8D000914209D169468978E28E914204D1694614
:10E8E000C978228F914209D0608668464078A08618
:10E8F00068468078E0866846C0782087A868FDF77B
:10E9000075FE618F884203D0A868FDF76FFE6087AF
:10E9100003F01EF9FDF704FB00280BD0FDF700FB08
:10E9200080190069002805D0FDF7FAFA80190169FD
:10E9300005A08847012020840020F8BD4552524F91
:10E94000520D0A00B83700204F4B0D0A000000009E
:10E95000F8B50B26F6010D46032812DAFDF7E0FAAA
:10E9600000280BD0FDF7DCFA80190069002805D0DB
:10E97000FDF7D6FA8019016923A088470020C0431B
:10E98000F8BD69466868FDF7A5FC214C684600782B
:10E99000E18C88420ED169464978228D914209D195
:10E9A00069468978628D914204D16946C978A28D01
:10E9B000914209D0E0846846407820856846807896
:10E9C00060856846C078A085A868FDF70FFEE18DD8
:10E9D000884203D0A868FDF709FEE08503F0B8F887
:10E9E000FDF79EFA00280BD0FDF79AFA801900690E
:10E9F000002805D0FDF794FA8019016905A0884721
:10EA0000012020840020F8BD4552524F520D0A00CB
:10EA1000B83700204F4B0D0A00000000F8B50B2658
:10EA2000F6010D46022812DAFDF77AFA00280BD01B
:10EA3000FDF776FA80190069002805D0FDF770FA15
:10EA40008019016914A088470020C043F8BD6946B9
:10EA50006868FDF73FFC6868FDF7C8FD104C218B26
:10EA6000884203D06868FDF7C1FD208303F070F889
:10EA7000FDF756FA00280BD0FDF752FA801900690D
:10EA8000002805D0FDF74CFA8019016905A08847D8
:10EA9000012020840020F8BD4552524F520D0A003B
:10EAA000B83700204F4B0D0A0000000070B54868D1
:10EAB000F6F711FC0C4CE08703F04AF8FDF730FA4A
:10EAC00000280DD0FDF72CFA0B25ED014019006947
:10EAD000002805D0FDF724FA4019016903A08847F2
:10EAE00001202084002070BDB83700204F4B0D0A54
:10EAF0000000000070B54868F6F7EDFB0C4C20866E
:10EB000003F026F8FDF70CFA00280DD0FDF708FAFF
:10EB10000B25ED0140190069002805D0FDF700FA2A
:10EB20004019016903A0884701202084002070BD9E
:10EB3000B83700204F4B0D0A00000000002070473E
:10EB400010B502A0FCF702FA10BD00004576656E14
:10EB5000743A25750D0A000070B50B24E4010D46CA
:10EB600002280FD0FDF7DCF900280BD0FDF7D8F90B
:10EB700000190069002805D0FDF7D2F900190169D4
:10EB800015A088476868F6F7A6FB00F085F900280D
:10EB900011D0FDF7C5F900280BD0FDF7C1F9001918
:10EBA0000069002805D0FDF7BBF9001901690BA029
:10EBB0008847002070BDFDF7B3F90028F9D0FDF7B4
:10EBC000AFF9001900690028F3D0FDF7A9F9001981
:10EBD000016904A0ECE70000417267204552524FE2
:10EBE000520D0A004F4B0D0A00000000F8B50B242F
:10EBF000E4010D4604280FD0FDF792F900280BD050
:10EC0000FDF78EF900190069002805D0FDF788F995
:10EC10000019016919A088476868F6F75CFB074688
:10EC2000AE68E868F6F757FB82B23146384600F026
:10EC30006DF9002811D0FDF773F900280BD0FDF70E
:10EC40006FF900190069002805D0FDF769F900196E
:10EC500001690BA088470020F8BDFDF761F9002885
:10EC6000F9D0FDF75DF9001900690028F3D0FDF730
:10EC700057F90019016904A0ECE700004172672010
:10EC80004552524F520D0A004F4B0D0A0000000032
:10EC900038B50020034600901D4A0121684600F067
:10ECA00055F90B24E401002811D0FDF739F90028AB
:10ECB0000BD0FDF735F900190069002805D0FDF7E4
:10ECC0002FF90019016913A08847002038BDFDF70E
:10ECD00027F900280CD0FDF723F900190069002856
:10ECE00006D0FDF71DF9001902690CA000999047A4
:10ECF000FDF716F90028E8D0FDF712F900190069B0
:10ED00000028E2D0FDF70CF90019016906A0DBE745
:10ED100041EB00084552524F520D0A00536F636B8E
:10ED200049443A25750D0A004F4B0D0A00000000BA
:10ED300070B50B24E4010D4603280FD0FDF7F0F861
:10ED400000280BD0FDF7ECF800190069002805D069
:10ED5000FDF7E6F80019016919A088476868F6F719
:10ED6000BAFAAD6806462846F6F77BFA0246294607
:10ED7000304600F0C9FA002811D0FDF7D1F800287C
:10ED80000BD0FDF7CDF800190069002805D0FDF77C
:10ED9000C7F8001901690BA08847002070BDFDF776
:10EDA000BFF80028F9D0FDF7BBF80019006900286A
:10EDB000F3D0FDF7B5F80019016904A0ECE70000F5
:10EDC000417267204552524F520D0A004F4B0D0AB7
:10EDD00000000000002070470020704738B514483C
:10EDE00069460880FDF79CF800280DD0FDF798F8DB
:10EDF0000B24E40100190069002805D0FDF790F804
:10EE0000001901690BA08847112400232403022262
:10EE100021461846FEF798FD02236A462146002047
:10EE2000FEF70AFF064801210184002038BD0000DA
:10EE3000AAAA0000757064617465204F4B0D0A002A
:10EE4000B837002070B51048104C408F218900253C
:10EE500088420AD20E480078002806D001214902D3
:10EE60000C48F9F717FF002801D065700AE001206F
:10EE7000607002F0B7FD6078002803D0E089401C84
:10EE8000E08170BDE58170BD783700200000002072
:10EE9000DC0100200004005009490A4A4143891856
:10EEA00003280AD2002908D00878002803D00128B6
:10EEB00001D005200870002070470020C043704733
:10EEC0004C05000038110020F8B500240D4D2646F1
:10EED00001270D48604340190178032903D0042914
:10EEE00001D0062908D1867007708368002B03D0F3
:10EEF000C268022120469847641C032CE9DB0020ED
:10EF0000F8BD0000381100204C05000070B5154612
:10EF10000B4A0C4B4243D41803280DD2002C0BD0C3
:10EF20000B46204608A22A211030FDF710FB65870A
:10EF300003202070002070BD0020C04370BD000081
:10EF40004C0500003811002025730000FFB51F4854
:10EF500081B01F460E4600251D4969430C1802D09A
:10EF60002178002906D06D1C032DF5DB0020C0435D
:10EF700005B0F0BD16492046FDF76CF96560667076
:10EF8000022020700398E7601023A0605F012146F3
:10EF900020463A46C4313C30FDF7D4FBB120800016
:10EFA000012E0AD02118204610233A466C30FDF776
:10EFB000C9FB019805600020DAE7211820460123EB
:10EFC0003A46B030FBF7C5FEF3E7000038110020E9
:10EFD0004C0500000649074A41438918032804D21A
:10EFE000002902D00020087070470020C0437047FD
:10EFF0004C050000381100200549064A4143891894
:10F00000032801D300207047014880380818704752
:10F010004C050000381100200649074A4143891871
:10F02000032802D3FF202D3070470920C0010818A3
:10F03000806C70474C05000038110020032805DA69
:10F0400003494843034940181030704702A07047F5
:10F050004C0500003811002000000000032805DAEC
:10F060000349484303494018408F704700207047C8
:10F070004C05000038110020032805DA03494843F5
:10F08000034940183C307047002070474C05000091
:10F0900038110020032804DA034948430349085C77
:10F0A00070470020704700004C0500003811002018
:10F0B000032805DA0349484303494018407870475C
:10F0C000002070474C050000381100200C490D4A03
:10F0D00041438918002210B5D24303280ED20029DB
:10F0E0000CD00B78042B09D001220A708B68002BFE
:10F0F00002D0CA6802219847002010BD104610BDFA
:10F100004C050000381100200A490B4A414310B554
:10F11000891803280BD2002909D007220A708B68AE
:10F12000002B02D0CA6800219847002010BD0020A3
:10F13000C04310BD4C0500003811002070B50546D5
:10F140001A481B4968434418032D25D2002C23D0AC
:10F150000620207010235E01214620463246C4312D
:10F160003C30FDF7EFFA1149114BB1206943627849
:10F170008000C9180918012A11D0204610233246F0
:10F180006C30FDF7DFFAA368002B03D0012128467D
:10F19000E2689847002070BD0020C04370BD204643
:10F1A00001233246B030FBF7D4FDECE74C050000FC
:10F1B0003811002009490A4A414310B5891803282B
:10F1C00009D2002907D08B68002B02D0CA6803211E
:10F1D0009847002010BD0020C04310BD4C05000022
:10F1E00038110020FFB5014617461F481F4A00246A
:10F1F0004843E443801881B01E4603291AD20028F0
:10F2000018D0002E16D04178012916D06C3000900D
:10F21000FDF74CFA05000DD06A68BA4206D229689B
:10F220000298F5F7D0FF68680024306029460098FE
:10F23000FDF710FA204605B0F0BD0024B030254699
:10F2400000900BE0029801190098FBF7A7FD002839
:10F2500002D000203560EEE7641C6D1CBC42F1D387
:10F2600000243560E6E700004C050000381100205E
:10F27000F7B505461A481B49684300244018671E25
:10F280001646032D1FD200281DD04178012910D029
:10F290006C3007461146FDF727FA040019D03246B4
:10F2A00020680199F5F78FFF38462146FDF7E8F908
:10F2B00013E00546B03509E0019801192846FBF72F
:10F2C0002DFD002801D03846FEBD641CB442F3D3A6
:10F2D00003E0294604A0FBF739FE0020FEBD000034
:10F2E0004C05000038110020536F636B65745B257B
:10F2F000755D2052656376204275666665722046AC
:10F30000756C6C0D0A000000F7B5054613481449EA
:10F31000684300274018FF4382B01646032D16D2DB
:10F32000002814D0002E12D03C3011460090FDF77A
:10F33000DBF904000DD0324620680399F5F743FF4E
:10F3400021460098FDF79CF9002005B0F0BD384635
:10F35000FBE7294603A0FBF7F9FDF8E74C050000A1
:10F3600038110020736F636B65745B25645D2073D7
:10F37000656E64206275662066756C6C0D0A00000F
:10F38000032805DA044A5043044A11540020704708
:10F390000020C043704700004C05000038110020D9
:10F3A0000649074A41438918032801D300207047C2
:10F3B0001320800108180079704700004C050000F8
:10F3C0003811002010B5FCF7C5FEF9F7B3FC10BDED
:10F3D00010B59AB034216846F5F70EFF142115A830
:10F3E000F5F70AFF20210DA8F5F706FF244801686C
:10F3F0000324E402A143C21489180160F9F756FE00
:10F4000020480169A14301610E200090FF200130D6
:10F4100002901020049002200990400401210B90DA
:10F420000001059100240C9003910A946846FAF7B4
:10F430005FF8002801D072B6FEE70F201590032078
:10F440001690179418940121199415A8F9F726FF1E
:10F45000002801D072B6FEE7A7200D9001204004DD
:10F460000E9003200F9480041490109411940DA812
:10F47000F9F756FE002801D072B6FEE71AB010BDAB
:10F480000070004040100240024901488860704707
:10F490000050000800ED00E0F0B502680124A40768
:10F4A000144D154E154FA04205D0A84203D0B042CE
:10F4B00001D0B84204D11346702293434A681A43DC
:10F4C000A04205D0A84203D0B04201D0B84204D136
:10F4D00003231B029A43CB681A4380239A430B6988
:10F4E0001A4302608A68C26209688162012141612F
:10F4F000F0BD00000004004000080140001401407D
:10F5000030B5026A520852000262026A4568836995
:10F510007024A3439C080B68A40023430224A24345
:10F520008C6845601443836149684163046230BD5F
:10F5300030B5026A10239A430262036A4568826901
:10F5400073242402A2430C68240214432022934310
:10F550008A68456012011A438461496881630262C6
:10F5600030BD30B5026AFF2301339A430262026A5A
:10F570004568C3697024A3439C080B68A400234317
:10F5800001246402A2438C68456024021443C361D1
:10F590004968C163046230BD30B5026A01231B03B0
:10F5A0009A430262036A4568C26973242402A24333
:10F5B0000C68240214430122520393438A68456075
:10F5C00012031A43C46149680164026230BD10B578
:10F5D000818CC90707D001684A6801235B049A43FC
:10F5E000836A1A434A60818C890707D501684A6893
:10F5F00001231B049A43C36A1A434A60818C49075A
:10F6000007D501684A6801239B049A43036B1A4398
:10F610004A60818C090707D501684A680123DB032A
:10F620009A43436B1A434A60818CC90607D5026826
:10F63000916801231B039943836B19439160818C6B
:10F64000890607D501688A6801235B039A43C36B67
:10F650001A438A60818C490612D503685A680121D1
:10F660000905046C8A4322435A60026C8A4207D11E
:10F670000268516803235B059943436C1943516049
:10F68000818C090607D501684A680123DB04806C78
:10F690009A4302434A6010BDFEB5074600258037F5
:10F6A00004467D60F9F702FB019020680068264659
:10F6B00000076036002819DA27480090012100224F
:10F6C00049052046019B00F03BFC00280ED0EFF3DB
:10F6D0001080012181F3108821680A6880239A43F1
:10F6E0000A6080F310882020E06729E02068006825
:10F6F000400728D51848009001210022890520469E
:10F70000019B00F01DFC00281DD0EFF310800121AB
:10F7100081F3108821680A68FF2321339A430A6025
:10F7200080F31088EFF31080012181F310882168A5
:10F730008A68520852008A6080F31088202038605E
:10F7400035760320FEBD2020E067386025666566BB
:10F7500035760020FEBD0000FFFFFF0110B5806A76
:10F760000022014640314A834A82FAF72AFD10BD41
:10F77000F8B5846AE06F254680352E68216889686F
:10F7800000270906002906DA212804D15220075350
:10F79000204600F0CCF820688068400606D5222E6E
:10F7A00004D15A200753204600F091F868681021D0
:10F7B000084368602046FAF704FDF8BD70B50146BD
:10F7C0000968806A096800228906002938DB5A2105
:10F7D0000A52EFF31081012383F3108803681C6839
:10F7E000FF250135AC431C6081F31088EFF31081D5
:10F7F000012383F3108803689C68640864009C609C
:10F8000081F31088EFF31081012383F310880368DC
:10F810009C684025AC439C6081F3108820238021A4
:10F820000B50016E01290BD1EFF31081012383F3FB
:10F83000108803681C681025AC431C6081F3108895
:10F840004266016E012902D0FBF728F870BD5821ED
:10F85000095AFAF793FC70BD10B5806A0121416620
:10F86000016E012902D0FBF71DF810BD5821095A7D
:10F870004908FAF783FC10BD10B501460968806A93
:10F88000096889061BD4002252210A52EFF3108125
:10F89000012282F31088026893688024A343936056
:10F8A00081F31088EFF31081012282F31088006841
:10F8B000026840231A43026081F3108810BDFBF7F1
:10F8C000E5F810BD10B5806AFBF7E4F810BD10B57F
:10F8D000EFF31081012282F3108802681368FF247D
:10F8E0002134A343136081F31088EFF310810122C8
:10F8F00082F31088026893685B085B00936081F371
:10F900001088016E01290BD1EFF31081012282F3DF
:10F910001088026813681024A343136081F31088D1
:10F92000202280210A5000210166816610BD10B599
:10F93000EFF31081012282F3108802681368C0245B
:10F94000A343136081F310882021C16710BD00001C
:10F9500070B501464031034680338C8B1D680268C8
:10F96000222D04D0906908210843906170BD526A2D
:10F97000456D22402A80426D921C42654A8B521E80
:10F980004A834A8B002AF1D1EFF31082012484F3D9
:10F99000108804682568FF262136B543256082F368
:10F9A0001088EFF31082012484F310880468A5689E
:10F9B0006D086D00A56082F3108820221A60002374
:10F9C00083664366174A046894420ED06268120246
:10F9D0000BD5EFF31082012585F3108825680126E9
:10F9E000B606B543256082F31088026E012A02D064
:10F9F000FAF754FF70BD0366EFF31082012383F31F
:10FA000010880468256810239D43256082F31088C0
:10FA10000268D469E443E40600D41362098BFAF760
:10FA2000ADFB70BD0048004070B501464031034653
:10FA300080338C8B1D680268222D04D090690821C8
:10FA40000843906170BD526A2240446D2270426D3D
:10FA5000521C42654A8B521E4A834A8B002AF1D1BE
:10FA6000EFF31082012484F3108804682568FF26D0
:10FA70002136B543256082F31088EFF3108201240C
:10FA800084F310880468A5686D086D00A56082F392
:10FA9000108820221A60002383664366174A046890
:10FAA00094420ED0626812020BD5EFF3108201254A
:10FAB00085F3108825680126B606B543256082F3D4
:10FAC0001088026E012A02D0FAF7E8FE70BD0366C4
:10FAD000EFF31082012383F3108804682568102354
:10FAE0009D43256082F310880268D469E443E406EC
:10FAF00000D41362098BFAF741FB70BD0048004047
:10FB0000F8B50446016880682269E66910436269B5
:10FB1000002532431043754B0A68754E324002434C
:10FB20000A6020684168032212039143E26811438E
:10FB300041602168A069994201D0226A10438A6815
:10FB40000B263602B24302438A606A4922686A4839
:10FB50008A420CD1C0688007800F06D001283FD0B0
:10FB600002283BD0032827D124E0012725E0634960
:10FB70008A420AD1C0680C2108402DD004282FD019
:10FB800008282BD00C2817D114E05D498A4223D0D5
:10FB90005C498A4220D09A420ED1C168032080027B
:10FBA000014019D001208002091A19D0091A15D074
:10FBB000814201D1082700E010274F4952484039BF
:10FBC00086009A4234D1002F0CD0022F0DD0042F82
:10FBD00010D0082F7ED128E00027EEE70227ECE7BF
:10FBE0000427EAE7F9F728FC06E00968C90605D406
:10FBF000304603E0F9F740FC002872D062685100FB
:10FC00005118814266D81103814263D3010E060266
:10FC10005008002330185941F5F794FA03210902DE
:10FC20003A4A411A91425AD954E00120C003E5E70B
:10FC30000122E369D20393422AD13B0001F0BBF8D1
:10FC40000906090C4A114A4A4A264A00F9F7F4FB08
:10FC500009E0F9F701FC06E00968C90605D4304659
:10FC600003E0F9F709FC00283BD0616840004A082E
:10FC70008018F5F73DFA0146254A1039914229D8F6
:10FC8000511C01400007400F084328E01046ECE7F4
:10FC90003B0001F090F80906090C1F111F1F1F21DE
:10FCA0001F00F9F7C9FB09E0F9F7D6FB06E0096880
:10FCB000C90605D4304603E0F9F7DEFB002810D072
:10FCC00061684A081018F5F713FA02461049103A0D
:10FCD0008A4203D9012504E01046F1E780B2216889
:10FCE000C8600020A066E0662846F8BD00480040D5
:10FCF000F369FFEF0038014040100240004400402B
:10FD0000004C00400050004000093D00FFFC0F0087
:10FD1000EFFF000070B504464165403002830020CB
:10FD200025468035686022212960616F002919D03D
:10FD3000204BCB62636F20491963636F1F4959637E
:10FD4000616F13468863666D216832462431606FA7
:10FD5000F8F738FD002805D01020686020202860C2
:10FD6000012070BD206900280CD0EFF31080012124
:10FD700081F3108821680A68FF2301331A430A605F
:10FD800080F31088EFF31080012181F3108822683E
:10FD900093680B43936080F31088EFF3108081F336
:10FDA000108821688A6840231A438A6080F310888B
:10FDB000002070BDBDF7000859F8000871F7000871
:10FDC00070B54165014640310A834A83002383664A
:10FDD000012284681203FF25944204D10469002C97
:10FDE00013D1264C0AE07F26002C09D001252D07CF
:10FDF000AC420CD10469002C05D03F248C8307E071
:10FE00000469002C01D08E8302E08D8300E08B8397
:10FE1000014680314B6022230B60EFF310810123F8
:10FE200083F3108803689C6801252C439C6081F350
:10FE300010888168914202D1016900290ED01049D1
:10FE40008166016900290BD0EFF31081012282F352
:10FE5000108800680268FF23213309E009498166A0
:10FE6000EFF31081012282F31088006802682023DA
:10FE70001A43026081F31088002070BDFF0100006A
:10FE800029FA000851F9000810B5C16F212910D1D5
:10FE9000014640314A8A002A0CD0C26C036812889D
:10FEA000D205D20D9A62C26C921CC264488A401E6E
:10FEB000488210BDEFF31081012282F3108802689E
:10FEC00013688024A343136081F31088EFF310813B
:10FED000012282F310880068026840231A430260FE
:10FEE00081F3108810BD10B5C16F21290ED10146D4
:10FEF00040314A8A002A0AD0C26C036812789A629A
:10FF0000C26C521CC264488A401E488210BDEFF386
:10FF10001081012282F31088026813688024A343B1
:10FF2000136081F31088EFF31081012282F31088AF
:10FF30000068026840231A43026081F3108810BDF4
:10FF4000FFB5064681B080360546044660350A9FF7
:10FF50002EE0781C2CD0F8F7A9FE0499401AB8427C
:10FF600014D8002F12D020680168490720D5C16934
:10FF7000C94309070CD4082707622046FFF7A7FCEE
:10FF8000776000202876012005B0F0BD0320FBE754
:10FF9000C069C04300050BD401202168C00208627B
:10FFA0002046FFF794FC2020706000202876EDE7C3
:10FFB0002068C1690298884305D0002103988142D6
:10FFC000C7D00020E0E70121F8E70000F3B5FFB05B
:10FFD0008CB0F849F8A0FAF7B9FF0722F8A18B987E
:10FFE000F5F76AF9F94D01272C46F74E4034002801
:10FFF0003FD00E22F6A18B98F5F75EF900286CD061
:020000040801F1
:100000000922F7A18B98F5F757F900287ED008222E
:10001000F6A18B98F5F750F9002878D00822F6A1C0
:100020008B98F5F749F9002872D00922F5A18B9831
:10003000F5F742F900286CD00A22F5A18B98F5F764
:100040003BF9002814D00922F4A18B98F5F734F974
:10005000002872D00922F4A18B98F5F72DF9002819
:100060006CD00A22F3A18B98F5F726F900287DD0F1
:100070009EE10C2301AA2C218B98FCF791FA05280C
:1000800075D30298FCF717F9A9888842F0D10025AA
:100090000398FCF7ABFA218E814235D0208632E0FE
:1000A0006946C978A28D91420CD0E08468464078B8
:1000B00020856846807860856846C0780125A085DF
:1000C000002030700598FCF791FAE18D884236D017
:1000D0000598FCF78BFAE08510E10C2301AA2C218E
:1000E0008B98FCF75DFA0528CAD30298FCF7E3F871
:1000F000A9888842BCD100250398FCF777FAE18FE4
:10010000814201D0E0870125694603E01AE03DE025
:100110007AE085E00498FCF7DDF868460078E18C29
:100120008842C2D169464978228D9142BDD1694643
:100130008978628D9142B8D1B2E7A2E0BEE0002D8D
:10014000CAD135E10C2301AA2C218B98FCF728FA9F
:10015000032895D30298FCF7AEF8A988884287D186
:100160000398FCF7A8F8012803D101E0CCE0DBE01C
:10017000B7700398FCF79FF8022800D1F770039836
:10018000FCF799F80328DCD1377111E10C2301AA9F
:100190002C218B98FCF704FA0428A5D30298FCF7CD
:1001A0008AF8A9888842CCD1A5A10498F5F760F80F
:1001B0000028C6DDA54869460880A5A0FAF7C6FE56
:1001C000112400232403022221461846FDF7BCFB1C
:1001D00002236A4621460020FDF72EFD0924002354
:1001E000FF226403013221461846FDF7ADFB039858
:1001F000F5F737F8431C21460020039AFDF71CFD54
:100200000A20F8F713FBD3E00C2301AA2C218B98CA
:10021000FCF7C6F903289CD30298FCF74CF8C7E01A
:100220000C2301AA2C218B98FCF7BAF903287BD365
:100230000298FCF740F8A9888842A6D18AA10398C1
:10024000F5F716F8002803D10498FCF7CFF93081B0
:1002500087A10398F5F70CF8002896D1854904206A
:1002600088610402AB8884A221465248FCF76FF9EA
:1002700002465049F068FFF747F8AB887EA2214656
:1002800016E00FA800900DAB80A28C998B98FCF71C
:100290006BF8022835D10E9A0D99002088540D98DC
:1002A000FCF709F8AB8898422BD1012172A2890290
:1002B0004048FCF74CF902463E4976E00C2301AA7F
:1002C0002C218B98FCF76CF900900298FBF7F3FF58
:1002D0003E49898888426BD10098022824D303982C
:1002E000FCF784F985B20498FCF780F980B2102DF0
:1002F00008D0FF2D02D835496A00885201F028FC49
:10030000278455E0308153E00C2301AA2C218B98DF
:10031000FCF746F904460298FBF7CDFF2B49898884
:10032000884245D1022C04D20020C0437FB00EB0D9
:10033000F0BD0398FCF75AF984B20498FCF756F91B
:1003400087B257A10DA800F0DDFC85B21F4857A168
:1003500082880DA8401900F0D5FC281885B23F19F5
:100360000BE01A486100425A0DA8401950A100F054
:10037000C9FC2818641C85B2A4B2A742F1D8652133
:100380000DA841556D1CA9B26E224254491C89B278
:1003900064224254491C89B20D224254491C89B23C
:1003A0000A224254491C8AB20146F068FEF7ACFFAB
:1003B0000020BBE77833002025730D0A0000000001
:1003C000244750535F532C00BC0100207837002095
:1003D00024434841494348554750535F532C00003C
:1003E00024726563656976652C000000247570646D
:1003F0006174652C00000000246765746C6F672CC5
:100400000000000024636F6E74726F6C2C0000009B
:100410002475736572646174612C000024736574C3
:10042000746F6E652C0000002473657470617261D6
:100430002C0000002472656164706172612C000000
:10044000563230323130353130303000CCCC0000D3
:10045000676F746F204F5441204170706C69636105
:1004600074696F6E0D0A0000626565706572000048
:1004700054545300000C005024526563656976653E
:10048000766F6963652C25580D0A00002473657426
:10049000746F6E652C25702C25700D0A000000000D
:1004A000247265706C79706172612C0025782C0063
:1004B00025642C0030B51A4C89B0207802282BD145
:1004C000FCF7AAFD174B184A1849A5791B78127832
:1004D0000978089505AD0EC5154963794A880390DA
:1004E000D5B2120A01921348029504930078009045
:1004F0008B88012110A289021A48FCF728F80546CA
:10050000A0792A46401CA0711649E068FEF7FCFE5F
:1005100029461448F4F770FE002009B030BD0000F1
:10052000BC01002001000020DB010020940000201D
:100530007837002000000020245854422C25582CE5
:100540002530327525252C25642E25642C25732C09
:1005500025642C312E2C25642C25642C25642C2517
:10056000640000007833002010B50023034A022104
:100570000348FEF7EBFC002010BD00003106010827
:10058000C8010020FEB5FCF73BFA00251C491D4CB4
:10059000012805D011200002086025700020FEBD52
:1005A0001120000408602078002813D00228F5D11B
:1005B000154E21693068401AFF212D318842EDD354
:1005C00012A000F08FFB657030682061FFF772FFAA
:1005D0006571E3E70120114D2070288DAA8D698D8A
:1005E0006B4607C30121EB8C0DA289020F48FBF774
:1005F000AEFFEA8D0D49E068FEF788FCCEE700000B
:100600008C000020BC01002014000020B7A2CBCD3C
:100610003447D0C4CCF8B0FC0D0A0000B837002035
:1006200025752E25752E25752E257500783300200D
:1006300038B5114800240278002914D0012916D0B9
:10064000022912D003290DD100946B460B4A0C49A4
:10065000C068FEF7C7FD002804D10948009944543A
:10066000FFF7B4FC38BD012AFCD1047038BD012A63
:10067000FCD10221017038BDBC010020FF03000045
:100680007833002010B50848017802290BD1074CB7
:1006900007492278C068FEF737FE21780448F4F74E
:1006A000ABFD0020207010BDBC01002081010020A6
:1006B000E025002010B50248F9F788FD10BD0000C4
:1006C000A806002010B50248F9F780FD10BD000013
:1006D0003007002010B50248F9F778FD10BD000082
:1006E000B8070020F8B51D4D0E0034D0042832D2D2
:1006F000742148431A494418A078002802D00128E0
:1007000022D028E0E168A068421860680090406F3D
:10071000006840682769101A0818C01BF4F7E8FC45
:10072000012905D817D100980068C069800612D445
:100730003878307061692069884201D1A06800E092
:10074000401C2061002506E0204618303146FAF7AB
:1007500025FB0028F6D02846F8BD0000FFFFFFFF6C
:10076000A82D0020002901D0042802D30020C04376
:10077000704774225043034A801840680860002084
:1007800070470000A82D002070B50C00064601D06F
:10079000042E02D30020C04370BD74214843214978
:1007A0000E54227845186A706078A8706068A86056
:1007B000A168E9606278002A02D0012A05D00BE026
:1007C00028614018401E686106E028461830012361
:1007D000A2686168FAF7BDFAE068E86220692863F8
:1007E000A0692867606968632078002801D0012823
:1007F00006D121460C310EC928463830FBF7A2FF3E
:100800006078002804D0012806D0022804D006E031
:10081000304600F009F802E0304600F021F80020F0
:1008200070BD0000A82D002038B50C49742250433B
:1008300042185068016804E04C6A6B461C801C88B2
:100840001C80CB691B07F7D491681161D368CC1861
:10085000641E54619AB2F9F7BDFF38BDA82D00207F
:1008600074214843044910B5401801466831406876
:100870000122F9F7E1FF10BDA82D002070B50E464A
:10088000044674200A49604345186868F9F778FC03
:10089000686846606868F9F7EFFD002802D000201C
:1008A000C04370BD204600F005F8002070BD000078
:1008B000A82D002070B5054674201A4968434418D5
:1008C000A078002802D0012807D00DE0A0682061A0
:1008D000E1684018401E606106E0204618300123A0
:1008E000E268A168FAF735FA6078002801D001289B
:1008F00006D121462C310EC920463830FBF722FFA5
:10090000A078002804D0012806D0022804D006E0F0
:100910002846FFF789FF02E02846FFF7A1FF0020E5
:1009200070BD0000A82D002070B50D0001D0042876
:1009300002D30020C04370BD7421484304494418C9
:1009400074212046FBF786FC0020656070BD000026
:10095000A82D002010B502460E4900207423434301
:100960005B185B6893420FD1742242435118897817
:10097000002906D0012901D0022901D1FFF770FF1B
:1009800010BDFFF751FF10BD401CC0B20428E5D3D5
:1009900010BD0000A82D002038B5014613480024E2
:1009A00074226243121852688A4219D17421614339
:1009B0000818817801290BD0022908D1016F00297C
:1009C00002D0806EC0B288472046FFF749FF38BD8D
:1009D000816E6A46117069461830FAF79FF9F3E79D
:1009E000641CE4B2042CDBD338BD0000A82D002029
:1009F000F7B582B00021009103991546002903D074
:100A0000002D01D0042803D30020C04305B0F0BD61
:100A1000742148432B4946187078344638340028EE
:100A200004D0012820D0022842D049E0FBF7B8F9D1
:100A300020462946FBF758FE070033D020463946AA
:100A4000FBF71EFE2A4638680399F4F7BCFB2046E4
:100A5000FBF72CFE0446FBF791FBA088216882B2CD
:100A60007068F9F781FF2BE0FBF79AF920462946D9
:100A7000FBF73AFE070015D020463946FBF700FE8B
:100A80002A4638680399F4F79EFB2046FBF70EFED2
:100A90000446FBF773FBA088216882B27068F9F7FF
:100AA000B9FF0DE0FBF76AFB0020C043009007E0B0
:100AB000134664204343AAB270680399F9F7F3FE22
:100AC0000098A3E7A82D002070B51F4A00217423C9
:100AD0004B439B185B68834231D1742041438C188F
:100AE0006078002816D0012813D1204638300546FA
:100AF000FBF7DCFD01462846FBF7ACFD2846FBF77B
:100B0000D5FD002805D081888AB201686068F9F7B0
:100B100081FF70BD204638300546FBF7C7FD014612
:100B20002846FBF797FD2846FBF7C0FD0028F0D0CC
:100B300081888AB201686068F9F716FF70BD491CA8
:100B4000C9B20429C3D370BDA82D0020F8B5002573
:100B5000184C194F64280CD0622826D0602807D181
:100B6000258400F0F5FF6420F6F7DEFD1348C7602A
:100B7000F8BD13486946088072B680211148F6F71F
:100B80004FFE064607E080210E48F6F749FE06466E
:100B9000C820F6F7C9FD002EF5D0022269460948A3
:100BA000F6F7E8FE62B6A584DBE7024865844038C4
:100BB0000580D6E7B83700200400FA0500ED00E014
:100BC000CCCC0000384A0008F8B5414C002321780D
:100BD000404A1D46082910D007294ED0062957D073
:100BE000052959D004295AD003295BD000295DD0AA
:100BF00001295FD0022961D062E0A17800264A1F56
:100C000004E0344FBF5DFB189BB2761C9642F8DBC4
:100C1000627927799B185B18E1785E186378F6187B
:100C2000F6198019C00723D0012A1DD0022A1FD12E
:100C300028480078012802D10846FFF787FF264898
:100C4000E178627840182349F4F7BDFA00F080FF9C
:100C50006420F6F769FDBFF34F8F21491F48C86034
:100C6000BFF34F8F00BFFDE749081846FDF7F2F8C4
:100C70002570E570A570A571F8BDA1795054491C87
:100C8000C8B2A071A178491F8842F5D1082001E0BF
:100C9000607007202070F8BDE0700620FAE76071F0
:100CA0000520F7E7A070E5700420F3E7552807D189
:100CB0000120EFE7AA2803D10220EBE7032803D0A5
:100CC0002570E570A570F8BD032020702071F8BD77
:100CD000BA020020403A0020783700200400FA05CC
:100CE00000ED00E00FB410B503A9044B044A0298CC
:100CF00000F072F910BC08BC04B01847F5170108E1
:100D00007C0500200FB410B504A9074B02AA039874
:100D100000F062F9044602A9002000F004FD20461C
:100D200010BC08BC04B01847271701087CB515464D
:100D3000024600201C4600290BD0491E009201915A
:100D4000044B6A462146284600F046F9009A0021E5
:100D500011707CBD111701082021020C01D0102157
:100D60001046020A01D010460839020901D0104687
:100D7000091F820801D01046891E420801D0881E32
:100D80007047081A7047F8B5040C8BB2264682B239
:100D90005E430D0C1046370C584336048019002171
:100DA000794116466E43370C360480197941264640
:100DB0006E438919F8BD30B47446641E2578641CEE
:100DC000AB4200D21D46635D5B00E31830BC1847A0
:100DD0008307FF22DB0E9A408907090E99400028FD
:100DE00008DB830809489B001B18186890430843D8
:100DF000186070470007000F0838830804489B00FC
:100E00001B18D86990430843D861704700E400E09C
:100E100000ED00E0004870478005002001480068B0
:100E2000704700008005002002E008C8121F08C1BA
:100E3000002AFAD170477047002001E001C1121F5B
:100E4000002AFBD17047000001490860704700008C
:100E500080050020F0B51FB486B00998089A030DEC
:100E60000021024314D05148514A18185043051428
:100E70001198012810981AD0281A401C00264D4FAE
:100E80004D49009601910490002812DA444211E085
:100E90001198012449A3012801D11098C143069853
:100EA000119A84600360C26041600BB0F0BD4042A3
:100EB000E4E70446210500203F4A001C514103910C
:100EC000029012E0E00707D032463B4601990098B5
:100ED000F4F7FEFA0191009032463B46104619465F
:100EE000F4F7F6FA06460F466410002CEAD104988F
:100EF000039B0028029A0999089806DAF4F7E8FAA1
:100F0000019B009AF4F7E4FA05E0F4F749FB019B32
:100F1000009AF4F745FB04460E460022284BF4F7EE
:100F200013FC03D80020C043014607E00022254BF4
:100F300020463146F4F71AFAF4F784FD102409E04C
:100F4000002C0ADB0A220023F4F7FCF8079B30325E
:100F50001A55641E02460A43F2D11122641C079BF3
:100F6000121B1C19119B012B03D0012308430ED126
:100F70000AE0084304D0112010900020119077E778
:100F80001098151A6D1E0BE01098824202DD0023A6
:100F90006D1C03E0824201DA00236D1E002BEED0AF
:100FA000069811998260C16030C07EE701FCFFFFA6
:100FB000104D0000000014400000F03F3000000021
:100FC0000000F0430000E03F30380A2801D2012041
:100FD0007047002070470000FFB597B00646002517
:100FE00018E2252877D100242746FD49049400E023
:100FF0000443761C32780120203A90400842F7D111
:1010000030782A280ED0022230780146303909295A
:1010100016D804990A235943303940181443761CD2
:101020000490F1E7189802C804911890002904DA96
:101030000120400304434842049002200443761CEC
:1010400030782E2814D1042004437078761C2A2886
:1010500009D11898761C80C8189009E00A214F43DE
:10106000303FC719761C3078014630390929F5D947
:1010700030786C2810D006DC4C281AD068280ED0A6
:101080006A2817D104E0742813D07A2812D110E00E
:101090000120400504430CE00121090501E0032182
:1010A00009050C437178814203D101200005241801
:1010B000761C761C3078119066280BD013DC5828EB
:1010C0007DD009DC00287BD04528F6D04628F4D016
:1010D00047281AD1A5E118E0632835D0642870D0DC
:1010E000652812D19DE170286CD008DC6728F1D00A
:1010F00069287BD06E280DD06F2806D1BAE07328FE
:101100002ED0752871D0782859D01A9A19999047FD
:101110006D1C7EE16002400F022809D003280DD02B
:101120000428189801680DD00D60001D189070E11A
:101130001898EA1701680D604A60F6E71898016888
:101140000D80F2E70D70F0E718986A460178117289
:10115000001D18900020507202A80090012005E0A8
:10116000189802C8189000200091C04361070DD55F
:10117000002101E00199491C0191B94212DA814232
:10118000F8DB009A515C0029F4D10BE0002101E06A
:101190000199491C01918142FADB019A0099895C0D
:1011A0000029F5D1019904981A9B471A214638461F
:1011B000199A00F097FA0199401945180BE04FE091
:1011C0002CE113E04EE0009800990078491C009152
:1011D0001A9A199990470198401E0190401CF2D12B
:1011E000214638461A9B199A10E137E00A2000215F
:1011F000009001916002410F022907D0189A01CA9C
:101200001892C2179446032908D00AE01898C01D06
:10121000C108C90005C91891944607E000B2C21779
:101220009446042902D140B2C1178C46002261467F
:10123000944506DA0A460021404291418C462D2110
:1012400002E0210504D52B216A461173012103E038
:10125000E10701D02021F7E7029155E00A200AE0DA
:10126000102008E010200090002104200443019188
:10127000082703E008200021019100906002410F3F
:10128000022907D0189A01CA18920022944603290D
:1012900008D008E01898C01DC108C90005C91891F8
:1012A000944603E080B2042900D1C0B2002102912B
:1012B000210729D51199702906D0009A1021019B88
:1012C0004A401A4305D00EE040216A4611730121BD
:1012D00008E06146014306D030216A461173119936
:1012E000517302210291009A0821019B4A401A433E
:1012F0000AD16146014301D1610705D530216A4613
:10130000117301217F1E02911199582904D035A132
:101310000E910DA90D910DE037A1F9E76146019BF2
:10132000009AF3F70FFF0E9B8C469B5C0D9A521EA2
:101330000D92137061460143F0D10D9805A9081A6A
:1013400020300190600703D501200004844300E0B1
:1013500001270198874201DD381A00E00020019939
:1013600000904118029809180498401A0490E0036C
:1013700006D421461A9B199A049800F0B3F945192E
:10138000002706E003A81A9AC05D199990476D1CC2
:101390007F1C02988742F5DBE0030CD521461A9B9F
:1013A000199A049800F09EF9451904E01A9A302021
:1013B000199990476D1C0099481E00900029F5DC92
:1013C00008E00D980D990078491C0D911A9A199909
:1013D00090476D1C0199481E01900029F1DC63E1E2
:1013E00009280100303132333435363738396162FB
:1013F00063646566000000003031323334353637BF
:1014000038394142434445460000000000F05AF993
:101410004519761C3078002800D0E2E528461BB03C
:10142000F0BD600700D406271898C01DC108C90088
:1014300048680A680831C30FDB071891190001D00A
:101440009CA108E0210501D59BA104E0E10701D0A2
:101450009AA100E09AA1430011985B0810916528B9
:101460000CD006DC452809D046281DD0472841D19C
:1014700041E0662818D067283CD13CE00021112FBC
:1014800001DB112000E0781C0191009008A911A84F
:10149000FFF7E0FC139905910021119A15927F1C2A
:1014A00012980197009150E00120C007039001209D
:1014B000019008A9009711A8FFF7CCFC139A149982
:1014C00005920022119B009212981593059A0192A1
:1014D000002901D0104602E0791C40180190381A0A
:1014E00001D5019804E04042401E0090781C019014
:1014F000C01B029043E0012F00DA01270021112FC9
:1015000001DD112000E038460191009008A911A8E2
:10151000FFF7A0FC13990591119A002112981592DA
:101520000091019721070CD40599B94201DB01997B
:1015300000E00191012904DD159A491E515C302912
:1015400006D0B84201DA011D05DA0121029115E049
:101550000199491EEDE7002805DC0099411800912A
:101560000199091A03E0019A411C914200DD0191A1
:101570000099401A401C02900120C00703902007E8
:1015800006D402990198814202DB0020C0430290F8
:1015900000206946C87707AF012103980337C907C0
:1015A000884224D0022011902B201290039800280A
:1015B0000CDA404203902D20129007E00A21039894
:1015C000F3F796FD30317F1E039039701199481E54
:1015D00011900029F2DC03980028EFD1791E1298AF
:1015E00008703078202108404530BF1E387006A8AA
:1015F000C01BC01D039010980078002800D0012067
:10160000019941180298C0170918039809180498FD
:10161000401A401E0490E00306D421461A9B199AF2
:10162000049800F05FF8451910980078002803D05E
:101630001A9A199990476D1CE00324D521461A9BEC
:10164000199A049800F04EF845191CE000980028FB
:1016500007DB00990598884203DD1598405C1999CD
:1016600001E0199930201A9A904700986D1C401C8F
:1016700000900298401E0290002804D11A9A2E2051
:10168000199990476D1C0199481E01900029DDDCD5
:1016900005E038781A9A7F1C199990476D1C0399B8
:1016A000481E03900029F4DC21461A9B199A0498DD
:1016B000ACE600002D0000002B0000002000000020
:1016C00000000000F8B5044600251E4617468804B1
:1016D00004D405E039462020B0476D1C641EF9D5BE
:1016E0002846F8BDFFB50446002581B01E46C80354
:1016F00001D5302700E02027880404D505E03846CE
:101700000399B0476D1C641EF9D5284605B0F0BD9D
:101710004A68002A06D00A68531C0B60107048689B
:10172000401E486070470A68531C0B601070704779
:1017300030B583B00446FFF771FB054600200090EA
:101740000246019021466846F4F76DF82846FFF7F7
:101750007BFB0199009803B030BD7D2110B5C90015
:101760004843F5F7E8FF10BD002140E000BF00BF8F
:1017700000BF00BF00BF00BF00BF00BF00BF00BF71
:1017800000BF00BF00BF00BF00BF00BF00BF00BF61
:1017900000BF00BF00BF00BF00BF00BF00BF00BF51
:1017A00000BF00BF00BF00BF00BF00BF00BF00BF41
:1017B00000BF00BF00BF00BF00BF00BF00BF00BF31
:1017C00000BF00BF00BF00BF00BF00BF00BF00BF21
:1017D00000BF00BF00BF00BF00BF00BF00BF00BF11
:1017E00000BF00BF00BF00BF00BF00BF491C814257
:1017F000BCD3704713B501231A4669460248F9F76E
:1018000052F800981CBD0000A806002008B5F7F7A4
:1018100099FAFDF7DDFDFBF75DFA6548016B0122E2
:1018200011430163006B10400022009011460A2012
:10183000F7F72AFC0A20F7F71BFC002211460B20C1
:10184000F7F722FC0B20F7F713FC5A495A480024FB
:1018500012C07F2101608460C4600461FF21446183
:1018600041600838F8F75EF8002801D072B6FEE74C
:10187000FBF78CFBFBF76EFBFBF7ECFAFBF7F2F9DF
:101880004E494F4812C004608461C4614D490462EE
:10189000C1600838F7F71AFB002801D072B6FEE7DE
:1018A000FBF73CFBFBF7F6FA454847491038016067
:1018B000062141604549C1608160F7F7FDF90028C4
:1018C00001D072B6FEE73E48414930300160846085
:1018D000E121C460490204614160846104620C2119
:1018E00044624161F8F7C8FD002801D072B6FEE7F6
:1018F00033490020B831FFF717F836490320FFF7C6
:1019000013F82F4902203031FFF70EF82A49002042
:101910002431FCF72BFA304C0122920221460020A0
:10192000F4F7A6FD0021202322460846FCF7DEF846
:101930000020FCF743F8F5F7EBFDFCF7F9FCFBF7AB
:1019400083FDF6F701F9FBF753F8FEF70DFE0122D0
:101950000520D1030007F7F7A2F9FBF75FF8FF2492
:10196000F5342046F6F762FF00221C491448F7F7C9
:101970001DFB002801D072B6FEE7112000040346CB
:101980001A461146FCF7A6FA2046F6F74FFFFCF779
:10199000BFFA2046F6F74AFFF6F79AF82046F6F720
:1019A00045FFF6F7A3FB0E490870FBF70BFBFCE7BE
:1019B000001002400028004040080020007C004049
:1019C000F0050020FFFF000000300040FF0F000086
:1019D000004800403007002000040050FF7F000056
:1019E0000000002000B585B014216846F3F704FC20
:1019F000F6F7FCFAF8F78AFA00231A461946184651
:101A0000FCF768FA1748F8F7C7FA1648F8F7E2FA49
:101A100014485838F8F706F81348F8F7B1FB12489D
:101A20008830F8F7ADFB10488838F8F7A9FB0F4865
:101A3000016B4908490001630D48009003200190A3
:101A40000020029069460B48F7F746F869460A48B5
:101A5000F7F742F80949012088700146F7F72EFB95
:101A600005B000BDBC080020A80600200010024000
:101A7000FFFF00000004005000080050000000209C
:101A8000F8B5012252022B492B48F5F7E9FE294807
:101A90002A490288044600257926212740348A42B3
:101AA00037D00180264981807D21C900C1800A216B
:101AB00001811E214581C94381810121C181858325
:101AC000618302220287782242878187C187E5826B
:101AD00025846584A584C583A5802721E1846A21A6
:101AE0002185D22161850D21A1851649E185668672
:101AF000A786E221E1862A212187134961874B21AC
:101B0000C9002186E121C900E1870521818200F019
:101B10001FF86584A5842584608E0C49884207D10E
:101B20006686A786E220E0862A202087064860870E
:101B3000F8BD00007837002000F80108AA55000021
:101B400072180000581B00004F230000FFFF000028
:101B500070B572B601250C4E6D0229463046F5F778
:101B60005FFE044607E029463046F5F759FE044675
:101B7000C820F5F7D9FD002CF5D02A460349304698
:101B8000F5F7F8FE62B670BD00F80108783700205E
:101B9000002100E0491C8142FCD370470000000096
:101BA00000000000010203040607080903040608F8
:101BB0000C10182030000000000102030400000097
:101BC000E02601080200000098260108020000003B
:101BD0003824010803000000EC270108030000007E
:101BE000C423010807000000CC23010808000000FE
:101BF0008424010809000000282401080A000000CC
:101C0000402301080B000000142401080C00000010
:101C1000A424010810000000E023010811000000C6
:101C2000302401081200000090260108180000006E
:101C3000E426010819000000FC230108160000003A
:101C40001822010814000000042201081A000000F4
:101C50007823010817000000842301081B000000FE
:101C6000982801081C000000702401081D000000D5
:101C7000F02301081E000000642401081F0000007A
:101C800078240108200000006423010821000000DE
:101C90008C230108220000009C230108230000007F
:101CA0004C23010824000000E8230108250000005F
:101CB0002423010826000000F0210108270000006D
:101CC0000824010828000000B823010829000000AA
:101CD0001C2401082A000000582301082B000000E2
:101CE000342301082C000000442401082D000000CA
:101CF000982401082E0000008C2401082F00000009
:101D0000D4230108300000005824010831000000ED
:101D1000702301081500000090290108320000001E
:101D20005024010833000000AC23010834000000F7
:101D30002822010835000000482201083600000072
:101D400060220108370000007822010838000000F6
:101D50009022010839000000A82201083A00000082
:101D6000C02201083B000000D82201083C0000000E
:101D7000F02201083D000000082301083E00000099
:101D8000202301083F00000094290108B828010819
:101D9000CC260108D827010820290108BC27010802
:101DA000B8260108282601083C260108F028010869
:101DB000A82701088C2701086027010804290108C9
:101DC0006829010808270108682601080C2801086D
:101DD000F4270108E0240108C42401086C25010847
:101DE0004C27010880250108A0260108F0260108DB
:101DF000FC2501085825010880280108C42801088D
:101E00001C270108A0280108D8280108402501083E
:101E100094250108B0250108102501087C26010839
:101E2000A82401086828010834270108E4250108CE
:101E30007427010828250108F8240108242801082E
:101E400050290108382901085026010850280108A6
:101E50007C2901083C280108CC250108102601082E
:101E6000342201084C220108642201087C22010866
:101E700094220108AC220108C4220108DC220108D6
:101E8000F42201080C2301082C2A0108000000009C
:101E9000B81E010801690008AC2A0108881E010863
:101EA000B81E01089D670008502A0108881E010815
:101EB0000000000015680008702A0108981E01083B
:101EC0000000000065680008DC2A0108981E01086F
:101ED0000000000009620008102B0108981E01088C
:101EE00000000000C5700008C82A0108981E0108FB
:101EF00000000000C5600008442A0108881E01088F
:101F00000000000081670008F02A0108881E01080F
:101F1000C01F0108CD690008B82A0108081F010880
:101F200000000000BD640008002B0108081F010824
:101F3000381F010809670008602A0108281F0108E6
:101F40000000000095660008082A010888130000B8
:101F500001000000F42901088813000001000000BE
:101F6000E82901088813000001000000002A010888
:101F70008813000001000000C82901088813000030
:101F800001000000B82901088813000001000000CA
:101F9000D82901088813000001000000A0290108C9
:101FA00060EA000003000000142A010860EA000053
:101FB00003000000202A0108E803000005000000DB
:101FC000282B0108081F010800000000356A0008DE
:101FD0006C2B0108281F010800000000F16D0008AB
:101FE000882B0108281F010800000000616E00080E
:101FF000A02B0108281F010800000000416C000808
:10200000582B0108281F0108000000007D6B000804
:10201000402B0108281F010800000000E16E0008A5
:102020002052D800001000000080000000000100D5
:10203000782D0108D9ED0008702D0108C5E50008CC
:102040005C2D010869E50008AC2C0108EDE40008EE
:10205000542D010865E50008F42C01083DEB00084B
:10206000EC2C010821E20008E02B010825DF000824
:10207000C82C010855E10008842C01080DE1000876
:10208000282D010869DF0008382D010845E4000803
:10209000D42C0108B5E40008902C01087DE4000868
:1020A000502C0108DDED0008582C010891EC0008C7
:1020B000482D0108EDEB0008E82B010831ED000880
:1020C000442C010859EB0008F42B0108A1DF00089B
:1020D000642C010899E10008742C0108D1E500087E
:1020E000D42B010889E00008E02C010851E9000820
:1020F000082D0108F5EA0008142D0108ADEA0008D2
:10210000A02C010885E80008202C010895E60008AD
:102110008C2D010881E70008002C0108F5E7000874
:10212000102C01081DEA0008FC2C01080DE700082E
:10213000C42B010841E40008C82B01083DE4000855
:102140009C2C010845E30008BC2C0108B5E30008FD
:10215000642D0108E9E30008342C010865DF00085C
:10216000802D0108D5ED000800404040404040402F
:10217000404041414141414040404040404040405A
:1021800040404040404040404005020202020202FE
:10219000020202020202020202202020202020204D
:1021A0002020200202020202020290909090909061
:1021B000101010101010101010101010101010101F
:1021C0001010101002020202020288888888888893
:1021D000080808080808080808080808080808087F
:1021E00008080808020202024000000069210108F4
:1021F0002B51495552433A202270647064656163E3
:10220000742200002B51495552433A2022636C6FCF
:10221000736564222C0000002B51495552433A202B
:102220002272656376222C002B5245434549564560
:102230002C000000414952373830455F4556454E25
:10224000545F4E554D5F3000300000004149523719
:102250003830455F4556454E545F4E554D5F310011
:1022600031000000414952373830455F4556454EF0
:10227000545F4E554D5F32003200000041495237E5
:102280003830455F4556454E545F4E554D5F3300DF
:1022900033000000414952373830455F4556454EBE
:1022A000545F4E554D5F34003400000041495237B1
:1022B0003830455F4556454E545F4E554D5F3500AD
:1022C00035000000414952373830455F4556454E8C
:1022D000545F4E554D5F360036000000414952377D
:1022E0003830455F4556454E545F4E554D5F37007B
:1022F00037000000414952373830455F4556454E5A
:10230000545F4E554D5F3800380000004149523748
:102310003830455F4556454E545F4E554D5F390048
:10232000390000002B5147505358545241444154F6
:10233000413A00002B514D545355423A00000000E1
:102340002B43495047534D4C4F433A002B51475074
:10235000534C4F433A0000002B514D5444495343D2
:102360003A0000002B5148545450524541443A0021
:102370002B434349443A00002B514953454E443ABC
:10238000000000002B514952443A00002B514854A0
:1023900054505245414446494C453A002B5148540B
:1023A0005450504F535446494C453A002B514C54CD
:1023B0004F4E453A000000002B514D54434C4F53B3
:1023C000453A00002B435245473A00002B43475201
:1023D00045473A002B514D5450494E473A000000B2
:1023E0002B434D54493A00002B43434C4B3A0000D9
:1023F0002B51464F50454E3A000000002B51494F9B
:1024000050454E3A000000002B514D544F50454E60
:102410003A0000002B4350494E3A00002B514D54D6
:10242000434F4E4E3A0000002B4353513A000000F8
:102430002B434D47523A00002B434D452045525205
:102440004F523A002B514D54554E533A0000000064
:102450002B435454533A00002B514D545354415480
:102460003A0000002B51485454504745543A00005C
:102470002B51464C53543A002B5148545450504F12
:1024800053543A002B43474154543A002B514D5476
:10249000524543563A0000002B514D545055424589
:1024A000583A00003E000000414952373830455F3D
:1024B0004556454E545F514750535854524144413C
:1024C00054410000414952373830455F4556454E2A
:1024D000545F4E45575F49505F44415441000000EE
:1024E000414952373830455F4556454E545F534D4C
:1024F000535F444154410000414952373830455FF1
:102500004556454E545F514D54535542000000000E
:10251000414952373830455F4556454E545F514723
:1025200050534C4F43000000414952373830455F0B
:102530004556454E545F514D5444495343000000A5
:10254000414952373830455F4556454E545F5148F2
:102550005454505245414400414952373830455F48
:102560004556454E545F524541440000414952375B
:102570003830455F4556454E545F4343494400005B
:10258000414952373830455F4556454E545F5345B3
:102590004E440000414952373830455F4556454E5C
:1025A000545F51485454505245414446494C4500AB
:1025B000414952373830455F4556454E545F514882
:1025C000545450504F535446494C4500414952379A
:1025D0003830455F4556454E545F514C544F4E453B
:1025E00000000000414952373830455F4556454E9E
:1025F000545F514D54434C4F5345000041495237AD
:102600003830455F4556454E545F434C4F53450067
:10261000414952373830455F4556454E545F524523
:102620004345495645000000414952373830455F1F
:102630004556454E545F4352454700004149523785
:102640003830455F4556454E545F43475245470035
:10265000414952373830455F4556454E545F514DDC
:102660005450494E47000000414952373830455FC9
:102670004556454E545F41434B0000004149523797
:102680003830455F4556454E545F43434C4B000040
:1026900053454E44204F4B0053485554204F4B0058
:1026A000414952373830455F4556454E545F534592
:1026B0004E445F4F4B000000414952373830455F70
:1026C0004556454E545F4F4B000000004849444F6B
:1026D0005F41545F4556454E545F4F4B000000002C
:1026E0004F4B000053454E44204641494C000000EA
:1026F000414952373830455F4556454E545F534542
:102700004E445F4641494C002D41495237383045CF
:102710005F4556454E545F504F4C4C00414952372F
:102720003830455F4556454E545F51464F50454EF3
:1027300000000000414952373830455F4556454E4C
:10274000545F514D544F50454E000000414952379F
:102750003830455F4556454E545F4F50454E00005A
:10276000414952373830455F4556454E545F4350D6
:10277000494E0000414952373830455F4556454E75
:10278000545F514D54434F4E4E0000004149523763
:102790003830455F4556454E545F4C42535F4C4F71
:1027A000434154494F4E0000414952373830455F4C
:1027B0004556454E545F4353510000004849444F2D
:1027C0005F41545F4556454E545F53454E445F4507
:1027D00052524F52000000004849444F5F41545F3D
:1027E0004556454E545F4552524F52004552524F46
:1027F00052000000414952373830455F4556454E3A
:10280000545F524541445F534D5300004149523794
:102810003830455F4556454E545F4E45575F534DE2
:1028200053000000414952373830455F4556454E08
:10283000545F514D54554E530000000041495237EA
:102840003830455F4556454E545F5154545300004F
:10285000414952373830455F4556454E545F514DDA
:102860005453544154000000414952373830455FB9
:102870004556454E545F5044504445414354000032
:10288000414952373830455F4556454E545F434FB6
:102890004E4E454354000000434F4E4E45435400B6
:1028A000414952373830455F4556454E545F51488F
:1028B00054545047455400004556454E545F4558C2
:1028C00049540000414952373830455F4556454E1E
:1028D000545F51464C535400414952373830455F9C
:1028E0004556454E545F5148545450504F53540030
:1028F000414952373830455F4556454E545F43474E
:1029000041545400414952373830455F4556454E91
:10291000545F494E49545F54494D454F555400004A
:102920004849444F5F41545F4556454E545F5449B2
:102930004D454F5554000000414952373830455FEE
:102940004556454E545F514D545245435600000084
:10295000414952373830455F4556454E545F514DD9
:102960005450554245580000414952373830455F70
:102970004556454E545F44454C41590041495237F4
:102980003830455F4556454E545F5244590000006B
:10299000524459004556454E545F454E54525900D5
:1029A00041542B435354543D222573222C22222C74
:1029B00022220D0A0000000041542B434950525876
:1029C000463D310D0A00000041542B434647524911
:1029D0003D310D0A0000000041542B4349504D5534
:1029E000583D310D0A00000041542B434349440D2A
:1029F0000A00000041542B43494D490D0A000000D4
:102A00004154490D0A00000041542B4347534E0DD9
:102A10000A00000041542B43494943520D0A00006B
:102A200041542B43494653520D0A00004149523745
:102A3000383045004149523738304552756E41545F
:102A4000436D64004149523738304549646C650034
:102A500041495237383045506F7765724F6666008E
:102A6000414952373830454950506F6C6C00000076
:102A700041495237383045506F7765724F6E0000CC
:102A800041495237383045436C6F736557697265F9
:102A90006C65737300000000414952373830454F70
:102AA00070656E576972656C657373004149523782
:102AB000383045496E6974004149523738304549CC
:102AC00050496E6974000000414952373830454121
:102AD00054436D64496E69740000000041495237E7
:102AE0003830454154436D645465737400000000F0
:102AF0004149523738304552656164790000000021
:102B00004149523738304549505265616479000077
:102B1000414952373830455761697453696D436193
:102B200072645265616479004149523738304553C7
:102B30006561726368696E674E6574776F726B006A
:102B400041495237383045536F636B657453656E36
:102B50006444617461000000414952373830455384
:102B60006F636B6574436C6F736500004149523746
:102B7000383045536F636B65744865617274436F99
:102B80006E6669670000000041495237383045538E
:102B90006F636B657448656172746265617400008F
:102BA00041495237383045536F636B6574436F6EDC
:102BB0006E65637400000000414952373830454368
:102BC000535100006F7461006C6F675F75706C6FBC
:102BD000616400006465766963655F696400000094
:102BE00061745F636D6400007463705F73656E642D
:102BF000000000006462675F6D6F646500000000A4
:102C00007365745F7274636D6D6F646500000000BE
:102C10007365745F757762656E61626C6500000054
:102C20007365745F67707375706461746574696DE2
:102C300065000000617564696F5F766F6C756D6526
:102C4000000000007463705F636C6F7365000000C8
:102C500075706461746500007463705F63726561B0
:102C6000746500006770735F626175645F726174A0
:102C7000650000007365745F6461746172617465FE
:102C80000000000064656275675F6F6666000000A3
:102C900034675F706F7765726F6666006C6F670090
:102CA0007365745F7274636D000000007274635F1B
:102CB0007365745F616C61726D0000006C6F675FBB
:102CC000636C65616E00000064656275675F6F6EBE
:102CD0000000000034675F706F7765726F6E0000F0
:102CE0007365727665725F696E666F00696E666F96
:102CF00000000000736C6565700000007365745F10
:102D00006E747269700000007365745F6770735F42
:102D1000730000007365745F636861696368756759
:102D200070735F7300000000636C6F73655F776999
:102D300072656C65737300006F70656E5F776972A2
:102D4000656C6573730000007463705F636F6E6E13
:102D5000656374007274635F676574007274635FA7
:102D6000736574006C6F675F7072696E7400000049
:102D70007265626F6F740000746573740000000008
:102D80007474735F706C6179000000007365745F28
:102D90007178777A00000000636C65617200000052
:102DA0006C730000C42D01080000002084050000A1
:102DB000D85F00085C2E01088405002084400000D4
:102DC000380E0108011858152443434D53472C521F
:102DD0004D432C312C302C2A30340D0A145C4753CF
:102DE00041149A44144A56148B3141145B4C4C14D0
:102DF0007A46145C5458543C041C300D0A3201923B
:102E00000402492085342A010813DD699B088010DB
:102E10001329639B08981013C167790C011C8BB8A8
:102E20002B340B246162340916F409131879194BF9
:102E3000C8420401200A16644B1103CD55AA091794
:102E4000E80118320217982D0108D1BD1B08A0080F
:0C2E5000132DBF02FF0801FF0176B20144
:04000005080050C1DE
:00000001FF
